:100000000C94861B0C94B71B0C94B71B0C94B71B59
:100010000C94B71B0C94B71B0C94B71B0C94B71B18
:100020000C94B71B0C94B71B0C94B71B0C94B71B08
:100030000C94B71B0C94B71B0C94B71B0C94B71BF8
:100040000C94B71B0D9471000C94B71B0C94B71B48
:100050000C94B71B0C94B71B0C94FDA80D94FD02D7
:100060000C94B71B0C94E6560C94DC560C94B71BFE
:100070000C94B71B0C94B71B0C94B71B0C94B71BB8
:100080000C94B71B0C94B71B0C94B71B0C94B71BA8
:100090000C94B71B0C94B71B0C94B71B0C94B71B98
:1000A0000C94B71B0C94B71B0C94B71B0C94B71B88
:1000B0000C94B71B0C94B71B0C94B71B0C94B71B78
:1000C0000C94B71B0C94B71B0C94B71B0C94B66F15
:1000D0000C948C6F0C94B71B0C94B71B0C94B71B2F
:1000E0000C94B71B511C971C9D1CC41CD11CDA1C02
:1000F000E51CCE24E025BD26E82628332833032836
:10010000A428BC2528332833912A3F2C772C283368
:100110009D2E28332833F02F283328337F30B230F8
:10012000283380313B3219571F57315741574957B0
:1001300076574D57765751575557765759575D57FC
:10014000615769577657735727B649B669B68EB661
:10015000B3B66AB8D8B6FBB61EB743B768B78DB7A3
:10016000B2B7D7B76AB8FCB721B846B8DAB9DDB9C3
:10017000E1B9E4B9E7B911BAEBB9EEB9F2B9F5B939
:10018000F8B9FCB9FFB902BA11BA06BA09BA0CBA81
:1001900009CA0CCAFBC9FFC905CA43CA10CA14CA96
:1001A0001ACA1ECA22CA28CA2CCA30CA43CA36CAA8
:1001B0003ACA3ECA8AD18FD194D19ED1A8D121D238
:1001C000B2D1BAD1C2D1CCD1D6D1E0D1EFD1F9D10F
:1001D00021D203D20DD217D2084AD73B3BCE016EB3
:1001E00084BCBFFDC12F3D6C74319ABD56833DDA8E
:1001F0003D00C77F11BED9E4BB4C3E916BAAAABE9D
:10020000000000803F05A84CCDB2D44EB93836A9C5
:10021000020C50B9918688083CA6AAAA2ABE000002
:1002200000803F000C94BD260C9430CA0C94FCB79F
:100230000C949D1C0C94AD6E0D94F90D0C94F9D199
:100240000C94EBB90C947F300C94D7B70C94756E6A
:100250000C9403D20C9403280C94FFC90C94BC2575
:100260000C9421B80C94E4B90C94B2D10C944D5771
:100270000C943ECA0C943ACA0C9411BA0C948DB7E3
:100280000C94772C0D941A0C0C9436CA0C94FCB96F
:100290000C94EEB90C949D2E0C9455570C948EB67C
:1002A0000C9405CA0C94166E0C94A8D10C9468B7E3
:1002B0000C94FFB90C94E7B90C945D570C9431572A
:1002C0000C948AD10C94E51C0C9476570C9417D29C
:1002D0000C9480310C9446B80C9414CA0C94C2D17E
:1002E0000C9449570C941ECA0C948FD10C94912AEB
:1002F0000C9427B60C94676E0C9422CA0C94615728
:100300000C94E1B90C94D6D10C9473570C9443B768
:100310000C94D11C0C941F570C9409BA0C94F5B989
:100320000C9459570C94E0250C9406BA0C94A4280C
:100330000C94C41C0C9409CA0C94CE240C94F2B9ED
:100340000C94F02F0C94F8B90C94DDB90C94FBC903
:100350000C941ACA0C94E0D10C9402BA0C94D8B63E
:100360000C9428330C946AB80C94FBB60C949ED170
:100370000C940DD20C9441570C94DAB90C94446E41
:100380000C9419570C9449B60C9428CA0C94536ECB
:100390000C94B3B60C9469570C94971C0C94FA6E99
:1003A0000C94EFD10C940CCA0C9421D20C9494D1DF
:1003B0000C9443CA0C940CBA0C9451570C94CCD1A5
:1003C0000C941EB70C94B2B70C943F2C0C94DA1C0E
:1003D0000C94B2300C9410CA0C943B320C94BAD1E9
:1003E0000C9469B60C942CCA0C94511C0C94E826FD
:1003F0004E414E494E495459494E46CDCCCC3D0A0A
:10040000D7233C17B7D13877CC2B329595E6241FEC
:10041000B14F0A000020410000C84200401C4620A5
:10042000BCBE4CCA1B0E5AAEC59D7400407A10F378
:100430005A00A0724E18090010A5D4E80000E87612
:1004400048170000E40B54020000CA9A3B00000069
:10045000E1F505000080969800000040420F000082
:1004600000A08601000000102700000000E8030043
:100470000000006400000000000A0000000000010D
:1004800000000000002C76D888DC674F0823DFC10D
:10049000DFAE59E1B1B796E5E3E453C63AE65199C8
:1004A0007696E8E6C28426EB898C9B62ED407C6FF1
:1004B000FCEFBC9C9F40F2BAA56FA5F490055A2AA8
:1004C000F75C936B6CF9676DC11BFCE0E40D47FEB4
:1004D000F520E6B500D0ED902E03009435770500A9
:1004E00080841E080000204E0A000000C80C333330
:1004F00033330F986E12831141EF8D2114893BE63F
:100500005516CFFEE6DB18D1844B381BF77C1D90C7
:100510001DA4BBE424203284725E228100C9F12430
:10052000ECA1E53D274D323520500A4D32340052C2
:100530006573756D65005549205061757365004E92
:100540006F204D61746368203A004D333033452D80
:1005500031533635433455004D393939004D353036
:10056000320A4D353030004D33303345305332315F
:1005700035433855000A202A2A2A7265636461745B
:100580002E646174615B305D203D004732380A475C
:1005900031204631303030205A313000556E73757D
:1005A00070706F72746564204F7074696F6E205341
:1005B000656C6563746564004732380047312046D6
:1005C00031303030205A302E30004732380A47312F
:1005D000204631303030205A302E30004D3530300A
:1005E000005A204F6666736574203A202573004DCB
:1005F000353030005A204F6666736574203A2025E6
:1006000073004732385A0A473146313530305A3054
:100610002E30004732380A473146313530305A30B3
:100620002E30004D383400473146313030305A30AA
:100630002E30004732380A473146313030305A3098
:100640002E30005A204F6666736574203A20257359
:10065000004D353030004D383400426567696E53C7
:100660007769746368007265636461742E616464A1
:1006700072203D3D007265636461742E6461746133
:100680005B305D203D3D0077616974776179203D85
:100690003D000A202A2A2A4E6F7A7A6C6554656DCD
:1006A000705374617475735B325D203D00434F4D30
:1006B0004D554E49434154494F4E004452595255AD
:1006C0004E004552524F525300494E464F0045434B
:1006D000484F0047322F47332062616420706172B7
:1006E000616D65746572730A00536C6565702E2EBA
:1006F0002E005A2050726F62652050617374204240
:1007000065640A005A2050726F62652050617374EC
:100710002042656400486F6D652058592046697213
:1007200073740A00486F6D652058592046697273CA
:100730007400206F6620004D424C204732392070F3
:100740006F696E742000290A004A206F7574206F4B
:10075000662072616E67652028302D00290A0049E5
:10076000206F7574206F662072616E676520283077
:100770002D004D6573682070726F62696E6720642A
:100780006F6E652E0A005374617274206D65736814
:100790002070726F62696E672077697468202247E3
:1007A0003239205331222066697273742E0A004751
:1007B00032380A47323920533200686173206E6F35
:1007C00020646174612E0A004D657368204265647F
:1007D000204C6576656C696E67200053206F7574D8
:1007E000206F662072616E67652028302D35292EB6
:1007F0000A004D65736820706F696E742063616EC6
:100800006E6F74206265207265736F6C7665640A22
:10081000004D302F3120427265616B2043616C6C5A
:10082000656400436F6E74696E7565004D302F31DD
:1008300020427265616B2043616C6C6564004E6F91
:10084000204D6F76652E00456E642066696C6520CC
:100850006C6973740A00426567696E2066696C652D
:10086000206C6973740A004469736D697373005274
:100870006573756D696E6720534400286E6F20663E
:10088000696C65290043757272656E742066696CC7
:10089000653A20002E0A0044656C6574696F6E200D
:1008A0006661696C65642C2046696C653A20004677
:1008B000696C652064656C657465643A00507269A2
:1008C0006E742074696D653A20000A537461747304
:1008D0003A2046696C616D656E7420757365643A83
:1008E00020002C204C6F6E67657374206A6F623A2B
:1008F0002000546F74616C2074696D653A20005358
:10090000746174733A20002C204661696C65643A06
:1009100020002C2046696E69736865643A20005097
:1009200072696E74733A200053746174733A2000D4
:100930006F6B006F666600CE06C906C206BB06ADC9
:100940000644454255473A004D3131332053004269
:10095000656420436F6F6C696E672E2E2E004265B2
:10096000642048656174696E672E2E2E00434841ED
:100970004D4245525F54454D5045524154555245A4
:10098000004D4F54494F4E5F4D4F4445530054481E
:1009900045524D414C5F50524F54454354494F4E80
:1009A000004155544F5245504F52545F53445F538A
:1009B00054415455530050524F4D50545F5355506D
:1009C000504F525400454D455247454E43595F5094
:1009D000415253455200434153455F4C49474854A7
:1009E0005F4252494748544E45535300544F47477E
:1009F0004C455F4C494748545300534F4654574168
:100A000052455F504F574552004255494C445F5044
:100A1000455243454E54004C4556454C494E475F60
:100A200044415441005A5F50524F42450041555491
:100A30004F4C4556454C005052494E545F4A4F4228
:100A40000050524F4752455353004155544F524561
:100A5000504F52545F54454D5000564F4C554D45E4
:100A60005452494300454550524F4D0042494E4172
:100A700052595F46494C455F5452414E5346455288
:100A80000053455249414C5F584F4E5F584F4646C0
:100A9000004649524D574152455F4E414D453A4DF2
:100AA00061726C696E20322E305F44573420544D91
:100AB00033442053534D444E4E20534F55524345DB
:100AC0005F434F44455F55524C3A68747470733AB3
:100AD0002F2F6769746875622E636F6D2F496E736F
:100AE000616E6974794175746F6D6174696F6E2F91
:100AF0004D61726C696E2F747265652F437265610A
:100B00006C6974795F4D61726C696E322E302E782B
:100B10002050524F544F434F4C5F56455253494F0C
:100B20004E3A312E30204D414348494E455F54598D
:100B300050453A544D33442043522D582045585483
:100B400052554445525F434F554E543A3220555505
:100B500049443A63656465326132662D34316132ED
:100B60002D343734382D396231322D6335356336C3
:100B7000326633363766660A002F2F200020466C17
:100B80006F773A200050726F74656374656420500B
:100B9000696E0A004261627973746570205A004D73
:100BA000424C2041646A757374205A00496E766124
:100BB0006C69642065787472756465720A002064DB
:100BC0003A0020693A0020703A0020643A00206917
:100BD0003A0020703A0064697300656E0043290A88
:100BE0000061626C656420286D696E2074656D70AB
:100BF0002000436F6C64206578747275646573209F
:100C0000617265200046696C616D656E7420727555
:100C10006E6F75742064697374616E636520286DEE
:100C20006D293A200046696C616D656E742072759D
:100C30006E6F757420004F66667365747320417023
:100C4000706C696564004572723A20546F6F20665B
:100C500061722100546F6F206661722066726F6D41
:100C6000207265666572656E636520706F696E746B
:100C70000A00454550524F4D204F4B0A00416476C3
:100C8000616E6365204B003F4B2076616C7565207B
:100C90006F7574206F662072616E67652028302D35
:100CA0003130292E0A003F542076616C7565206F23
:100CB0007574206F662072616E67652E0A0045723A
:100CC000726F722077726974696E6720746F204545
:100CD0004550524F4D210A00363726033C3D380E11
:100CE0002E303E121A1C1824221E08440AFF430804
:100CF00009070001627573793A2070617573656444
:100D000020666F7220696E7075740A00627573795F
:100D10003A2070617573656420666F722075736523
:100D2000720A00627573793A2070726F636573732B
:100D3000696E670A007061757365004D363030006A
:100D40002066696C616D656E745F72756E6F757427
:100D5000200066696C616D656E745F72756E6F758B
:100D60007420540046696C616D656E7452756E6FC7
:100D7000757420540053544F505045442E20005059
:100D800072696E7465722073746F7070656420642C
:100D9000756520746F206572726F72732E204669BC
:100DA0007820746865206572726F7220616E6420AD
:100DB000757365204D39393920746F2072657374ED
:100DC0006172742E202854656D706572617475723D
:100DD000652069732072657365742E2053657420D5
:100DE00069742061667465722072657374617274CF
:100DF000696E67290A004E6F20436865636B7375DF
:100E00006D2077697468206C696E65206E756D62FF
:100E100065722C204C617374204C696E653A200019
:100E20004E6F20436865636B73756D2077697468D6
:100E3000206C696E65206E756D6265722C204C6148
:100E40007374204C696E653A2000636865636B7348
:100E5000756D206D69736D617463682C204C6173CE
:100E600074204C696E653A20004C696E65204E75A1
:100E70006D626572206973206E6F74204C617374AB
:100E8000204C696E65204E756D6265722B312C2089
:100E90004C617374204C696E653A20004D313130DD
:100EA00000776169740A004D313137004D333100EC
:100EB00053442072656164206572726F720A004447
:100EC0006F6E65207072696E74696E672066696CFA
:100ED000650A004B494C4C20636175736564206260
:100EE0007920746F6F206D75636820696E6163741B
:100EF0006976652074696D65202D20637572726551
:100F00006E7420636F6D6D616E643A200065636876
:100F10006F3A004572726F723A0024F4D43050C3B5
:100F20008E20C2A24017828B7011127A910D816CB3
:100F3000D90AA861E108C7586607615143061E4BEC
:100F40005D05C145A7041A411104093D9803713993
:100F500031034036DB0265339102D4305402802ED7
:100F60001D02632CEE01752AC501B028A0011027CF
:100F700081018F2564012B244B01E0223401AC2137
:100F80001F018D200D01801FFC00841EED00971DA8
:100F9000DF00B81CD200E61BC600201BBC00641A90
:100FA000B200B219A8000A19A0006A189900D11756
:100FB000910040178B00B516840031167E00B315E2
:100FC00079003A157300C7146F0058146A00EE13C5
:100FD00066008813630025135E00C7125B006C1265
:100FE000570015125400C111510070114F0021110A
:100FF0004B00D61049008D104700461044000210E7
:101000004200C00F4000800F3E00420F3C00060F20
:101010003B00CB0E3800930E37005C0E3500270ED8
:101020003400F30D3200C10D3100900D3000600D21
:101030002E00320D2D00050D2C00D90C2B00AE0C0E
:101040002900850C29005C0C2700350C27000E0CAC
:101050002600E80B2400C40B2400A00B23007D0B0A
:1010600023005A0B2100390B2100180B2000F80A2D
:101070001F00D90A1E00BB0A1E009D0A1D00800A1F
:101080001D00630A1C00470A1B002C0A1B00110AE2
:101090001A00F7091A00DD091900C4091900AB0983
:1010A0001900920917007B091800630917004C0901
:1010B000160036091600200916000A091500F50861
:1010C0001500E0081400CC081400B8081400A408A7
:1010D0001400900813007D0812006B0813005808D4
:1010E00012004608120034081100230811001208EB
:1010F000110001081100F0071000E0071000D007F0
:101100001000C0071000B0070F00A10710009107E2
:101110000E0083070F0074070F0065070E005707C6
:101120000E0049070E003B070D002E070E0020079A
:101130000D0013070D0006070D00F9060C00ED0663
:101140000D00E0060C00D4060C00C8060C00BC061E
:101150000C00B0060C00A4060B0099060C008D06CE
:101160000B0082060B0077060B006C060B00610675
:101170000A0057060B004C060A0042060A00380611
:101180000A002E060A0024060A001A060A001006A3
:10119000090007060A00FD050900F4050900EB0532
:1011A0000900E2050900D9050900D0050900C705B5
:1011B0000900BE050900B5050800AD050800A50534
:1011C00009009C050800940508008C0508008405AA
:1011D00008007C050800740508006C05070065051B
:1011E00008005D050700560508004E050700470585
:1011F00007004005080038050700310507002A05EB
:101200000700230507001C050600160507000F054B
:1012100007000805060002050700FB040600F504A8
:101220000700EE040600E8040600E2040700DB0401
:101230000600D5040600CF040600C9040600C30456
:101240000600BD040600B7040600B1040500AC04A6
:101250000600A6040600A00405009B0406009504F1
:101260000500900406008A0405008504050080043A
:1012700006007A04050075040500700405006B047F
:10128000050066040500610405005C0405005704C0
:101290000500520405004D04050048040500430400
:1012A00005003E0404003A0405003504050030043E
:1012B00004002C04050027040400230405001E0478
:1012C00004001A04040016040500110404000D04AF
:1012D0000400090405000404040000040400FC03E5
:1012E0000400F8030400F4030400F0030400EC031A
:1012F0000400E8030400E4030400E0030400DC034A
:101300000400D8030400D4030400D0030400CC0379
:101310000400C8030300C503030024F404D9201B00
:10132000C40C5C0E9804C4095F0265077101F405E2
:10133000F900FB04B30048048700C10369005803A7
:10134000550003034500BE023A00840231005302F7
:101350002A002902250004022000E4011C00C80123
:101360001900AF01170098011400840113007101E6
:1013700010006101100051010E0043010D00360103
:101380000B002B010B0020010B00150109000C01C3
:10139000090003010800FB000800F3000800EB004F
:1013A0000700E4000600DE000600D8000600D200B8
:1013B0000600CC000500C7000500C2000500BD0006
:1013C0000400B9000400B5000400B1000400AD0041
:1013D0000400A9000400A5000300A20003009F0070
:1013E00004009B0003009800030095000200930096
:1013F0000300900003008D0002008B0003008800B2
:1014000002008600020084000300810002007F00C9
:1014100002007D0002007B000200790002007700DC
:1014200001007600020074000200720001007100E9
:1014300002006F0002006D0001006C0002006A00F3
:1014400001006900020067000100660001006500FC
:101450000100640002006200010061000100600000
:1014600001005F0002005D0001005C0001005B0004
:1014700001005A0001005900010058000100570006
:101480000100560001005500010054000100530006
:101490000000530001005200010051000100500003
:1014A00001004F0001004E0000004E0001004D0001
:1014B00001004C0001004B0000004B0001004A00FD
:1014C00001004900010048000000480001004700F9
:1014D00001004600000046000100450000004500F4
:1014E00001004400010043000000430001004200ED
:1014F00000004200010041000000410001004000E6
:1015000001003F0000003F0001003E0000003E00DF
:1015100001003D0000003D0001003C0000003C00D7
:1015200000003C0001003B0000003B0001003A00CD
:1015300000003A00010039000000390001003800C5
:1015400000003800000038000100370000003700BC
:1015500001003600000036000000360001003500B2
:1015600000003500000035000100340000003400A8
:10157000000034000100330000003300000033009D
:101580000100320000003200000032000100310092
:101590000000310000003100010030000000300088
:1015A0000000300001002F0000002F0000002F007D
:1015B00000002F0001002E0000002E0000002E0071
:1015C00001002D0000002D0000002D0000002D0066
:1015D00001002C0000002C0000002C0000002C005A
:1015E00001002B0000002B0000002B0000002B004E
:1015F00001002A0000002A0000002A0000002A0042
:101600000100290000002900000029000000290035
:101610000000290001002800000028000000280028
:10162000000028000000280001002700000027001B
:10163000000027000000270000002700010026000E
:101640000000260000002600000026000000260002
:1016500001002500000025000000250000002500F5
:1016600000002500000025000100240000002400E7
:1016700000002400000024000000240001002300DA
:1016800000002300000023000000230000002300CE
:1016900000002300000023000100220000002200BF
:1016A00000002200000022000000220000002200B2
:1016B00001002100000021000000210000002100A5
:1016C0000000210000002100000021000100200096
:1016D000000020000000200000002000000020008A
:1016E00000002000000020000000200001001F007A
:1016F00000001F0000001F0000001F0000001F006E
:1017000000001F0000001F0001001E0000001E005E
:1017100000001E0000001E000000232C0000B82264
:101720000000561800003A0F0000B8080000B1048D
:101730000000710200003E0100002020506C616E2C
:101740006E657242756666657242797465733A2099
:10175000002046726565204D656D6F72793A2000F4
:10176000436F6D70696C65643A204F637420323743
:1017700020323031390A00204C6173742055706476
:10178000617465643A20323031392D31302D303575
:10179000207C20417574686F723A2054696E794DCF
:1017A000616368696E657333440A00322E305F44AA
:1017B00057340A004D61726C696E0020536F667475
:1017C000776172652052657365740A0020576174F1
:1017D0006368646F672052657365740A0020427203
:1017E0006F776E206F75742052657365740A0020E0
:1017F00045787465726E616C2052657365740A0079
:10180000506F77657255700A0073746172740A00C4
:101810006175746F25632E67006572726F72207731
:10182000726974696E6720746F2066696C650A005E
:10183000446F6E6520736176696E672066696C65BA
:101840002E0A004D323900205A3A0020593A002021
:10185000583A00656E6473746F7073206869743AE7
:1018600020004732385859002042002050006F6B4A
:1018700000526573656E643A200043616E6E6F744A
:10188000206F70656E20737562646972200025692F
:10189000730025696D202569730025696820256915
:1018A0006D202569730025696420256968202569F4
:1018B0006D202569730025697920256964202569D3
:1018C000682025696D202569730023646566696E4B
:1018D000652044454641554C545F000062656400F4
:1018E0004B6420004B6920004B702000504944207D
:1018F0004175746F74756E652066696E697368658D
:1019000064212050757420746865206C61737420A4
:101910004B702C204B6920616E64204B6420636FF8
:101920006E7374616E74732066726F6D2062656C85
:101930006F7720696E746F20436F6E66696775728A
:101940006174696F6E2E680A0050494420417574B5
:101950006F74756E65206661696C656421207469B9
:101960006D656F75740A00453120544845524D41EC
:101970004C2052554E41574159004245442054484D
:1019800045524D414C2052554E41574159005468E3
:1019900065726D616C2052756E61776179004531B9
:1019A0002048656174696E67204661696C656400F2
:1019B0004265642048656174696E67204661696CA0
:1019C00065640048656174696E67206661696C656D
:1019D0006400504944204175746F74756E652066CB
:1019E00061696C6564212054656D70657261747500
:1019F000726520746F6F20686967680A00204B6405
:101A00003A2000204B693A2000204B703A20000A0F
:101A100020436C617373696320504944200A00209D
:101A20004B643A2000204B693A2000204B703A204A
:101A3000000A204E6F206F76657273686F6F740AAC
:101A4000002054753A2000204B753A2000206D612B
:101A5000783A2000206D696E3A200020643A200018
:101A600020626961733A2000504944204175746FC7
:101A700074756E652073746172740A005049442055
:101A80004175746F74756E65206661696C6564215B
:101A90002054656D706572617475726520746F6F26
:101AA00020686967680A00504944204175746F7462
:101AB000756E65206661696C6564212042616420F1
:101AC0006578747275646572206E756D6265720AF0
:101AD0000043616E6E6F74206F70656E2073756267
:101AE000646972200053442063617264206F6B0A42
:101AF000006F70656E526F6F74206661696C65640B
:101B00000A00766F6C756D652E696E69742066616A
:101B1000696C65640A00534420696E6974206661CB
:101B2000696C0A004D3234004D3233202573005762
:101B3000726974696E6720746F2066696C653A20FB
:101B4000002E0A006F70656E206661696C65642CFA
:101B50002046696C653A20002E0A006F70656E2081
:101B60006661696C65642C2046696C653A200046A4
:101B7000696C652073656C65637465640A00205345
:101B8000697A653A200046696C65206F70656E65FC
:101B9000643A2000667265736800646F696E67005E
:101BA0002066696C653A20004E6F772000454E44F0
:101BB00020535542524F5554494E450A0022207039
:101BC0006F73002220706172656E743A2200535563
:101BD00042524F5554494E452043414C4C2074616C
:101BE000726765743A2200747279696E6720746F47
:101BF0002063616C6C207375622D67636F64652070
:101C000066696C6573207769746820746F6F206DE6
:101C1000616E79206C6576656C732E204D4158207D
:101C20006C6576656C2069733A310A005344207004
:101C300072696E74696E67206279746520004E6FF8
:101C400074205344207072696E74696E670A0000D4
:101C500000000000000000000000000000484200FA
:101C6000004842000080405761726E696E673A20FA
:101C7000486F6D696E672042756D702044697669A2
:101C8000736F72203C20310A000202040000A04061
:101C90000000A04000000040000096430000964372
:101CA0000000C843FFFFFF0000000100000001002A
:101CB000008000555555000000400033333300AA22
:101CC000AA2A004992240000002000C7711C009934
:101CD000991900D1451700555515003BB113002443
:101CE00049120011111100000010000F0F0F00E346
:101CF000380E0043790D00CCCC0C00C3300C00E84A
:101D0000A20B0064210B00AAAA0A00703D0A009DE4
:101D1000D80900427B090092240900DCD30800881E
:101D20008808001042080000000800F0C107008782
:101D300087070075500700711C07003EEB0600A1E5
:101D4000BC06006990060066660600703E060061EB
:101D500018060017F4050074D105005BB00500B249
:101D6000900500627205005555050078390500B8E8
:101D70001E0500050505004EEC040087D40400A1F3
:101D8000BD040090A7040049920400C17D0400EE48
:101D9000690400C7560400444404005C320400088F
:101DA00021040041100400000004003FF00300F88B
:101DB000E0030026D20300C3C30300CCB503003AFE
:101DC000A803000A9B0300388E0300C08103009F14
:101DD000750300D0690300505E03001D53030034F7
:101DE000480300913D0300333303001629030038F4
:101DF0001F030097150300300C0300030303000BBF
:101E0000FA020049F10200BAE802005CE002002D8B
:101E1000D802002DD0020059C80200B0C002003123
:101E2000B90200DAB10200AAAA0200A0A30200BC13
:101E30009C0200FA9502005C8F0200DF880200829B
:101E4000820200457C0200277602002770020043D0
:101E50006A02007C640200D05E02003F590200C8A2
:101E6000530200FFFDFCFAF8F6F4F2F0EEECEAE9BA
:101E7000E7E5E3E1E0DEDCDAD9D7D5D4D2D0CFCDC7
:101E8000CBCAC8C7C5C3C2C0BFBDBCBAB9B7B6B458
:101E9000B3B2B0AFADACAAA9A8A6A5A4A2A1A09EBA
:101EA0009D9C9A99989795949392908F8E8D8B8AFA
:101EB0008988878684838281807F7E7D7B7A79781A
:101EC00077767574737271706F6E6D6C6B6A69681A
:101ED00067666564636261605F5E5D5C5B5A59580A
:101EE000585756555453525150504F4E4D4C4B4AE3
:101EF0004A4948474646454443424241403F3E3EA8
:101F00003D3C3B3B3A39383837363535343332325D
:101F10003130302F2E2E2D2C2B2B2A292928272704
:101F200026252524232322212120201F1E1E1D1C9F
:101F30001C1B1B1A1919181817161615151413132C
:101F400012121111100F0F0E0E0D0D0C0C0B0A0AB0
:101F50000909080807070606050504040303020229
:101F600001000020746F6F206C6F6E6720657874BD
:101F7000727573696F6E2070726576656E746564D4
:101F80000A0020636F6C6420657874727573696FE2
:101F90006E2070726576656E7465640A007C3C3EE6
:101FA0005E2B3D3F2F5B5D3B2C2A225C000A4D657A
:101FB00061737572656420706F696E74733A0A009C
:101FC000357835206D6573682E205A206F666673EC
:101FD00065743A20002F2F616374696F6E3A006256
:101FE0007574746F6E00656E640070726F6D7074DE
:101FF0005F0073686F77004D383736205265737015
:102000006F6E64696E672050524F4D50545F00559B
:102010004E4B4E4F574E2053544154450047434F6B
:1020200044455F494E464F004C43445F5041555331
:10203000455F524553554D450046494C414D454E2F
:10204000545F52554E4F55545F434F4E54494E5571
:10205000450046494C414D454E545F52554E4F55F3
:1020600054004D323400436F6E74696E75650044E0
:10207000697361626C6552756E6F7574005075722C
:102080006765204D6F7265005061757365640070FF
:10209000617573656400486F74656E6420746F6F5A
:1020A00020636F6C640A004469736D697373005038
:1020B0006175736500507265737320627574746F17
:1020C0006E20286F72204D3130382920746F2072B5
:1020D0006573756D650A00496E7365727420666973
:1020E0006C616D656E7420616E64207072657373CF
:1020F00020627574746F6E20286F72204D313038F5
:10210000290A00436F6E74696E75650052656865D3
:10211000617420446F6E6500526568656174696E14
:10212000672E2E2E00526568656174696E670048DF
:10213000656174657254696D656F75740052656888
:102140006561740048656174657254696D656F7589
:102150007400507265737320627574746F6E2028FA
:102160006F72204D3130382920746F20686561749A
:10217000206E6F7A7A6C650A004E6F7A7A6C6520F1
:102180005061726B656400436F6E74696E756500B3
:102190004E6F7A7A6C65205061726B656400486F8F
:1021A00074656E6420746F6F20636F6C640A0072D4
:1021B0006573756D656400626567696E00436F6E77
:1021C00074696E75650044697361626C6552756E01
:1021D0006F75740050757267654D6F726500506160
:1021E00075736564004C6F61642046696C616D6550
:1021F0006E7400436F6E74696E7565004C6F616438
:102200002046696C616D656E74205400496E73657B
:1022100072742066696C616D656E7420616E6420F5
:10222000707265737320627574746F6E20286F729C
:10223000204D313038290A004469736D6973730089
:10224000526573756D696E6700453120544845527B
:102250004D414C2052554E41574159004245442072
:10226000544845524D414C2052554E41574159001A
:10227000546865726D616C2052756E61776179008A
:102280004531204572723A204D415854454D500019
:102290004572723A204D415854454D5020424544B4
:1022A000004D415854454D502074726967676572FE
:1022B0006564004531204572723A204D494E5445BF
:1022C0004D50004572723A204D494E54454D5020B4
:1022D000424544004D494E54454D50207472696743
:1022E0006765726564000A0A0020205A5F4D494EF6
:1022F0003A002020595F4D494E3A002020585F4D4A
:10230000494E3A004D383420582059205A20450073
:10231000202F002042403A0020403A00436F6F6C6B
:10232000696E672E2E2E0048656174696E672E2EC9
:102330002E0020573A0020573A00496E76616C69AA
:10234000642065787472756465720A00416374690B
:1023500076652045787472756465723A2000486F1E
:1023600074656E6420746F6F20636F6C640A00295B
:102370000A002062797465733B2063726320005306
:10238000657474696E67732053746F726564202876
:1023900000454550524F4D206461746173697A6500
:1023A000206572726F722E0A00290A002062797409
:1023B00065733B2063726320002073746F726564E1
:1023C0002073657474696E677320726574726965D1
:1023D000766564202800202863616C63756C6174E5
:1023E000656429210A0020213D2000454550524FB7
:1023F0004D20435243206D69736D61746368202DD5
:10240000202873746F7265642920002053697A65EF
:102410003A2000496E6465783A2000204D61726C64
:10242000696E3D563730290A00454550524F4D20C0
:1024300076657273696F6E206D69736D6174636820
:102440002028454550524F4D3D005A5F53544F5040
:102450005F50494E005A5F535445505F50494E00FB
:102460005A5F4D494E5F50494E005A5F454E4142BA
:102470004C455F50494E005A5F4449525F50494EA7
:10248000005A5F43535F50494E00595F53544F50B9
:102490005F50494E00595F535445505F50494E00BC
:1024A000595F4D494E5F50494E00595F454E41427C
:1024B0004C455F50494E00595F4449525F50494E68
:1024C00000595F43535F50494E00585F53544F507B
:1024D0005F50494E00585F535445505F50494E007D
:1024E000585F4D494E5F50494E00585F454E41423E
:1024F0004C455F50494E00585F4449525F50494E29
:1025000000585F43535F50494E0053535F50494E4C
:1025100000534552564F335F50494E005345525673
:102520004F325F50494E00534552564F315F50492C
:102530004E00534552564F305F50494E005344535E
:10254000530053445F4445544543545F50494E0043
:1025500053434B5F50494E0052414D50535F4439F5
:102560005F50494E0052414D50535F44385F5049CF
:102570004E0052414D50535F4431305F50494E0040
:102580004D4F53495F50494E004D4F534645545FA0
:10259000445F50494E004D49534F5F50494E004DE6
:1025A0004158363637355F53535F50494E004C45DE
:1025B000445F50494E004845415445525F424544AE
:1025C0005F50494E004845415445525F305F504985
:1025D0004E0046494C5F52554E4F5554325F50495C
:1025E0004E0046494C5F52554E4F55545F50494E30
:1025F0000046414E315F50494E0046414E5F5049C2
:102600004E0045315F535445505F50494E004531AF
:102610005F454E41424C455F50494E0045315F4455
:1026200049525F50494E0045315F43535F50494E18
:102630000045305F535445505F50494E0045305F70
:10264000454E41424C455F50494E0045305F44493C
:10265000525F50494E0045305F43535F50494E0032
:10266000455F4D5558325F50494E00455F4D5558B6
:10267000315F50494E00455F4D5558305F50494ECF
:10268000004245455045525F50494E004156525F09
:1026900053535F50494E004156525F53434B5F5076
:1026A000494E004156525F4D4F53495F50494E00CD
:1026B0004156525F4D49534F5F50494E0054454D6E
:1026C000505F4245445F50494E0054454D505F3184
:1026D0005F50494E0054454D505F305F50494E00A9
:1026E00046494C57494454485F50494E0054584459
:1026F000005258440050574D3A2020253464005071
:10270000574D3A20202534640050574D3A2020255B
:1027100034640050574D3A20202534640050574D02
:102720003A20202534640050574D3A202025346447
:102730000050574D3A20202534640050574D3A2020
:10274000202534640050574D3A2020253464005031
:10275000574D3A20202534640050574D3A2020250B
:1027600034640050574D3A20202534640050574DB2
:102770003A20202534640050574D3A2020253464F7
:102780000050574D3A20202534640050574D3A20D0
:1027900020253464003A200020202020434F4D00A3
:1027A0002020206E6F6E2D7374616E6461726420E0
:1027B00050574D206D6F646500202020636F6D7051
:1027C00061726520696E7465727275707420656ED1
:1027D00061626C6564002020206F766572666C6FA4
:1027E0007720696E7465727275707420656E6162AF
:1027F0006C6564003A20002020202054494D534B42
:1028000000423A2000202020205443435200413A05
:102810002000202020205443435200202020204329
:10282000533A20002020202057474D3A200050578F
:102830004D3A20202534640050574D3A202025344D
:10284000640047004800000088008A008C00B30044
:10285000B400000098009A009C00A800AA00AC00F8
:1028600028012A012C012020202054494D455200E6
:10287000440045006E00800081006F00B000B10090
:102880007000900091007100A000A1007200200172
:102890002101730020697320616C736F2074696576
:1028A0006420746F20746869732070696E005449E5
:1028B0004D45523143000A202E0020200020205098
:1028C0006F72743A200020202000202020416E6189
:1028D0006C6F6720696E203D2025356C64003C7567
:1028E0006E757365642F756E6B6E6F776E3E00202C
:1028F00028412532642920200025336420002573D7
:1029000050494E3A20004F7574707574203D200078
:10291000496E70757420203D2000416E616C6F67B8
:1029200020696E203D2025356C640070726F7465DF
:10293000637465642000202841253264292020002A
:102940002533642000257350494E3A2000F12600BB
:1029500001ED260101E0263B00D5264300CA2645AD
:1029600000BD264400B0263201A326330197263449
:10297000018C26350181262501762628016B262A21
:102980000160262C0156262A014B261C013D2618E3
:102990000131261A0127262C011C2622010E261E93
:1029A0000102262401FA250901F1250701E2250289
:1029B00001D2250F01C5250A01B6250801AE250D56
:1029C000019F254201962532018925070180253383
:1029D0000172250A01652508015825090150253491
:1029E00001422531013D25350132250B0127250600
:1029F000011C250501112504010A25350101253594
:102A000001F7243701EA242601E0240301D5243606
:102A100001CA240301C1243101B7243D01AA24388D
:102A200001A0240E0195243C018A240E0181242852
:102A300001772430016A243E016024120155242EBE
:102A4000014A241201446F6E652E0A005345525606
:102A50004F206E6F74207365742075702E0A004DC0
:102A6000343320576169742043616C6C65640043A2
:102A70006F6E74696E7565004D34332057616974EB
:102A80002043616C6C6564005761746368696E67AC
:102A90002070696E730A0064697300656E0061627C
:102AA0006C65640A00656E6473746F70206D6F6E80
:102AB00069746F72200057616974696E6720666F70
:102AC00072206865617475702E0A004C65617669C4
:102AD0006E6720473236003F5370656369666965EB
:102AE0006420582C5920636F6F7264696E6174653D
:102AF000206F7574206F6620626F756E64732E0A86
:102B0000003F28522965706561742076616C756597
:102B1000206E6F7420706C61757369626C653B2008
:102B20006D757374206265206174206C65617374C7
:102B300020312E0A003F2852296570656174206D8E
:102B40007573742062652073706563696669656476
:102B5000207768656E206E6F74207573696E6720CC
:102B6000616E204C43442E0A003F537065636966D2
:102B7000696564206E6F7A7A6C652074656D706526
:102B8000726174757265206E6F7420706C617573FC
:102B900069626C652E0A003F5370656369666965FA
:102BA000642066696C616D656E742073697A652056
:102BB0006E6F7420706C61757369626C652E0A00AB
:102BC0003F537065636966696564207072696D65FD
:102BD000206C656E677468206E6F7420706C617510
:102BE0007369626C652E0A003F5072696D65206CD6
:102BF000656E677468206D757374206265207370EC
:102C000065636966696564207768656E206E6F74B8
:102C1000207573696E6720616E204C43442E0A0054
:102C20003F537065636966696564206E6F7A7A6C7C
:102C3000652073697A65206E6F7420706C6175739E
:102C400069626C652E0A003F526574726163746933
:102C50006F6E204D756C7469706C696572206D754E
:102C60007374206265207370656369666965642E9C
:102C70000A003F5370656369666965642052657434
:102C800072616374696F6E204D756C7469706C69E4
:102C90006572206E6F7420706C61757369626C650B
:102CA0002E0A003F537065636966696564206C6134
:102CB00079657220686569676874206E6F7420702A
:102CC0006C61757369626C652E0A0043292E0A00D7
:102CD0003F5370656369666965642062656420744A
:102CE000656D7065726174757265206E6F742070A9
:102CF0006C61757369626C65202834302D00473231
:102D000036207374617274696E672E2E2E0A00006D
:102D1000002100240027002A002D0030003300018C
:102D2000010000040107010A01000022002500281B
:102D3000002B002E003100340002010000050108C4
:102D4000010B01000020002300260029002C002F89
:102D5000003200000100000301060109010505051C
:102D600005070508080808020202020A0A08080402
:102D70000404040101010101010101030303030330
:102D8000030303040707070C0C0C0C0C0C0C0C02BF
:102D900002020206060606060606060B0B0B0B0BC6
:102DA0000B0B0B01021020200808102040102040BF
:102DB00080020102010804020101020408102040FF
:102DC000808040201008040201800402018040201D
:102DD0001008040201080402010102040810204046
:102DE00080010204081020408000000A0B02090C38
:102DF0000D0E0807030401000000000000000000A1
:102E000000000000000000000000000000000000C2
:102E1000000000000012111000000000000000007F
:102E2000000000000000000000000000000000475B
:102E3000323800486F6D6520257325732573204651
:102E40006972737400220A00556E6B6E6F776E2084
:102E5000636F6D6D616E643A202200204500205A38
:102E600000205900204D39322058004F4646004F6F
:102E70004E00205A0020590020580020204D617833
:102E80003A2000200020204D696E3A2000536F66E2
:102E90007420656E6473746F70733A2000576172AA
:102EA0006E696E67203A20436C65616E20436972DB
:102EB000636C652072657175697265732058590A73
:102EC0000020496E76616C6964206578747275645F
:102ED000657220006F70656E005452494747455235
:102EE0004544003A200066696C616D656E74007A35
:102EF0005F6D696E00795F6D696E00785F6D696EF8
:102F0000005265706F7274696E6720656E647374C9
:102F10006F70207374617475730A00205A3A002030
:102F2000593A0020436F756E7420583A0020453A94
:102F300000205A3A0020593A00583A0000009643BF
:102F4000000096430000C84300000000000000009D
:102F50000000000020746F6F206C6F6E6720657832
:102F600074727573696F6E2070726576656E7465C4
:102F7000640A0020636F6C642065787472757369ED
:102F80006F6E2070726576656E7465640A00452008
:102F90002553002E0A006F70656E206661696C65AE
:102FA000642C2046696C653A2000706F7765726FFB
:102FB0006666004B494C4C45442E20005072696EA9
:102FC0007465722068616C7465642E206B696C6C2A
:102FD00028292063616C6C6564210A004469666677
:102FE0003A200046726F6D5374703A0053746570E6
:102FF0007065723A00556E4C6576656C3A004C65AA
:1030000076656C65643A005261773A202020200092
:103010000A4C6F676963616C3A004361703A002241
:103020000A00656E7175657565696E672022000A14
:1030300020696E6974207A70726F62655F7A6F665C
:1030400066736574203D2000454550524F4D204920
:103050006E697469616C697A65640A0048617264BA
:10306000636F6465642044656661756C74205365A4
:103070007474696E6773204C6F616465640A000044
:1030800000FA430000FA430000204100009642008D
:1030900000A0420000A0420000C8430000BE42DC85
:1030A000050000DC050000640000004B000000206B
:1030B000204D363033200020440020204D34313262
:1030C00020530046696C616D656E742072756E6F79
:1030D00075742073656E736F723A0A00546F6F6C6B
:1030E0002D6368616E67696E673A0A002055005467
:1030F00031204C002055005430204C0046696C6152
:103100006D656E74206C6F61642F756E6C6F616499
:10311000206C656E677468733A0A00204B002020AB
:103120004D3930302054004C696E65617220416425
:1031300076616E63653A0A00204400204900202031
:103140004D33303420500020440020490020204DD1
:103150003330312050005049442073657474696ED7
:1031600067733A0A00205A0020590020204732395C
:10317000205333205800205A0020204D3432302074
:1031800053004D65736820426564204C6576656C1C
:10319000696E673A0A00205A0020590020204D32FB
:1031A0003036205800486F6D65206F666673657411
:1031B0003A0A00204A0020540020530020204D32BB
:1031C0003035204200204A3C6A756E635F64657644
:1031D0003E00416476616E6365643A20423C6D69ED
:1031E0006E5F7365676D656E745F74696D655F753D
:1031F000733E20533C6D696E5F66656564726174F1
:10320000653E20543C6D696E5F74726176656C5FDB
:1032100066656564726174653E002054002052004A
:1032200020204D323034205000416363656C65725C
:103230006174696F6E2028756E6974732F733229FB
:103240003A20503C7072696E745F616363656C3ED6
:1032500020523C726574726163745F616363656C74
:103260003E20543C74726176656C5F616363656C8B
:103270003E0A00204500205A0020590020204D32EF
:1032800030312058004D6178696D756D2041636360
:10329000656C65726174696F6E2028756E697473F0
:1032A0002F7332293A0A00204500205A0020590085
:1032B00020204D3230332058004D6178696D756D96
:1032C000206665656472617465732028756E697423
:1032D000732F73293A0A00537465707320706572F6
:1032E00020756E69743A0A0020204D323030204437
:1032F000300A0020204D323030205431204400204C
:10330000204D3230302044002044697361626C6586
:10331000640A0046696C616D656E7420736574742F
:10332000696E67733A0020286D6D290020204732AE
:1033300031202020203B20556E69747320696E2057
:103340006D6D00486F6D696E67204661696C6564DC
:10335000004F46460A004661646520486569676813
:10336000742000426564204C6576656C696E672048
:10337000004661696C656420746F20656E61626CE3
:103380006520426564204C6576656C696E670A004D
:103390004D65736820426564204C6576656C2064D9
:1033A0006174613A0A00496E76616C6964206D65EA
:1033B00073682E0A00206E6F7420656E74657265E6
:1033C000642E0A004D65736820706F696E74206307
:1033D000616E6E6F74206265207265736F6C7665C6
:1033E000640A004D34323120696E636F7272656316
:1033F0007420706172616D657465722075736167A8
:10340000650A00205400205200416363656C6572B8
:103410006174696F6E3A2050003F4A206F757420C6
:103420006F662072616E67652028302E30312074FF
:103430006F20302E33290A00546F6F6C6368616E01
:1034400067653A0020204D32313700205A0020595C
:10345000002058002052002050002045002053003A
:1034600070012C0190012701B0012201C0011D0152
:10347000F00118011002130130020E01600209016F
:1034800090020401C002FF000003FA004003F500AF
:103490008003F000D003EB002004E6007004E1009C
:1034A000E004DC004005D700C005D2004006CD0096
:1034B000D006C8008007C3003008BE00F008B9007D
:1034C000C009B400B00AAF00B00BAA00D00CA50030
:1034D000000EA000500F9B00C010960050129100EB
:1034E00000148C00C0158700B0178200B0197D0051
:1034F000D01B7800001E730040206E0090226900EF
:10350000F024640040275F0090295A00E02B55000A
:10351000102E500020304B0010324600E0334100A6
:1035200090353C001037370070383200A0392D003C
:10353000B03A2800A03B2300603C1E00103D19005B
:10354000903D1400103E0F00703E0A00C03E050082
:10355000003F0000403FFBFF803FF6FFC03FF1FF10
:10356000626564002C2073797374656D2073746FC9
:103570007070656421204865617465725F49443AE2
:1035800020004265642048656174696E6720466169
:10359000696C65640048656174696E67206661697D
:1035A0006C65640042454420544845524D414C20CE
:1035B00052554E4157415900546865726D616C20F7
:1035C00052756E6177617900453120486561746993
:1035D0006E67204661696C65640048656174696E58
:1035E00067206661696C6564004531205448455226
:1035F0004D414C2052554E41574159005468657217
:103600006D616C2052756E6177617900202D2049C3
:103610006E76616C69642065787472756465722079
:103620006E756D62657220210A001000C9021001DA
:103630002C014001220170011801B0010E01F001BE
:1036400004015002FA00B002F0003003E600D0039B
:10365000DC009004D2007005C800A006BE0000087F
:10366000B400B009AA00D00BA000600E9600601153
:103670008C000015820020197800C01D6E00A02269
:103680006400B0275A00902C500000314600E0340E
:103690003C0010383200903A2800603C1E00A03DEB
:1036A0001400803E0A00203F0000544D3344204364
:1036B000522D582052656164792E005072696E74E3
:1036C000696E672E2E2E005072696E7420506175DF
:1036D0007365640063616E63656C005072696E743B
:1036E0002041626F72746564004469736D6973731D
:1036F0000055492041626F7274656400726573758C
:103700006D65004D323400001C01420111241FBEC2
:10371000CFEFD1E2DEBFCDBF00E00CBF17E0A0E0ED
:10372000B2E0E8EEFEE302E00BBF02C007900D92AC
:10373000A43EB107D9F72EE1A4EEB7E001C01D9277
:10374000AD35B207E1F71BE1C5E8DBE100E006C0FB
:1037500021970109802FFE010F94911BC438D107D6
:1037600080E00807A9F70F9447030D94621F0C949B
:1037700000002F923F924F925F926F927F928F92B2
:103780009F92AF92BF92CF92DF92EF92FF920F93F0
:103790001F93CF93DF93CDB7DEB7A7970FB6F894FB
:1037A000DEBF0FBECDBF80910901817091E09827E7
:1037B00020910308921781F190930308811116C09C
:1037C0000E9493708091241783FF09C083EC93E0DB
:1037D0000E94C24F61E080E00E9469CA1DC060E0A3
:1037E00081E00E9469CA8CED93E014C00091241717
:1037F00003FB002700F90E94227080912417877F25
:1038000080932417002341F060E081E00E9469CAA0
:1038100085EF93E00E94C24F8091020881110C94C1
:10382000203780910008909101089C012F5F3F4F45
:103830003093010820930008883E934010F40C94C4
:10384000203781E08093020810920108109200084E
:1038500080910818882309F48EC30E948A6381111D
:103860008AC38091FF078F5F8093FF078091FF07D6
:10387000853620F01092FF0710920818E091081882
:103880008E2FEE0F990BAA0BBB0BFC013197E73083
:10389000F10508F0A0C08827EE58FF4F8F4F0D9418
:1038A000911B0E948263882309F495C081E0809374
:1038B000730288E094E00E94C24F80E190E0909310
:1038C00081158093801585E08093741502E800933C
:1038D000771584E190E1A0E0B0E0809378159093B3
:1038E0007915A0937A15B0937B150E9407E181E0CA
:1038F0009AE5909381158093801586E390E09093EC
:1039000083158093821587E0809374150093771553
:1039100084E890E0A0E0B0E080937815909379156A
:10392000A0937A15B0937B150E9407E152C00E94C4
:103930008263882309F44FC048C086E194E00E9466
:10394000C24F81E09AE5909381158093801580E4C1
:1039500090E0909383158093821507E0009374158F
:1039600082E88093771584E890E0A0E0B0E080934F
:10397000781590937915A0937A15B0937B150E94D2
:1039800007E10093081827C08091FE07882319F1EA
:103990000E9482638823F9F00E948A6381111BC010
:1039A000EDC20E9482638823B1F00E948A63811174
:1039B00012C012C30E948A6381110DC042E060E010
:1039C00070E0CB010E94D56304C00E948A6381111C
:1039D00002C01092081880917302882309F4B3C2C0
:1039E0008091041890910518892B09F08FC180915E
:1039F000FB079091FC07892B09F01EC184E096E03B
:103A0000909381158093801580EA90E890938315B8
:103A10008093821517E01093741502E800937715D0
:103A200080EA90E0A0E0B0E080937815909379155B
:103A3000A0937A15B0937B150E9407E18091120242
:103A400090911302A0911402B09115020097A10564
:103A5000B10511F5109281151092801515E01093A3
:103A60007415009377158AE890E1A0E0B0E08093A8
:103A7000781590937915A0937A15B0937B150E94D1
:103A800007E189E090E09093811580938015109371
:103A900074150093771540C00196A11DB11D65E016
:103AA000B695A795979587956A95D1F70197A1093E
:103AB000B109009721E0A207B10558F0B093811534
:103AC000A09380159093831580938215109374159D
:103AD00007C0909381158093801585E080937415BD
:103AE00012E8109377158AE890E1A0E0B0E08093A7
:103AF000781590937915A0937A15B0937B150E9451
:103B000007E188E090E0909381158093801585E02F
:103B100080937415109377158CE890E1A0E0B0E0E5
:103B20008093781590937915A0937A15B0937B15AF
:103B30000E9407E18091120290911302A091140259
:103B4000B0911502009731E0A307B10550F0B09392
:103B50008115A0938015909383158093821587E03B
:103B600005C0909381158093801585E0809374152E
:103B700082E88093771588E890E1A0E0B0E0809338
:103B8000781590937915A0937A15B0937B150E94C0
:103B900007E18091120290911302A0911402B0915A
:103BA0001502BA2FA92F982F88270097E1E0AE07BA
:103BB000B10550F0B0938115A093801590938315B3
:103BC0008093821587E005C09093811580938015BE
:103BD00085E08093741512E81093771581EA90E0E0
:103BE000A0E0B0E08093781590937915A0937A15B2
:103BF000B0937B150E9407E18091E40D882319F0B2
:103C000082E090E002C083E090E090938115809381
:103C1000801585E0809374151093771585E490E105
:103C2000A0E0B0E08093781590937915A0937A1571
:103C3000B0937B150E9407E10091FB071091FC07F0
:103C4000053611057CF4109381150093801585E0ED
:103C50008093741582E88093771580E090E1A0E06E
:103C6000B0E011C0C80184569109909381158093EA
:103C7000801585E08093741582E88093771581E044
:103C800090E1A0E0B0E08093781590937915A0932F
:103C90007A15B0937B150E9407E10F5F1F4F1093B9
:103CA000FC070093FB07093C110564F184E294E0F2
:103CB0000E94C24F81E090E0909305188093041811
:103CC0008093730281E09AE590938115809380152B
:103CD0008DE290E0909383158093821587E0809326
:103CE000741582E88093771584E890E0A0E0B0E056
:103CF0008093781590937915A0937A15B0937B15DE
:103D00000E9407E1109202080C9420378091D2148F
:103D10009091D314891B8F7009F0DCC10E94914DE2
:103D20008111D8C18091241782FDD4C17FC184E65E
:103D300090E09093811580938015109374150093F3
:103D400077158EE090E1A0E0B0E080937815909335
:103D50007915A0937A15B0937B150E9407E1C601EF
:103D600082539048880F991F9093811580938015F6
:103D700010937415009377158FE090E1A0E0B0E008
:103D80008093781590937915A0937A15B0937B154D
:103D90000E9407E10E944CFF90E090938115809370
:103DA000801585E08093741582E88093771586E10D
:103DB00090E1A0E0B0E08093781590937915A093FE
:103DC0007A15B0937B150E9407E160917B13709187
:103DD0007C13072E000C880B990B0F94A91420E07C
:103DE00030E048EC52E40F9408150F94121D7093C4
:103DF00081156093801515E01093741502E8009307
:103E0000771586E290E1A0E0B0E08093781590937A
:103E10007915A0937A15B0937B150E9407E120E0F5
:103E200030E0A9016091290970912A0980912B093C
:103E300090912C090F94A61B0F94121D709381155D
:103E400060938015109374150093771586E390E1C5
:103E5000A0E0B0E08093781590937915A0937A153F
:103E6000B0937B150E9407E1609140097091410970
:103E700080914209909143090F94121D709381150E
:103E80006093801510937415009377158CE390E17F
:103E9000A0E0B0E08093781590937915A0937A15FF
:103EA000B0937B150E9407E180912D0990912E0916
:103EB0009093811580938015109374150093771556
:103EC00084E390E1A0E0B0E08093781590937915B9
:103ED000A0937A15B0937B150E9407E18091440965
:103EE00090914509909381158093801510937415D6
:103EF000009377158AE390E1A0E0B0E08093781515
:103F000090937915A0937A15B0937B150E9407E1E1
:103F10000091F70701117FC18091F90781117BC1E1
:103F20008091FE0781113CC280912815909129153E
:103F3000A0912A15B0912B158C34F0E19F07A105B3
:103F4000B10509F052C284ECC82E85E1D82E0AE1F1
:103F50008EEB93E10E94756EE090EC07F090ED0718
:103F6000181619060CF09DC31AE1E116F10414F4B9
:103F70000C943B3396C31092FF0778CC8EEE95E0FD
:103F80000E94C24F8091FD0790E0A0E0B0E0895B05
:103F90009F4FAE4FB54A21E03AE53093811520930B
:103FA0008015909383158093821587E08093741514
:103FB00082E88093771584E890E0A0E0B0E08093F9
:103FC000781590937915A0937A15B0937B150E947C
:103FD00007E11092FE07FDCC81E0809373021092FE
:103FE00008188CEF95E00E94C24F81E09AE590930B
:103FF0008115809380158EE490E0909383158093D3
:10400000821587E08093741582E88093771584E8A1
:1040100090E0A0E0B0E08093781590937915A0939C
:104020007A15B0937B150E9407E1D5CC0091400929
:1040300010914109209142093091430908A319A325
:104040002AA33BA36091440970914509072E000CF7
:10405000880B990B0F94A9146B017C0120E030E0D0
:1040600040E050E40F94A51B28A139A14AA15BA10F
:104070000F94061E18160CF433C220E030E0A9019C
:104080006091290970912A0980912B0990912C093E
:104090000F94A61B6CA37DA38EA39FA360912D09F3
:1040A00070912E09072E000C880B990B0F94A91400
:1040B0004B015C0120E030E040E251E40F94A51B8D
:1040C0002CA13DA14EA15FA10F94061E18160CF461
:1040D00007C226C28CE090E09093811580938015F2
:1040E00005E00093741582E88093771584E190E1F0
:1040F000A0E0B0E08093781590937915A0937A159D
:10410000B0937B150E9407E10E9479FD20E13EE01B
:1041100040E050E00F94F81A2115310511E04107F5
:10412000510560F0509381154093801530938315AD
:104130002093821587E08093741506C03093811513
:10414000209380150093741502E80093771580E1A1
:1041500090E1A0E0B0E08093781590937915A0935A
:104160007A15B0937B150E9407E10E9479FD20E14A
:104170003EE040E050E00F94F81A2CE330E040E0DD
:1041800050E00F94F81A309381152093801515E0B4
:10419000109374150093771582E190E1A0E0B0E0F0
:1041A0008093781590937915A0937A15B0937B1529
:1041B0000E9407E10E944CFF882391F00E944CFF6F
:1041C0008F5F8093FA07C82ED12C833308F0AFCDD0
:1041D000C601880F991F909381158093801504C0A4
:1041E0001092811510928015109374150093771515
:1041F0008EE090E1A0E0B0E080937815909379157F
:10420000A0937A15B0937B150E9407E11092811557
:1042100010928015ADCD20E030E0A9016091290910
:1042200070912A0980912B0990912C090F94A61B5B
:1042300020E030E048EC52E40F9408156B017C015B
:1042400060912D0970912E09072E000C880B990B97
:104250000F94A9149B01AC01C701B6010F94A01CD7
:104260000F94191D6436710510F064E670E07093C8
:1042700081156093801595E0A92EA092741522E80F
:10428000B22EB092771584E290E1A0E0B0E0809386
:10429000781590937915A0937A15B0937B150E94A9
:1042A00007E120E030E0A9016091290970912A0915
:1042B00080912B0990912C090F94A61B6B017C0116
:1042C00020E030E04AE253E40F94061E18160CF08A
:1042D00069C1002309F466C11092F70720E030E0BD
:1042E00040E251E46091EF077091F0078091F1078F
:1042F0009091F2070F9408150F94121D7093811579
:1043000060938015A0927415B092771584E590E1C2
:10431000A0E0B0E08093781590937915A0937A157A
:10432000B0937B150E9407E120E030E040E251E4C9
:104330006091F3077091F4078091F5079091F6076B
:104340000F9408150F94121D7093811560938015BA
:10435000A0927415B092771588E590E1A0E0B0E0E6
:104360008093781590937915A0937A15B0937B1567
:104370000E9407E18AE096E00E94C24F81E09AE540
:10438000909381158093801581E490E0909383153C
:104390008093821587E080937415B092771551C190
:1043A0008091EE0701E0080F0093EE0790E09093F4
:1043B00081158093801585E08093741582E8809341
:1043C000771582E490E1A0E0B0E0809378159093B7
:1043D0007915A0937A15B0937B150E9407E10A30F6
:1043E00008F4A2CD1092EE079FCD8A349041A1052A
:1043F000B10509F4A8CD20E030E040E251E460913D
:10440000CC0D7091CD0D8091CE0D9091CF0D0F946C
:1044100008150F94121D709381156093801515E097
:104420001093741502E80093771588E490E1A0E0FA
:10443000B0E08093781590937915A0937A15B09396
:104440007B150E9407E120E030E040E251E46091FA
:10445000D00D7091D10D8091D20D9091D30D0F940C
:1044600008150F94121D7093811560938015109399
:104470007415009377158AE490E1A0E0B0E0809392
:10448000781590937915A0937A15B0937B150E94B7
:1044900007E120E030E040E251E46091D40D7091FA
:1044A000D50D8091D60D9091D70D0F9408150F94CE
:1044B000121D7093811560938015109374150093ED
:1044C00077158CE490E1A0E0B0E0809378159093AC
:1044D0007915A0937A15B0937B150E9407E133CD2F
:1044E0008DE090E0909381158093801585E0809316
:1044F000741582E88093771584E190E1A0E0B0E044
:104500008093781590937915A0937A15B0937B15C5
:104510000E9407E180910718811141C081E03FC0EE
:1045200020E030E040E050E4C701B6010F94A61B44
:1045300028A139A14AA15BA10F94A21487FD10C044
:1045400020E030E040E251E4C501B4010F94A61B25
:104550002CA13DA14EA15FA10F94A21487FF35CCE1
:1045600084E190E0909381158093801585E080939D
:10457000741582E88093771584E190E1A0E0B0E0C3
:104580008093781590937915A0937A15B0937B1545
:104590000E9407E180910718811101C082E0809399
:1045A000071813CC60912D0970912E09072E000C6D
:1045B000880B990B0F94A9149B01AC01C701B6019C
:1045C0000F94061E6091F90787FD4AC0662309F41F
:1045D000A7CC062E000C770B82E996E00E94294FAB
:1045E0001092F9071092FC071092FB0784E090E00C
:1045F000909381158093801585E08093741502E86F
:10460000009377158EE890E1A0E0B0E080937815F4
:1046100090937915A0937A15B0937B150E9407E1CA
:1046200081E09AE5909381158093801583E590E071
:10463000909383158093821587E08093741500937F
:10464000771584E890E0A0E0B0E08093781590932F
:104650007915A0937A15B0937B150E9407E160CC81
:10466000662309F45DCC8091FB079091FC079C01C7
:104670002F5F3F4F3093FC072093FB0765E070E00E
:104680000F947D1B909381158093801585E0809316
:10469000741582E8809377158EE890E1A0E0B0E091
:1046A000D4CF1E141F040CF02DCB909125158091B2
:1046B000C415981322C0909126158091C5159813A2
:1046C0001CC003E0E016F104C4F09091C61590936D
:1046D00024158091C715809327159330D1F4982F16
:1046E0009D7F9038B1F49091C8159F3409F05FC058
:1046F0009091C9159B3409F05AC08AE1E4ECF5E1C8
:10470000DF011D928A95E9F71092ED071092EC07F0
:10471000F9CA833809F04BC08091C8159091C9152A
:10472000982789279827A0E0B0E0809328159093D8
:104730002915A0932A15B0932B154091CA1550E066
:1047400060E070E040932C1550932D1560932E156A
:1047500070932F150BECA02E05E1B02E80E090E0B9
:10476000DC0184179507A607B70708F04EC06C0157
:104770007D01F694E794D794C79496012A5F3F4F42
:10478000220F331FF901EC5DFA4E7F01F501208104
:1047900030E0322F22270181202BF7013183208343
:1047A0000296A11DB11DF2E0AF0EB11CDACF813827
:1047B00061F58091C81590E0A0E0B0E080932815E5
:1047C00090932915A0932A15B0932B158091C915A4
:1047D000482F50E060E070E040932C1550932D1569
:1047E00060932E1570932F15AAECB5E1E0E3F5E187
:1047F00090E020E030E02817390739F04D9150E083
:10480000419351932F5F3F4FF6CF8AE1E4ECF5E1FE
:10481000DF011D928A95E9F71092ED071092EC07DF
:1048200085E394E00E94C24F60910818161664F464
:10483000062E000C770B87E896E00E94294F8AE04D
:104840000E94E64D0C942C33609130157091311517
:1048500085E796E00E94004F8AE00E94E64D409175
:1048600028155091291560912A1570912B1586E60F
:1048700096E00E94EF4E8AE00E94E64D8091281556
:1048800090912915A0912A15B0912B15E8E7F2E037
:1048900000E010E0419151916191719141155105F4
:1048A00061057105D1F1481759076A077B0791F532
:1048B000AC01BD01485050416109710945305105B5
:1048C0006105710568F1AC01BD01477F423350417C
:1048D0006105710541F18433F0E19F07A105B10540
:1048E00011F1AC01BD0146545041610971094730D5
:1048F000510561057105D0F0AC01BD014455504131
:1049000061097109453051056105710588F402E1BD
:1049100010E00EC00F5F1F4FBDCF0FEF1FEF08C09D
:1049200003E010E005C008E010E002C00FE010E076
:104930008A509042A109B109833D9105A105B105B5
:1049400030F00F3F2FEF120721F40C942C3309E1C4
:1049500010E0A6E5CA2EA4E0DA2EF60181916F01DF
:10496000882319F00E94E64DF8CFB801012E000C03
:10497000880B990B0E940D4F0E94BC4F8AE596E070
:104980000E94C24F0A31110510F00C942833F8012F
:104990008827E758FF4F8F4F0D94911B809130155A
:1049A0009091311581309105E1F4109273028FEFEF
:1049B0008093431060E080E00E9469CA04E614E03E
:1049C000D8018D918D01882319F00E94E64DF8CF12
:1049D00081E09AE590938115809380158EE290E0B6
:1049E000AFC08230910509F0B7C081E080937302B7
:1049F0000E94BDFF86E596E090937909809378093F
:104A00008BE090E0909381158093801505E00093F2
:104A1000741512E81093771580E092E1A0E0B0E001
:104A20008093781590937915A0937A15B0937B15A0
:104A30000E9407E110928115109280150093741561
:104A4000109377158EE090E1A0E0B0E080937815A8
:104A500090937915A0937A15B0937B150E9407E186
:104A6000109281151092801500937415109377158C
:104A70008FE090E1A0E0B0E08093781590937915F5
:104A8000A0937A15B0937B150E9407E110928115CF
:104A900010928015009374151093771586E190E1BC
:104AA000A0E0B0E08093781590937915A0937A15E3
:104AB000B0937B150E9407E162E070E080E090E037
:104AC0000E949964109281151092801500937415BC
:104AD0001093771580E190E1A0E0B0E08093781525
:104AE00090937915A0937A15B0937B150E9407E1F6
:104AF00010928115109280150093741510937715FC
:104B000082E190E1A0E0B0E0809378159093791570
:104B1000A0937A15B0937B150E9407E10EE814E08C
:104B2000F80181918F01882319F00E94E64DF8CF9A
:104B300081E09AE590938115809380158DE290E055
:104B4000909383158093821587E08093741582E893
:104B5000809377150C9449348330910549F581E0B1
:104B60008093730208EB14E0D8018D918D018823A6
:104B7000C9F00E94E64DF8CF809128159091291533
:104B8000A0912A15B0912B15823330E19307A1052E
:104B9000B10509F079C480913015909131150097D5
:104BA00009F03AC480911102882309F404C314C3A4
:104BB000049711F00C942C33109273020C942C3344
:104BC000809130159091311581309105D9F4109272
:104BD000730280911102882319F082E090E002C0F4
:104BE00083E090E0909381158093801585E0809319
:104BF000741582E8809377158EE190E1A0E0B0E033
:104C00000C944D348230910519F502EE14E0F80150
:104C100081918F01882319F00E94E64DF8CF81E041
:104C20008093730280910718843049F081E09AE5FF
:104C3000909381158093801585E390E081CF81E08A
:104C40009AE5909381158093801586E390E078CF64
:104C50008330910509F04CC020911102222319F1F3
:104C6000909381158093801585E08093741582E878
:104C7000809377158EE190E1A0E0B0E08093781505
:104C800090937915A0937A15B0937B150E9407E154
:104C900040E060E070E088EC92E40F942C00109209
:104CA00011020C942C3382E090E090938115809354
:104CB000801585E08093741582E8809377158EE1E6
:104CC00090E1A0E0B0E08093781590937915A093DF
:104CD0007A15B0937B150E9407E140E060E070E038
:104CE000CB010F942C0081E0809311020C942C33A3
:104CF000049711F00C942C33809153098823F1F020
:104D000082E090E0909381158093801585E08093F8
:104D1000741582E8809377158FE190E1A0E0B0E010
:104D20008093781590937915A0937A15B0937B159D
:104D30000E9407E1109253090C942C3383E090E019
:104D4000909381158093801585E08093741582E897
:104D5000809377158FE190E1A0E0B0E08093781523
:104D600090937915A0937A15B0937B150E9407E173
:104D700081E0809353090C942C33009130151091ED
:104D80003115B80180E090E00F94A7146B017C010D
:104D900020E030E040E251E40F94A21487FD0DC002
:104DA00020E030E04AEF53E4C701B6010F94061E3D
:104DB000181634F0902F812F05C09AE080E002C0D1
:104DC00094EF81E090936C0280936D020C942C33ED
:104DD0008091281590912915A0912A15B0912B1535
:104DE0008830F0E19F07A105B10509F050C081E0CE
:104DF0009AE590938115809380158DE290E09093D1
:104E000083158093821587E08093741512E81093C0
:104E1000771584E890E0A0E0B0E080937815909357
:104E20007915A0937A15B0937B150E9407E1109233
:104E300081151092801505E0009374151093771575
:104E400080E190E1A0E0B0E080937815909379152F
:104E5000A0937A15B0937B150E9407E110928115FB
:104E600010928015009374151093771582E190E1EC
:104E7000A0E0B0E08093781590937915A0937A150F
:104E8000B0937B150E9407E10E94BDFF8FC08A305E
:104E900000E19007A105B105E1F5809130159091F1
:104EA0003115813F910511F00C942C3381E09AE586
:104EB000909381158093801586E390E090938315FD
:104EC0008093821587E08093741582E8809377152C
:104ED00084E890E0A0E0B0E0809378159093791595
:104EE000A0937A15B0937B150E9407E14FE255E03D
:104EF00066E375E084E00E94409D60E087EC96E305
:104F00000E947EFF85E295E090937909809378096D
:104F10004DC08C309041A105B10509F047C080918A
:104F2000301590913115019709F040C00F945E0F34
:104F30001092071881E0809373028CE090E09093C8
:104F400081158093801585E08093741512E8109385
:104F5000771584E190E1A0E0B0E08093781590931C
:104F60007915A0937A15B0937B150E9407E181E033
:104F70009AE5909381158093801585E390E0909356
:104F800083158093821587E08093741510937715AD
:104F900084E890E0A0E0B0E08093781590937915D4
:104FA000A0937A15B0937B150E9407E18091281594
:104FB00090912915A0912A15B0912B158C30904114
:104FC000A105B10511F00C942C338091301590910E
:104FD0003115029711F00C942C330F945E0F81E081
:104FE0008093F90710920718809373021092FC07C0
:104FF0001092FB0781E09AE59093811580938015CC
:1050000082E590E09DCD2091301530913115B901A8
:1050100080E090E037FF09C00F94A71420E030E053
:1050200040E857E40F94A51B02C00F94A71420E09A
:1050300030E048EC52E40F94A01C6B017C0120E0AE
:1050400030E040EA51EC0F94061E00917B13109162
:105050007C1387FD2BC020E030E040EA51E4C7011B
:10506000B6010F94A21418160CF1B801110F880B99
:10507000990B0F94A914A70196010F94A51B20E08A
:1050800030E048EC53E40F94081590580F94121D2B
:10509000CB010E947FE4C701B6010E94A06381E5B5
:1050A00096E0909379098093780926C0B801110F92
:1050B000880B990B0F94A91420E030E048EC52E4DF
:1050C0000F9408150F94121D70938115609380152D
:1050D00085E08093741582E88093771586E290E1ED
:1050E000A0E0B0E08093781590937915A0937A159D
:1050F000B0937B150E9407E160917B1370917C1344
:10510000072E000C880B990B0F94A9148E010B5ECF
:105110001F4F23E041E00F947A0F9F938F9383E416
:1051200096E09F938F93045111091F930F930F944F
:105130003A14C8010E9473650F900F900F900F9062
:105140000F900F900C942C33809130159091311565
:10515000009729F481E0809373020C942C33813002
:105160009105B1F480911102882349F081E09AE51C
:1051700090938115809380158CE390E0E1CC81E0E1
:105180009AE590938115809380158BE390E0D8CCBD
:1051900082309105F9F28330910539F58091110241
:1051A00040E0882389F060E070E088EC92E40F949E
:1051B0002C001092110281E09AE590938115809362
:1051C000801589E390E0BCCC60E070E0CB010F94E7
:1051D0002C0081E08093110281E09AE59093811583
:1051E000809380158AE390E0ABCC8530910599F5EA
:1051F0000F94670084EB90E00E9491991092DD0C6F
:105200001092DE0C1092DF0C1092E00C1092E10C68
:105210000E94F4AA86E490E00E94AF9A84EB90E0AA
:10522000909381158093801505E00093741512E822
:105230001093771584E390E1A0E0B0E080937815B7
:1052400090937915A0937A15B0937B150E9407E18E
:1052500086E490E036C08630910509F040C00F9496
:10526000670080EF90E00E9491991092DD0C1092FF
:10527000DE0C1092DF0C1092E00C1092E10C0E94F8
:10528000F4AA8EE690E00E94AF9A80EF90E09093AF
:1052900081158093801505E00093741512E8109332
:1052A000771584E390E1A0E0B0E0809378159093C7
:1052B0007915A0937A15B0937B150E9407E18EE6CD
:1052C00090E090938115809380150093741510934E
:1052D00077158AE390E1A0E0B0E00C944D34813F73
:1052E000910511F00C942C3340E060E070E0CB01AC
:1052F0000F942C0041E060E070E0CB010F942C0093
:10530000109211020F94670080E090E00E94919942
:105310001092DD0C1092DE0C1092DF0C1092E00C5B
:105320001092E10C0E94F4AA80E090E00E94AF9AF3
:10533000109281151092801505E00093741512E803
:105340001093771584E390E1A0E0B0E080937815A6
:1053500090937915A0937A15B0937B150E9407E17D
:1053600061E070E080E090E00E9499641092811505
:105370001092801500937415109377158AE390E1CD
:10538000A0E0B0E08093781590937915A0937A15FA
:10539000B0937B150E9407E161E070E080E090E04F
:1053A0000E94996484E190E0909381158093801528
:1053B000009374151093771584E190E1A0E0B0E0BC
:1053C0008093781590937915A0937A15B0937B15F7
:1053D0000E9407E181E09AE5909381158093801502
:1053E00089E390E0909383158093821587E0809302
:1053F00074151093771584E890E0A0E0B0E08093F6
:10540000781590937915A0937A15B0937B150E9427
:1054100007E182E00C94253381309105B1F40F94BB
:10542000670080E090E00E9491991092811510929F
:10543000801585E08093741582E88093771584E366
:1054400090E1A0E0B0E00C944D34029711F00C9480
:105450002C331092DD0C1092DE0C1092DF0C1092A7
:10546000E00C1092E10C0E94F4AA80E090E00E940F
:10547000AF9A109281151092801585E08093741573
:1054800082E88093771525CF8433E0E19E07A1055C
:10549000B105D9F400913015109131150F946700C2
:1054A000B80180E090E00F94A71420E030E046E9D6
:1054B00053E40F94061E181614F0C80102C08CE2C3
:1054C00091E00E9491990C942C338A339041A1056C
:1054D000B10511F00C942C33009130151091311559
:1054E0001092DD0C1092DE0C1092DF0C1092E00C8A
:1054F0001092E10C0E94F4AAB80180E090E00F94B1
:10550000A71420E030E04CE053E40F94061E181678
:1055100014F0C80102C08CE890E00E94AF9A0C948D
:105520002C338091301590913115009709F412CEEB
:105530008130910509F04CC08091E40D882319F069
:1055400083E090E002C082E090E090938115809328
:10555000801585E08093741582E88093771585E443
:1055600090E1A0E0B0E08093781590937915A09336
:105570007A15B0937B150E9407E18AE090E0909342
:1055800081158093801585E08093741582E880935F
:10559000771580E092E1A0E0B0E0809378159093D9
:1055A0007915A0937A15B0937B150E9407E10E94AC
:1055B0008263811103C083E396E002C087E296E034
:1055C000909379098093780982E08093081886C1C6
:1055D0008230910509F0ADC081E08093730288E0CC
:1055E000EFEEF7E0DF011D928A95E9F780E090E0A9
:1055F000A0E2B1E48093EF079093F007A093F10746
:10560000B093F2078093F3079093F407A093F50704
:10561000B093F60784E690E090938115809380150F
:1056200005E00093741512E81093771584E590E176
:10563000A0E0B0E08093781590937915A0937A1547
:10564000B0937B150E9407E120E030E040E251E496
:105650006091F3077091F4078091F5079091F60738
:105660000F9408150F94121D709381156093801587
:10567000009374151093771588E590E1A0E0B0E0F1
:105680008093781590937915A0937A15B0937B1534
:105690000E9407E120E030E0A901609129097091A2
:1056A0002A0980912B0990912C090F94A61B0F9425
:1056B000121D7093811560938015009374151093DB
:1056C000771586E390E1A0E0B0E0809378159093A1
:1056D0007915A0937A15B0937B150E9407E180910C
:1056E0002D0990912E099093811580938015009338
:1056F00074151093771584E390E1A0E0B0E08093F7
:10570000781590937915A0937A15B0937B150E9424
:1057100007E162E070E080E090E00E94996481E03F
:105720009AE5909381158093801581E490E00C9424
:1057300040348330910509F086C01092FD0720E0C7
:1057400030E040E251E46091CC0D7091CD0D80913C
:10575000CE0D9091CF0D0F9408150F94121D7093DC
:1057600081156093801505E00093741512E810937D
:10577000771588E490E1A0E0B0E0809378159093ED
:105780007915A0937A15B0937B150E9407E120E06C
:1057900030E040E251E46091D00D7091D10D8091E4
:1057A000D20D9091D30D0F9408150F94121D709384
:1057B00081156093801500937415109377158AE412
:1057C00090E1A0E0B0E08093781590937915A093D4
:1057D0007A15B0937B150E9407E120E030E040E2AB
:1057E00051E46091D40D7091D50D8091D60D9091BA
:1057F000D70D0F9408150F94121D709381156093A7
:10580000801500937415109377158CE490E1A0E057
:10581000B0E08093781590937915A0937A15B093A2
:105820007B150E9407E162E070E080E090E00E945A
:10583000996481E09AE5909381158093801587E4BF
:1058400090E00C9440348430910509F405C785300C
:10585000910549F44EE750E160E070E089E095E0A1
:105860000E94C5E1F9C6069709F0F6C683E296E004
:1058700090937909809378098BE090E053C28091EE
:10588000301590913115019711F51092730281E056
:105890009AE590938115809380158FE390E0909323
:1058A00083158093821587E08093741582E8809336
:1058B000771584E890E0A0E0B0E0809378159093AD
:1058C0007915A0937A15B0937B150E9407E180911A
:1058D000301590913115029709F0BEC681E09AE526
:1058E000909381158093801580E490E029C9809180
:1058F0003015909131158E35910509F4A5C168F5E3
:105900008330910509F45FC1A0F48130910509F459
:105910006EC1029709F000C242E060E070E080E8EA
:1059200090E40E94D56340E060E070E08BE893E48F
:105930006AC18430910509F473C1059709F0ECC17F
:1059400042E060E070E080E890E40E94D56340E0CF
:1059500060E070E08BE893E46FC18136910509F453
:1059600069C098F58F35910509F48AC08036910594
:1059700009F0D2C183E08093081883E090E090930F
:1059800081158093801585E08093741582E880935B
:1059900077158DE890E1A0E0B0E0809378159093C2
:1059A0007915A0937A15B0937B150E9407E1E12C3D
:1059B000F12C00E0DD24D394AA24A39475E0972E63
:1059C000E5E08E2EF2E87F2E85C08236910561F0EB
:1059D0008336910509F0A0C180917B1380FF76C6C4
:1059E000869580FD76C672C660917B1370917C139C
:1059F000072E000C880B990B0F94A9142DEC3CEC8E
:105A00004CEC5DE30F94A61B6B017C0120E030E0C1
:105A100040EA51EC0F94061E87FD82C120E030E081
:105A200040EA51E4C701B6010F94A21418160CF015
:105A300057C676C160917B1370917C13072E000CC2
:105A4000880B990B0F94A9142DEC3CEC4CEC5DE306
:105A50000F94A51B6B017C0120E030E040EA51EC83
:105A60000F94061E87FD5CC120E030E040EA51E45F
:105A7000C701B6010F94A21418160CF094C650C1B9
:105A800080E00E94DE4C0E948263811103C08AEC98
:105A900095E002C08CEB95E09093790980937809AA
:105AA00082E08093081881E09AE5909381158093B5
:105AB000801584E590E0909383158093821587E0AC
:105AC0008093741582E88093771584E890E0A0E0D5
:105AD000B0E017C1DD2031F0CC24C39465E0B62ED0
:105AE00010E005C0CC24CA94BB24BA9414E0DA2494
:105AF000B116D1F1802F90E04897A4F50F5FF70120
:105B0000919EE00DF11D1124EE0FFF1FEE0FFF1F00
:105B1000EE5EF34F20E030E04AE754E460817181AB
:105B2000828193810F9408150F94121D7093811533
:105B3000609380158092741570927715802F90E095
:105B40008158974F880F991F092E000CAA0BBB0B89
:105B50008093781590937915A0937A15B0937B155F
:105B60000E9407E11C0DC4CFBFEFEB1AFB0AE5E072
:105B7000EE16F10409F0AECF81E09AE5909381151D
:105B80008093801585E590E090938315809382152E
:105B900087E08093741582E88093771584E890E01D
:105BA000A0E0B0E08093781590937915A0937A15D2
:105BB000B0937B150E9407E188EB95E090937909FB
:105BC00080937809ADC042E060E070E080E890E446
:105BD0000E94D56340E060E070E086E193E40E94BB
:105BE000D56341E060E070E086E193E413C042E0F9
:105BF00060E070E080E890E40E94D56340E060E0FF
:105C000070E080EB91E40E94D56341E060E070E0D9
:105C100080EB91E40E94D56386E08093081880C0F1
:105C200042E060E070E080E890E40E94D56340E0EC
:105C300060E070E080EB91E40E94D56341E060E0B9
:105C400070E08BE893E4E6CF8091E40D81111CC0F5
:105C500083E090E0909381158093801585E0809398
:105C6000741582E88093771585E490E1A0E0B0E0B8
:105C70008093781590937915A0937A15B0937B153E
:105C80000E9407E181E01BC082E090E090938115C3
:105C90008093801585E08093741582E88093771552
:105CA00085E490E1A0E0B0E08093781590937915B9
:105CB000A0937A15B0937B150E9407E180E00E94C3
:105CC000DE4C60917B1370917C13072E000C880BC7
:105CD000990B0F94A91420E030E048EC52E40F94A3
:105CE00008150F94121D709381156093801585E03F
:105CF0008093741582E88093771586E290E1A0E0A6
:105D0000B0E08093781590937915A0937A15B093AD
:105D10007B150E9407E104C08CE995E00E94C24F08
:105D20008AE090E0909381158093801585E08093C0
:105D3000741582E8809377154EC184E0809308182B
:105D40008091281590912915A0912A15B0912B15B5
:105D500060913015709131158834F0E19F07A105ED
:105D6000B10509F453C08A3400E19007A105B105DB
:105D700009F454C08C3410E19107A105B10509F470
:105D800056C086349041A105B10509F058C0633072
:105D90007105B9F58BE895E09093790980937809BE
:105DA00081E08093FE07809373021092EE0781E0FA
:105DB0009AE590938115809380158AE490E0909302
:105DC00083158093821587E08093741512E81093F1
:105DD000771584E890E0A0E0B0E080937815909388
:105DE0007915A0937A15B0937B150E9407E18AE09C
:105DF00090E0909381158093801585E080937415D1
:105E0000E8C06093FD071092081826C4412C512C5D
:105E100036E9632E33E4732E312C11C0412C512C02
:105E200026E9622E23E4722E3324339408C0412CD9
:105E3000512C88EC682E83E4782E92E0392E80E095
:105E400090E00F94A71420E030E040E251E40F947A
:105E5000A01C6B017C0120E030E0A9010F94A2148A
:105E600087FF09C01092E8071092E9071092EA072D
:105E70001092EB0719C0A3019201C701B6010F945C
:105E8000061E18164CF0C092E807D092E907E0927F
:105E9000EA07F092EB0708C04092E8075092E90742
:105EA0006092EA077092EB076091E8077091E9074A
:105EB0008091EA079091EB07432D0E94D56361E042
:105EC00070E080E090E00E94996420E030E040E2E1
:105ED00051E46091CC0D7091CD0D8091CE0D9091DB
:105EE000CF0D0F9408150F94121D709381156093B8
:105EF000801505E00093741512E81093771588E477
:105F000090E1A0E0B0E08093781590937915A0938C
:105F10007A15B0937B150E9407E120E030E040E263
:105F200051E46091D00D7091D10D8091D20D90917E
:105F3000D30D0F9408150F94121D70938115609363
:105F4000801500937415109377158AE490E1A0E012
:105F5000B0E08093781590937915A0937A15B0935B
:105F60007B150E9407E120E030E040E251E46091BF
:105F7000D40D7091D50D8091D60D9091D70D0F94C1
:105F800008150F94121D709381156093801500936E
:105F90007415109377158CE490E1A0E0B0E0809345
:105FA000781590937915A0937A15B0937B150E947C
:105FB00007E161E070E080E090E00E949964109257
:105FC00008188AE090E090938115809380150093E3
:105FD00074151093771580E092E1A0E0B0E05DC405
:105FE0008091281590912915A0912A15B0912B1513
:105FF000863530E19307A105B10509F046C020E0E0
:1060000030E0A9016091290970912A0980912B093A
:1060100090912C090F94A61B20E030E04AE253E453
:106020000F94A214209130153091311587FF40C490
:106030002530310508F03CC48AEA90E09093811540
:106040008093801585E08093741512E8109377157E
:1060500080E290E1A0E0B0E080937815909379150C
:10606000A0937A15B0937B150E9407E165E070E07C
:1060700080E090E00E94996481E09AE59093811518
:106080008093801582E490E0FBC38435E0E19E07B5
:10609000A105B105B9F4609130157091311580E01A
:1060A00090E00F94A71420E030E040E251E40F9418
:1060B000A01C6093EF077093F0078093F107909313
:1060C000F207CAC288359041A105B10509F0C4C2E2
:1060D000609130157091311580E090E00F94A71415
:1060E00020E030E040E251E40F94A01C6093F307FD
:1060F0007093F4078093F5079093F607ADC2609113
:1061000030157091311585E795E00E94004F809120
:1061100030159091311582309105A1F038F4009737
:1061200071F00197E1F482E395E094C28430910527
:1061300079F058F0059799F48AE495E00BC08CE16A
:1061400095E088C287E695E005C08DE595E002C040
:1061500088E595E090937909809378097DC286E47B
:1061600095E078C285E595E00E94C24F8091301598
:10617000909131158130910509F054C00E94C96396
:10618000811103C0649B08C067C2813009F064C2FA
:106190008091030180FD60C283E695E00E94C24FBA
:1061A00081E00E94299C8DE090E09093811580937E
:1061B000801585E08093741512E81093771584E1BB
:1061C00090E1A0E0B0E08093781590937915A093CA
:1061D0007A15B0937B150E9407E183E0809307183E
:1061E00081E09AE5909381158093801585E390E096
:1061F000909383158093821587E080937415109394
:10620000771584E890E0A0E0B0E080937815909353
:106210007915A0937A15B0937B150E9407E110922F
:10622000E4071AC2892B09F017C28BE795E00E9498
:10623000C24F8091E407813039F581E995E00E94F1
:10624000C24F81E09AE590938115809380158EE28C
:1062500090E0909383158093821587E08093741566
:1062600082E88093771584E890E0A0E0B0E0809326
:10627000781590937915A0937A15B0937B150E94A9
:1062800007E11092061835C0823069F485EA95E07E
:106290000E94C24F81E09AE590938115809380150A
:1062A00086E390E00EC0833031F589EB95E00E94E3
:1062B000C24F81E09AE5909381158093801581E427
:1062C00090E0909383158093821587E080937415F6
:1062D00082E88093771584E890E0A0E0B0E08093B6
:1062E000781590937915A0937A15B0937B150E9439
:1062F00007E11092F9171092E4070E94BDFFACC1AC
:1063000080913015909131158F3F910531F028F033
:106310008FEF90E0A0E0B0E002C0A0E0B0E080939A
:10632000120290931302A0931402B093150280916D
:10633000120290911302A0911402B09115020097DD
:10634000A105B10509F5109281151092801505E09F
:106350000093741512E8109377158AE890E1A0E095
:10636000B0E08093781590937915A0937A15B09347
:106370007B150E9407E189E090E09093811580935E
:106380008015009374153DC00196A11DB11D05E057
:10639000B695A795979587950A95D1F70197A10985
:1063A000B109009701E0A007B10550F0B093811545
:1063B000A0938015909383158093821587E005C084
:1063C000909381158093801585E08093741512E871
:1063D000109377158AE890E1A0E0B0E080937815FB
:1063E00090937915A0937A15B0937B150E9407E1DD
:1063F00088E090E0909381158093801585E08093EC
:106400007415109377158CE890E1A0E0B0E08093CC
:10641000781590937915A0937A15B0937B150E9407
:1064200007E18091120290911302A0911402B091A1
:106430001502BA2FA92F982F8827009711E0A107DE
:10644000B10550F0B0938115A093801590938315FA
:106450008093821587E005C0909381158093801505
:1064600085E08093741582E88093771581EA90E047
:10647000A0E0B0E012C28DEC95E00E94C24F0E94F5
:106480007663409128155091291560912A157091D5
:106490002B15882339F0433D20E252076105710531
:1064A00009F46EC3423D50426105710509F0D4C044
:1064B0008091301590913115019709F0B8C40E9470
:1064C0007663882309F4B3C48091431087FDC4C068
:1064D000A2E18A02C001112482509E4E0E943B70AC
:1064E000C12C90E2D92EE12CF12C05E012E810929B
:1064F0008115109280150093741510937715C09232
:106500007815D0927915E0927A15F0927B150E9459
:1065100007E1BFEFCB1ADB0AEB0AFB0AEAE0CE1673
:10652000E0E2DE06E104F10411F700914310F2E12C
:106530000F02800111240A561F4EF801019000201D
:10654000E9F7C8018E1B9F0B439697FD01967C01CE
:10655000F594E7941E141F040CF063C49E012F5F92
:106560003F4F690184E1D9011D928A95E9F7A7019E
:106570006EED75E0C9010F94191FB801C6018E0DAB
:106580009F1D0F94041F40E050E260E070E0C601E0
:106590000E94C5E162E070E080E090E00E949964B2
:1065A00040E060E070E08FE793E40F942C0041E05E
:1065B00060E070E08FE793E40F942C0010921102DA
:1065C0008DE090E0909381158093801585E0809315
:1065D000741512E81093771584E190E1A0E0B0E023
:1065E0008093781590937915A0937A15B0937B15C5
:1065F0000E9407E162E070E080E090E00E94996410
:1066000081E09AE5909381158093801585E390E071
:10661000909383158093821587E08093741510936F
:10662000771584E890E0A0E0B0E08093781590932F
:106630007915A0937A15B0937B150E9407E181E04C
:10664000809373028093061883E08093071804C038
:106650008FE395E00E94C24F80E5E4E2F5E1DF01BF
:106660001D928A95E9F78AE58093251585EA80933E
:1066700026150C94821E8EEB93E10E94536EF70157
:10668000EC53FA4E80838091C4158A3581F01E1434
:106690001F0414F00C94A81FD601E02F1D92EA9558
:1066A000E9F71092ED071092EC070C94A81F62E036
:1066B00070E080E090E00E949964FFEFEF1AFF0A1B
:1066C000F092ED07E092EC070C94A81F83E196E0AE
:1066D00002C082E096E09093790980937809F1CA2C
:1066E00088E290E00E947FE460917B1370917C13BC
:1066F000072E000C880B990B0F94A9142DEC3CEC81
:106700004CEC5DE30F94A61B0E94A06360917B1389
:1067100070917C13072E000C880B990B0F94A91411
:1067200020E030E048EC52E40F9408150F94121D5D
:10673000709381156093801585E08093741582E8CD
:106740008093771586E290E1A0E0B0E08093781521
:1067500090937915A0937A15B0937B150E9407E169
:1067600060917B1370917C13072E000C880B990BA2
:106770000F94A9148E010B5E1F4F23E041E00F948C
:106780007A0F9F938F9384EF95E09F938F9304519B
:1067900011091F930F930F943A14C8010E94736557
:1067A0008FEE95E062C088ED9FEF0E947FE46091DC
:1067B0007B1370917C13072E000C880B990B0F94A0
:1067C000A9142DEC3CEC4CEC5DE30F94A51B0E944E
:1067D000A06360917B1370917C13072E000C880BD3
:1067E000990B0F94A91420E030E048EC52E40F9488
:1067F00008150F94121D709381156093801585E024
:106800008093741582E88093771586E290E1A0E08A
:10681000B0E08093781590937915A0937A15B09392
:106820007B150E9407E160917B1370917C13072E0A
:10683000000C880B990B0F94A9148E010B5E1F4F4F
:1068400023E041E00F947A0F9F938F9381EE95E0C0
:106850009F938F93045111091F930F930F943A1430
:10686000C8010E9473658CED95E09093790980933F
:1068700078090F900F900F900F900F900F9050CAC3
:10688000909383158093821587E0809374151093FD
:10689000771584E890E0A0E0B0E0809378159093BD
:1068A0007915A0937A15B0937B150E9407E1D4CE99
:1068B0002430310589F481E00F94FB0B2091F3071C
:1068C0003091F4074091F5075091F6070F94A61BFD
:1068D00041E00F94CD0BBBC02530310508F4FCC05E
:1068E0002630310509F439C108F02BC181E08093CD
:1068F000F7070F9467008EEB90E00E94919920E0DB
:1069000030E0A9016091290970912A0980912B0931
:1069100090912C090F94A61B20E030E048EC52E443
:106920000F9408156B017C0160912D0970912E095F
:10693000072E000C880B990B0F94A9149B01AC0136
:10694000C701B6010F94A01C0F94191D6436710580
:1069500010F064E670E0709381156093801505E097
:106960000093741512E81093771584E290E1A0E08B
:10697000B0E08093781590937915A0937A15B09331
:106980007B150E9407E120E030E0A9016091290910
:1069900070912A0980912B0990912C090F94A61BC4
:1069A0000F94121D709381156093801500937415D8
:1069B0001093771586E390E1A0E0B0E0809378151E
:1069C00090937915A0937A15B0937B150E9407E1F7
:1069D00080912D0990912E099093811580938015B7
:1069E000009374151093771584E390E1A0E0B0E074
:1069F0008093781590937915A0937A15B0937B15B1
:106A00000E9407E165E070E080E090E00E949964F8
:106A100081E09AE5909381158093801584E490E05D
:106A2000909383158093821587E08093741510935B
:106A3000771584E890E0A0E0B0E08093781590931B
:106A40007915A0937A15B0937B150E9407E120E099
:106A500030E040E251E46091EF077091F0078091DF
:106A6000F1079091F2070F9408150F94121D70937F
:106A700081156093801505E00093741512E810935A
:106A8000771584E590E1A0E0B0E0809378159093CD
:106A90007915A0937A15B0937B150E9407E120E049
:106AA00030E040E251E46091F3077091F407809187
:106AB000F5079091F6070F9408150F94121D709327
:106AC000811560938015009374151093771588E5F0
:106AD00090E1A0E0B0E0E1CE2230310579F480E031
:106AE0000F94FB0B2091EF073091F0074091F107D5
:106AF0005091F2070F94A61B40E0EBCE23303105F6
:106B000070F081E00F94FB0B2091F3073091F407B4
:106B10004091F5075091F6070F94A51BD9CE21306F
:106B2000310509F094CF80E00F94FB0B2091EF0723
:106B30003091F0074091F1075091F2070F94A51B97
:106B4000DBCF213F310509F082CF1092F70761E0DA
:106B500070E080E090E00E94996481E09AE5909373
:106B600081158093801581E490E090938315809344
:106B7000821587E08093741582E88093771559CF4A
:106B80008BE296E00E94C24F809144109091451094
:106B9000992720913015309131158217930708F409
:106BA0005BCD86ED95E00E94C24F809130158150FB
:106BB00080934310A4ED8A2EA0E29A2EA12CB12C32
:106BC00005E012E81092811510928015009374155B
:106BD000109377158092781590927915A0927A1576
:106BE000B0927B150E9407E13FEF831A930AA30A34
:106BF000B30A8EED881680E29806A104B10411F75D
:106C000080914310A2E18A02C0011124FC01EA56DE
:106C1000FF4E7F0101900020E9F7C7018E1B9F0BFB
:106C2000439697FD01968C01159507951016110650
:106C3000FCF49E012F5F3F4F690184E1D9011D9251
:106C40008A95E9F7A8016EED75E0C9010F94191F47
:106C5000B701C601800F911F0F94041F44ED50E24D
:106C600060E070E0C6010E94C5E105E012E806C0E0
:106C700044ED50E260E070E0C701F5CF109281155D
:106C800010928015009374151093771580927815E3
:106C900090927915A0927A15B0927B150E9407E127
:106CA000BFEF8B1A9B0AAB0ABB0AE6EE8E16E0E238
:106CB0009E06A104B10411F78E010F5F1F4F84E1FE
:106CC000D8011D928A95E9F7809145108F938091A4
:106CD00044108F93809131158F93809130158F934D
:106CE00088EE95E09F938F931F930F930F94331F1C
:106CF0004EED50E260E070E0C8010E94C5E162E044
:106D000070E080E090E00E9499640FB6F894DEBFD6
:106D10000FBECDBF31E2C32E32E1D32EE12CF12CD8
:106D200043E1442E40E6542E612C712C8824839438
:106D3000912CAA24AA94BA2C75E0272EE2E83E2EC4
:106D40000AE010E080914410909145108815990553
:106D500094F1B0928115A092801520927415309212
:106D60007715409278155092791560927A15709245
:106D70007B150E9407E110938115009380152092E6
:106D8000741530927715C0927815D0927915E092EB
:106D90007A15F0927B150E9407E1FFEF8F1A9F0A88
:106DA00020E1420E511C611C711C3FEFC31AD30A33
:106DB000E30AF30AC7CF809130159091311524E092
:106DC000880F991F2A95E1F78D5F9F49A0E0B0E0F9
:106DD00020EF37E8309381152093801505E000936C
:106DE000741512E8109377158093781590937915A0
:106DF000A0937A15B0937B150E9407E1809130151E
:106E000090913115805E9D4EA0E0B0E026E030E02C
:106E10003093811520938015009374151093771586
:106E20003CCD40E050E260E070E0C801B1CB809121
:106E3000301590913115892B11F40C94AA280CCCA3
:106E4000A7960FB6F894DEBF0FBECDBFDF91CF91EE
:106E50001F910F91FF90EF90DF90CF90BF90AF9078
:106E60009F908F907F906F905F904F903F902F906A
:106E700008952F923F924F925F926F927F928F92DE
:106E80009F92AF92BF92CF92DF92EF92FF920F93B9
:106E90001F93CF93DF93CDB7DEB7C154D1090FB69F
:106EA000F894DEBF0FBECDBF22968FAF2297209100
:106EB00014082CAF81E08093140880918D178D34D5
:106EC00009F405C4843511F40C946848873411F032
:106ED0000C94794880918B1790918C178A31910589
:106EE00009F426C1B4F48430910534F4823091055C
:106EF000DCF597FF2DC0E7C38C30910509F414C170
:106F00008531910511F40C947B48049709F0DBC39B
:106F1000CCC08A32910509F457C354F48C319105E1
:106F200009F424C10CF408C14D9709F42FC1CBC357
:106F30008B35910509F4C7C28C35910509F4C8C297
:106F40008A35910509F0BFC3109213080C947B4851
:106F500080914802882311F40C947B480E948FD2C0
:106F60000E94E5DA0C947B4820914802222311F418
:106F70000C947B4811E0029709F010E00E948FD238
:106F800019821A821B821C821D821E821F82188611
:106F900082E50E94759B882309F457C00E94F59AE8
:106FA0006B017C0120E030E0A9010F94A21488233A
:106FB00009F461C08091CC0D9091CD0DA091CE0DC2
:106FC000B091CF0D88A799A7AAA7BBA78091D00D94
:106FD0009091D10DA091D20DB091D30D8CA79DA70A
:106FE000AEA7BFA78091AA0D9091AB0DA091AC0D5B
:106FF000B091AD0D88AB99ABAAABBBAB8091AE0D98
:107000009091AF0DA091B00DB091B10D8CAB9DAB37
:10701000AEABBFAB28A939A94AA95BA968A579A5D8
:107020008AA59BA50F94A21481110C949F482CA9AA
:107030003DA94EA95FA96CA57DA58EA59FA50F941E
:10704000A2148823C1F00C949F4889E40E94759B88
:10705000882331F00E94F59A69837A838B839C831D
:107060008AE40E94759B882331F00E94F59A6D8313
:107070007E838F83988720E030E0A90169817A813F
:107080008B819C810F94A21481110C94A44920E05F
:1070900030E0A9016D817E818F8198850F94A214C3
:1070A00081110C94A4490C94B74980E50E94759B0A
:1070B000882329F00E94CFF26B017C0103C0C12C10
:1070C000D12C760183E50E94759B882361F00E9494
:1070D000F59A20E030E04AE754E40F9408150F9445
:1070E000191D6B017C010E94497A80917C138111EA
:1070F00005C060E089EE96E00E947EFF0E9483D288
:10710000C60ED71EE81EF91E0E9483D2DC01CB01F9
:107110008C199D09AE09BF09B7FD02C00C947B48CC
:1071200080E00E94E34FF0CF0E9471D50C947B4821
:107130000E9477BF0C947B480E9459CF81110C9418
:107140007B488CE0E0EEF2E0DE01119601900D92BA
:107150008A95E1F760E070E080E50E945ED5BE01AF
:107160006F5F7F4F0E9401FE0C947B488091BB0DA6
:107170008770873011F00C94BE4960E08FE40E9464
:10718000829B81110C947B480C94BE4960E083E59E
:107190000E946BF4182F863030F08BED97E00E9440
:1071A000F84D0C947B48833009F405C128F48130F4
:1071B000E9F0823049F106C0843009F452C18530CB
:1071C00009F45FC188EC97E00E94F84D0E94F94CE9
:1071D000882339F08091E40D0E94074E0E9436A06A
:1071E00056C18AEB97E00E94F84D51C10E94CCA095
:1071F00010920102109200028FEA97E090937909B1
:10720000809378090C947B48809100029091010250
:1072100097FF06C086E897E00E94F84D0C947B48E3
:107220000097A1F480916B0280931B0819821A8247
:107230001B821C821C8E1D8E1E8E1F8EBE016F5FD8
:107240007F4FCE014C960E9453DF27C0815065E0EE
:107250000F945B1B80FF03C024E0291B922F25E0C5
:107260009202F0011124E80FF11D87FDFA95EE0F4F
:10727000FF1FEE0FFF1FEE5EF34F8091D40D909134
:10728000D50DA091D60DB091D70D80839183A283A7
:10729000B38380911B0880936B02809100029091D0
:1072A0000102893191050CF058C010926B029C01CB
:1072B0002F5F3F4F309301022093000265E00F944F
:1072C0005B1B80FF03C024E0291B922F34E0930254
:1072D000F0011124E950FA4E80809180A280B380A1
:1072E00094E08902F0011124ED51FA4E4080518062
:1072F000628073808DEC9CECACE4BEE38C8F9D8F40
:10730000AE8FBF8F19821A821B821C82DE011196FA
:107310006D01E12CF12C00EA10E4A3019201C501FA
:10732000B4010E9474DE19821A821B821C82B6018B
:10733000CE014C960E9453DF8092CC0D9092CD0DE1
:10734000A092CE0DB092CF0D4092D00D5092D10DA3
:107350006092D20D7092D30D9CC080E090E0A0EAC4
:10736000B0E48093D40D9093D50DA093D60DB09337
:10737000D70D81E692E00E9455DE0E94497A8FEF98
:107380009FEF909301028093000282E797E00E94B2
:10739000F84D63E972E084E690E00E941FFF6AEB1B
:1073A00072E084E690E00E941FFF0E9457D081E0C7
:1073B0000E94DE4C6EC089E40E94759B8823B1F068
:1073C0000E94F19A182F853060F064E070E08FE53C
:1073D00097E00E94294F8CE597E00E94F84D0C94AD
:1073E0007B488AE40E94759B811105C08AE40F9452
:1073F000580F0C947B480E94F19A082F853060F05A
:1074000064E070E089E497E00E94294F86E497E009
:107410000E94F84D0C947B488AE50E94759B882356
:10742000D9F00E94F59A9B01AC01B5E01B02F00176
:107430001124E00FF11D07FDFA95EE0FFF1FEE0F6F
:10744000FF1FEE5EF34F6083718382839383602F0F
:10745000812F0E94B46433C08AE50F94580F0C94B6
:107460007B488AE50E94759B8823B1F30E94F59AB8
:1074700060930E0C70930F0C8093100C9093110C72
:107480001EC080E00E94DE4C0E94CCA018C01230CA
:10749000B1F460910002709101026931710514F03C
:1074A00069E170E087E397E00E94294F69E170E0AD
:1074B00082E397E00E94294F8AE00E94E64D0E94F5
:1074C0009ADF0C947B488FE0809313080C947B48E0
:1074D0006DE7262E63E0362E72E0E72E7CE0F72E75
:1074E000ECECFDE0FDA3ECA3E6EFCE2EEBE0DE2E10
:1074F00000E010E0D1018D911D010E94759B882351
:1075000009F44BC00E94F59A2B013C01133049F05D
:10751000F60120813181428153810F94A51B2B01FB
:107520003C01ACA1BDA12D913D914D915C91C30158
:10753000B2010F94A51B4B015C012DEB37E346E82C
:1075400055EB0F94061E87FD0AC02DEB37E346E886
:1075500055E3C501B4010F94A2141816F4F41330C6
:1075600051F44092D80D5092D90D6092DA0D70927C
:10757000DB0D01E012C0A5019401F701608171816A
:10758000828193810F94A61BD7016D937D938D9378
:107590009C931397812F0E945D801F5FB4E0EB0ED8
:1075A000F11CECA1FDA13496FDA3ECA3F4E0CF0EF9
:1075B000D11C143009F09ECF002309F480CF88ED50
:1075C0009DE00E945A7A7BCF80914802882311F473
:1075D0000C947B4889E40E94759BF82E882321F047
:1075E0000E94F19A182F01C010E08AE40E94759B56
:1075F000082F882319F00E94F19A01C080E0FF2033
:1076000011F0153020F4002341F0853030F082EF86
:1076100097E00E94F84D0C947B4890E1ECECFDE083
:10762000AAEABDE001900D929A95E1F7FF2091F052
:1076300024E01202F0011124E950FA4E40815181F8
:10764000628173814093AA0D5093AB0D6093AC0D92
:107650007093AD0D002391F034E08302F00111240A
:10766000ED51FA4E80819181A281B3818093AE0D5C
:107670009093AF0DA093B00DB093B10D40E050E0EA
:10768000BA0186E40E94E2656B017C0120E030E0F3
:10769000A9010F94061E18164CF420E030E040E7D4
:1076A00052E4C701B6010F94A01C03C060E070E073
:1076B000CB0169837A838B839C83CE0101960E94E0
:1076C000EADD0C947B480E943FCF0C947B4880916C
:1076D0008B1790918C178537910509F4D3C70CF05F
:1076E00048C18B34910509F4DCC40CF067C08A31C1
:1076F000910509F455C39CF58431910509F4CFC275
:107700007CF48131910509F4B6C22CF4029708F497
:107710002FC20C946548429709F40BC70C94654836
:107720008731910509F4E0C28CF48531910509F4A3
:10773000D7C2469711F00C9465480E942270809140
:107740002417877F809324170C947B4888319105F8
:1077500009F4E2C2499709F418C30C9465488F31C3
:10776000910509F448C47CF48C31910509F48DC36A
:107770000CF424C38D31910509F491C34E9709F49B
:1077800095C30C9465488A32910509F454C464F495
:107790008032910509F4E9C3819711F00C94654892
:1077A0000E94516C0C947B488B32910509F466C49D
:1077B0008934910509F466C40C94654889369105AD
:1077C00009F4A4C5ECF58235910509F4A4C6FCF4CE
:1077D0008D34910509F46DC40CF467C48E349105A1
:1077E00009F46BC48135910511F00C9465480E9431
:1077F00043AB0F941C020E94F97B0E949F4D68EEE0
:1078000073E080E090E00E94264D0C947B48853523
:10781000910509F491C654F48335910509F482C6A3
:107820008435910509F485C60C9465488C3591051D
:1078300009F49BC68836910509F4D0C40C946548B8
:107840008E36910509F4A2C58CF48B36910509F4A6
:1078500093C50CF46BC58C36910511F40C947B48E0
:107860008D36910509F4ECC40C9465488137910577
:1078700009F4E2C55CF48F36910509F498C58037A8
:10788000910511F40C947B480C946548823791055E
:1078900009F4F5C68337910511F00C94654881E928
:1078A0009AE00E94F84D60E081E89AE00E942FEA99
:1078B00060E08CE69AE00E942FEA61E085E69AE0BB
:1078C0000E942FEA61E08AE59AE00E942FEA61E0D7
:1078D0008AE49AE00E942FEA60E081E49AE00E9444
:1078E0002FEA61E087E39AE00E942FEA60E08DE2F0
:1078F0009AE00E942FEA60E085E29AE00E942FEA77
:1079000061E087E19AE00E942FEA61E089E09AE075
:107910000E942FEA60E08AEF99E00E942FEA60E07F
:107920008CEE99E00E942FEA60E086ED99E00E94DB
:107930002FEA61E085EC99E00E942FEA61E086EB96
:1079400099E00E942FEA61E081EA99E00E942FEA23
:1079500061E08EE899E00E942FEA60E081E899E01A
:107960000E942FEA60E08DE699E00E942FEA0C94D5
:107970007B488D32A1E09A0711F40C948B450CF0F2
:107980006EC08B3C910509F45FC7ACF58D3791054E
:1079900009F4BEC5BCF48737910509F4BEC60CF4E2
:1079A00082C68837910509F4BBC68937910511F065
:1079B0000C94654810926809109267090E94F7E0DC
:1079C0000C947B488E3B910509F46AC554F48C38BD
:1079D000910509F453C58B39910509F473C50C94CD
:1079E0006548883C910509F4A3C6893C910509F4D2
:1079F00008C70C946548893D910509F46FC79CF44C
:107A00008D3C910509F445C70CF440C78E3C9105A7
:107A100009F442C7833D910511F00C9465480E941A
:107A2000B0D80C947B48823E910509F4BDC754F44C
:107A30008C3D910509F455C78D3D910509F45EC74C
:107A40000C9465488232E1E09E0711F40C942045C5
:107A50008C32914011F40C9476450C946548853F26
:107A600021E0920711F40C9449470CF044C08A3984
:107A7000A1E09A0711F40C947B48C4F48F32E1E042
:107A80009E0711F40C94C24614F40C947E46803385
:107A900021E0920711F40C940B468039914011F0CB
:107AA0000C9465480E94497A0C947B48853AA1E081
:107AB0009A0711F40C94E9467CF48C39E1E09E07B6
:107AC00011F40C94C546843A914011F00C94654829
:107AD0000E9477F40C947B488C3A21E0920711F4D1
:107AE0000C94EC46843F914011F00C9465480E9440
:107AF000BAB10C947B488835A2E09A0711F40C9433
:107B00007147B4F4873FE1E09E0711F40C944F47AE
:107B100014F40C944C47883F21E0920711F40C9424
:107B200058478C30924011F40C9469470C94654886
:107B30008438A3E09A0711F40C94EF476CF48B356A
:107B4000E2E09E0711F40C9474478C36934011F4D4
:107B50000C947B480C946548803A23E0920709F422
:107B60003AC2873E934011F40C9457480C946548F0
:107B70000091860B1091870B80E50E94759B8823EE
:107B800061F00E94CFF26B017C01BB24B394672BA0
:107B9000682B692B31F4B12C04C0B12CC12CD12C31
:107BA000760183E50E94759B882311F40C94A44B05
:107BB0000E94F59A20E030E04AE754E40F9408155B
:107BC0000F94191D6B017C01B1100BC0672B682B42
:107BD000692B39F40115110521F0D8018C9181111F
:107BE00002C0B12C02C0BB24B3940E94497AB110E8
:107BF00003C08AE396E001C0C8010E94B8651091F5
:107C0000140883E08093140881E08093F91743E21D
:107C100058E06CE278E082E00E94879C81E198E085
:107C20000E94B865C114D104E104F104B1F00E94CE
:107C300083D2C60ED71EE81EF91E0E9483D2DC0135
:107C4000CB018C199D09AE09BF09B7FF0EC0809109
:107C5000F91781110C94A94B08C08091F91788235A
:107C600021F080E00E94E34FF8CF1092F9171093B3
:107C700014080C947B488091871784FF02C00C94F1
:107C8000AE4B8091891787FF02C00C94AE4B809158
:107C90008A17837011F00C94AE4B0C94CB4B86E595
:107CA00098E00E94F84D84EB94E10E9470938BE180
:107CB000E4EBF4E1DE01119601900D928A95E1F773
:107CC00060E070E0CE0101960E942272CE01019622
:107CD0000E94A69487E498E00E94F84D0C947B489B
:107CE0000E9493700C947B48E091860BF091870B77
:107CF0008081882329F0803209F410823196F8CFF0
:107D000040E061E08091860B9091870B0E947F7329
:107D10001092FA170C947B488091880B8823E9F025
:107D200080E090E0A0EAB1E488A399A3AAA3BBA352
:107D30001C8E1D8E1E8E1F8E19821A821B821C8223
:107D400020E0AE01405E5F4FBE01645E7F4FCE011A
:107D500001960E94479D0C947B480E94914D882378
:107D600021F00E9433700F946C0161E08CEF96E378
:107D70000E94CD9B47E658E06FE678E085E00E94E0
:107D8000409D0F9402000C947B488091241782FF41
:107D900003C08B7F809324170E949BD40C947B4854
:107DA0008091241783FD02C00C947B4883E50E94D8
:107DB000759B81110C94DA4B0C947B4883E40E94F0
:107DC0002C9B8823C1F185E898E00E94F84D8091B2
:107DD0005E14882339F1BE016F5F7F4F8BE594E11C
:107DE0000E9437928E010F5F1F4FF80181918F0122
:107DF000882319F00E94E64DF8CFCE0101960E942B
:107E000051738091F40F882389F080E20E94E64D3F
:107E100004EF1FE0D8018D918D01882339F00E9475
:107E2000E64DF8CF8BE798E00E94F84D8AE00E947B
:107E3000E64D0C947B4883E50E94759B882309F1ED
:107E40000E94CD9A182F90E0CD970CF01CE3109370
:107E500008080E9483D26B017C01212F30E0A8EE3C
:107E6000B3E00F944C1BC60ED71EE81EF91EC0923D
:107E70000408D0920508E0920608F09207080C94D6
:107E80007B480E94FB6F0C947B4840E060E080914F
:107E9000860B9091870B0E947F730C947B48809196
:107EA00024178E7F809324170C947B48809124178D
:107EB00083FD02C00C947B480E9425CF809124173B
:107EC00083FD02C00C947B486091860B7091870BF8
:107ED000CE014C960E947DE38C01009711F40C9426
:107EE0007B486C8D7D8D19821C8222E0AC01CE0115
:107EF00001960E94A098811102C0F12C14C0CE01FD
:107F000001960E94EBE28823C1F361E0CE01019665
:107F10000E941B92009789F325EEFC0120831C82AE
:107F20000E942A94F82ECE0101960E94A694B801D0
:107F3000FF2089F08FEA98E00E94134E8AE00E94A9
:107F4000E64D1092201710922117109222171092CE
:107F500023170C947B4887E998E00E94134E84E92C
:107F600098E00E94F84D0C947B488091241782FD84
:107F70000E94497A8091241783FD02C00C947B48AB
:107F800060E080E50E94829B182F482F61E080917D
:107F9000860B9091870B0E947F7383E50E94759BEF
:107FA000882381F00E94BD9AAB01BC014093201749
:107FB0005093211760932217709323178BE594E158
:107FC0000E9431910E94337011110C947B480F94E0
:107FD0006C010C947B482091860B3091870B90911B
:107FE000241792609093241740E060E0C9010E943A
:107FF0007F730C947B480E9479FD6C8F7D8F8E8FF0
:108000009F8FBE016F5F7F4FCE014C960E94726BB7
:1080100060E0CE0101960E94D9FF0E942A4EBE0167
:108020006F5F7F4F8DEB98E00E94134E8AE00E94B5
:10803000E64D0C947B4883E50E94759B882311F4E0
:108040000C947B480E94CD9AF82E6DE070E080E59C
:108050000E940CF18C0197FF02C00C947B48E82E23
:1080600060E089E40E94829B81110C94EB4B802F8D
:108070000E944D4D8111B5C40C94EB4B0E9436BC4F
:108080000C947B4880E50E942C9B882311F40C946F
:108090007B488091241782FF02C00C947B480C948B
:1080A000044C0F946C010C947B480E94C8FD0C9406
:1080B0007B480F941C020C947B4860E070E083E5E1
:1080C0000E940CF18E34910531F40F94CE020F947E
:1080D00002000C947B4888E299E00E94F84D609180
:1080E0005709709158098FE199E00E94004F609103
:1080F000590970915A0982E199E00E94004F6091FC
:108100005709709158098091590990915A09681B33
:10811000790B80910D18815021E030E0823010F011
:1081200020E030E0621B730B87E099E00E94004F73
:108130008AE00E94E64D8FEF98E00E94F84D809112
:108140005B0990915C09A0915D09B0915E098C8FEB
:108150009D8FAE8FBF8FBE016F5F7F4FCE014C965C
:108160000E94726BBE016F5F7F4F82EF98E00E94AA
:10817000134E80915F0990916009A0916109B091BF
:1081800062098C8F9D8FAE8FBF8FBE016F5F7F4F57
:10819000CE014C960E94726BBE016F5F7F4F82EEE4
:1081A00098E00E94134E20E030E04AE754E46091EA
:1081B00063097091640980916509909166090F9433
:1081C000A01CAB01BC018AEC98E00E94AB4F8DE68D
:1081D0000E94E64D8AE00E94E64D8DC780913D0DDC
:1081E00083FD89C70E9456D3182F87FD84C783E576
:1081F0000E94759B882309F10E94F59A0F94121D25
:108200007B01212F110F330BF901EE0FFF1FEC5CE7
:10821000F24F718360834091CB0D50E024173507F6
:1082200009F069C7CB010E949199F6E5EF16F104B8
:1082300024F40F941C020F9402000F94340C5BC7BB
:1082400080913D0D83FD57C70E9456D3082F87FDAF
:1082500052C783E50E94759BF82E811107C082E505
:108260000E94759B182F882309F446C00E94F59A36
:108270000F94121D402F002E000C550BFA01EE0F2B
:10828000FF1FEC5CF24F718360832091CB0D30E0D7
:108290004217530709F02FC7CB010E9491990E9402
:1082A000F59A20E030E04AEA52E40F94A21418163E
:1082B00014F40C940F4C0F941C020F940200609164
:1082C0002D0970912E09072E000C880B990B0F9425
:1082D000A9142091290930912A0940912B09509124
:1082E0002C090F94061E181614F40C94134CFF203E
:1082F00011F40C94134C11E00F94340C112309F475
:10830000FAC66F2D802F0E9440A3F5C60E9456D357
:10831000182F87FDF7C680E399E00E94F84D812F62
:108320000E944AA18AE00E94E64DECC66091CB0D06
:1083300080E50E946BF4182F823008F0DCC681E4DF
:108340000E942C9B882341F0E091CB0DF0E0E65C8D
:10835000F24F608170E002C06FEF70E083E50E9431
:108360005ED58F3F910519F010F08FEF90E0BC01C2
:10837000812F0E943AFCBFC66091CB0D80E50E9420
:108380006BF460E070E00E943AFCB5C68EE40E9497
:10839000759B882309F4AFC60E94BD9A6093820B37
:1083A0007093830B8093840B9093850BA4C683E515
:1083B0000E942C9B882331F060E083E50E946BF4DF
:1083C00080933D0D0E942A4E81E499E00E94F84D71
:1083D00080913D0D882369F147E3E42E49E0F42EB6
:1083E00000E010E020E080913D0D90E0A0E0B0E0E2
:1083F000002E04C0B695A795979587950A94D2F755
:1084000080FF0EC0DD24D394D20E222319F08CE21B
:108410000E94E64DF701859194910E94F84D2D2D13
:108420000F5F1F4F32E0E30EF11C05301105D9F646
:10843000FDCC83E399E0F8CC83E50E94759B88230B
:1084400071F00E94CD9A282F30E02D3331051CF4B5
:108450008093020250C68CE3809302024CC60E94B5
:108460002A4E4091020250E060E070E088E499E01A
:108470000E94EF4E8AE00E94E64D3DC680913D0D80
:1084800083FD39C683E50E94759B882309F433C6B2
:108490000E94F59A0F94121DCB010E94AF9A2BC631
:1084A00080913D0D83FD27C683E50E94759B182FA3
:1084B00081110C94184C82E50E94759B81110C94DB
:1084C000184C19C683E50E94759B882309F413C6CE
:1084D0000E94CD9A182F90E0CD970CF01CE31093DA
:1084E0000D080E9483D26B017C01212F30E0A8EEA1
:1084F000B3E00F944C1BC60ED71EE81EF91EC092A7
:108500000908D0920A08E0920B08F0920C08F3C513
:108510000E949BD4F0C5809113088F7D8061809369
:108520001308E9C5809113088F7E80628093130839
:10853000E2C50E949FD9DFC583E50E942C9B88235A
:1085400009F4D9C50E94F59A20E030E04AE754E4E6
:108550000F9408150F94191D60930E0870930F085F
:108560008093100890931108C6C50E9456D387FDCA
:10857000C2C59091871794FD04C09091891797FF09
:108580000AC02DE7C22E23E0D22E3CEEE32E3CE0C3
:10859000F32E10E009C090918A17937091F7682F1D
:1085A00081E00E94F5D9A7C5D6018D916D010E9489
:1085B000759B882309F459C0133009F04FC00E94FD
:1085C000F59A4B015C0120E030E040EA51E40F9461
:1085D000A21487FF3AC0A501940160910C0D70911F
:1085E0000D0D80910E0D90910F0D0F94A01C2B017D
:1085F0003C019B01AC0160911C0D70911D0D80919F
:108600001E0D90911F0D0F94081560931C0D709313
:108610001D0D80931E0D90931F0D6091970C70910E
:10862000980C8091990C90919A0C0F94A714A30127
:1086300092010F9408150F94191D6093970C709375
:10864000980C8093990C90939A0C80920C0D9092B8
:108650000D0DA0920E0DB0920F0D07C00E94F59A5D
:10866000F701648B758B868B978B1F5FF4E0EF0EA1
:10867000F11C143009F098CF0E94257A3CC50E9465
:1086800049EA39C58091860B9091870B009741F09C
:10869000DC012C91222321F060E00E94D9FF2BC540
:1086A0000F94020028C50091860B1091870B94E06F
:1086B000F12C40E0915021F1F8018081282F2B7F8F
:1086C000213421F421812133D9F407C08035C1F44C
:1086D000818180538A3048F013C0813421F0853481
:1086E00021F441E002C0FF24F39498012E5F3F4F34
:1086F00089012F5F3F4FF80180818032C9F3DACFC3
:1087000041110E942A4EFF2021F089E79BE00E9440
:10871000F84DC8010E94C24FEEC40E94AFE0EBC406
:1087200081E080936809809367090E94F7E0E3C4C1
:108730000E9456D3182F87FDDEC484E40E942C9B30
:10874000882309F45BC00E94F59A6B017C0101E06B
:1087500020E030E0A9010F94A214811101C000E0D3
:108760000093760C20E030E0A901C701B6010F9418
:10877000A214882309F442C00E94F59A24E0120250
:10878000F0011124E158F34F608371838283938356
:1087900020E030E0A90160917F0C7091800C809105
:1087A000810C9091820C0F94A21481110CC080E076
:1087B00090E0A0EEBFE380937F0C9093800CA09399
:1087C000810CB093820C20E030E0A9016091830C11
:1087D0007091840C8091850C9091860C0F94A2145A
:1087E00081110CC080E090E0A0EEBFE38093830C89
:1087F0009093840CA093850CB093860C0E943C7DD2
:108800007AC40E9456D387FD76C49DE7E92E93E093
:10881000F92E0CEE1CE0D7018D917D010E942C9B5E
:10882000882359F00E94F59A0F94191DF80160836E
:108830007183828393830E94AE790C5F1F4FFCE0AB
:108840000C3F1F0741F757C40E9456D387FD53C4FE
:10885000BDE7EB2EB3E0FB2E0CEE1CE08CEFC82E38
:108860008CE0D82ED7018D917D010E942C9B88230E
:1088700039F00E94F59AF80164A375A386A397A323
:108880000C5F1F4FC016D10669F735C40E9459F21C
:1088900032C40E94DFF22FC4FDE7CF2EF3E0DF2EBB
:1088A000ABE6EA2EA9E0FA2E10E0D6018D916D011B
:1088B0000E942C9B882351F00E94F59AF701608357
:1088C000718382839383812F0E945D801F5FF4E018
:1088D000EF0EF11C133049F70C945F3A0E9483F1BC
:1088E0000AC483E50E94759B882309F404C40E948E
:1088F000F19A90936D0280936C02FDC30E9456D34F
:10890000F82E87FDF8C383E50E94759B0F2D0F2C71
:10891000000C110B882369F10E94F19AF801EE0F07
:10892000FF1FEB5DFD4F91838083000F111F000F30
:10893000111F98012B5C3D4F7901BC01990F880BE9
:10894000990B0F94A9142AE037ED43E25CE30F94EE
:108950000815F801E958F34F208131814281538194
:108960000F940815D7016D937D938D939C93139766
:10897000C2C30E942A4E85E40E94E64D80E38F0D1B
:108980000E94E64DF801EE0FFF1FEB5DFD4F608189
:1089900071818DE79BE00E94294F85E20E94E64DA0
:1089A0008AE00E94E64DA7C380E50E942C9B8823A5
:1089B00009F4A1C360E070E080E50E940CF1F82E9C
:1089C0006FEF7FEF83E50E940CF18C010196039716
:1089D00008F091C3F7FC8FC38F2D0E944D4D882363
:1089E00039F00E94264E85E89BE00E94F84D83C333
:1089F0000E94497A60E08F2D0E9425D10F3FBFEF82
:108A00001B0731F00130110571F000E010E00DC0DE
:108A10008F2D0E94CDD031E020E0892B09F030E08D
:108A2000032F122F02C001E010E08F2D0E94CDD045
:108A30008017910709F45FC380E00E94E34FF5CFF0
:108A40008AE50E94759B811105C083E50E94759B94
:108A5000882331F10E94F59A20E030E040E050ECAC
:108A60000F94A21487FD1EC70E94F59A20E030E003
:108A700040E050E40F94061E18160CF40EC70E9436
:108A8000F59A2091080D3091090D40910A0D5091F1
:108A90000B0D0F9408150F94121DCB010E947FE45B
:108AA0008091891787FD03C780918A17837009F029
:108AB000FEC60E942A4E40910E0C50910F0C609100
:108AC000100C7091110C8FE99BE00E94AB4F8AE073
:108AD0000E94E64D60917D1370917E1384E99BE0C6
:108AE0000E94294F8AE00E94E64D05C364E071E0D0
:108AF00083E50E945ED58C0168EE73E080E50E94FC
:108B00005ED58938E3E19E0710F088E893E1B8016B
:108B10000E941FFFF0C260E085E40E946BF48111A7
:108B200073C080E50E942C9B882351F00E94F59A27
:108B3000609330097093310980933209909333091F
:108B400089E40E942C9B882381F00E94F59A2CEAEC
:108B500035EC47E25EE30F94081560933409709397
:108B60003509809336099093370984E40E942C9B41
:108B7000882381F00E94F59A2CEA35EC47E25EE307
:108B80000F94A01C609338097093390980933A09B7
:108B900090933B090E942A4E40913009509131092F
:108BA000609132097091330986EC9BE00E94AB4FD3
:108BB0002CEA35EC47E25EE36091340970913509A7
:108BC00080913609909137090F94A01CAB01BC012C
:108BD00082EC9BE00E94AB4F2CEA35EC47E25EE36F
:108BE000609138097091390980913A0990913B0957
:108BF0000F940815AB01BC018EEB9BE00E94AB4FBC
:108C00008AE00E94E64D77C20E94264E8CEA9BE0E5
:108C10000E94F84D70C280E50E942C9B882351F081
:108C20000E94F59A60934709709348098093490917
:108C300090934A0989E40E942C9B882381F00E942A
:108C4000F59A2CEA35EC47E25EE30F940815609341
:108C50004B0970934C0980934D0990934E0984E41D
:108C60000E942C9B882381F00E94F59A2CEA35EC17
:108C700047E25EE30F94A01C60934F097093500984
:108C800080935109909352090E942A4E40914709BE
:108C9000509148096091490970914A0982ED9BE021
:108CA0000E94AB4F2CEA35EC47E25EE360914B0942
:108CB00070914C0980914D0990914E090F94A01C20
:108CC000AB01BC018EEC9BE00E94AB4F2CEA35EC73
:108CD00047E25EE360914F0970915009809151091C
:108CE000909152090F940815AB01BC018AEC9BE0EE
:108CF0000E94AB4F8AE00E94E64DFDC183E50E94D1
:108D00002C9B182F882371F00E94F59A0F94121D46
:108D1000709366026093650221E0672B09F020E002
:108D200020933C0D80E50E942C9B882359F02091D4
:108D3000650230916602232B11F00E94E19A809324
:108D40003C0DD9C11111D7C10E942A4E82EF9BE080
:108D50000E94F84D80913C0D882319F08AED9BE02C
:108D600002C086ED9BE00E94F84D60916502709113
:108D7000660281EE9BE00E94294F8DED9BE00E94F0
:108D8000F84DB9C10E94F965B6C1809187178878FE
:108D900009F093C580918917867009F08EC50E94ED
:108DA0002A4E85E29CE00E94F84D809103020E94C9
:108DB000074E40916E0250916F0260917002709167
:108DC000710285E09CE00E94AB4F8AE00E94E64D74
:108DD00092C10E9487F38FC10E9459CF81118BC12C
:108DE0000FE41CE12CEC3DE03DA32CA3CE01019649
:108DF0001C0154EAC52E5CE1D52E7C01F801659179
:108E0000759185919491ACA1BDA18D909D90AD90EF
:108E1000BD90BDA3ACA3A50194010F94A51B2B018C
:108E20003C01F701608371838283938320E030E00B
:108E300040EA51EC0F94061E87FD0AC020E030E0A6
:108E400040EA51E4C301B2010F94A21418162CF4A5
:108E5000F601849118160CF460C5D7018D909D9091
:108E6000AD90BD907D0120E030E040EA51ECC501BD
:108E7000B4010F94061E87FD5AC520E030E040EA99
:108E800051E4C501B4010F94A21418160CF061C589
:108E90004EC50E9496F02FC10E94C5EB2CC161E027
:108EA00083E50E94829B91E089270E9470ED23C197
:108EB00081E080938E170E94BDAB10928E1788239D
:108EC00009F419C10E942A4E82E79CE00E94F84DE5
:108ED00012C18091241782FF0EC1806480932417F1
:108EE0000AC10E9480D307C10E9456D3082F87FD74
:108EF00002C185E50E942C9B8823B1F1E02E002E53
:108F0000000CFF080E94F59A4B015C0120E030E064
:108F1000A9010F94061E87FF04C0B7FAB094B7F8F2
:108F2000B094C70133E0880F991F3A95E1F79C018F
:108F30002D56384E7901D9018D929D92AD92BC92F9
:108F4000139720E030E04AEF53E4C501B4010F94D9
:108F5000061E18164CF480E090E0AAEFB3E4F70187
:108F600080839183A283B3838CE40E942C9B88230B
:108F700009F4C1C0002E000C110B0E94F59A6B0180
:108F80007C0120E030E0A9010F94061E87FF04C099
:108F9000F7FAF094F7F8F09423E0000F111F2A95E8
:108FA000E1F70D56184ED8011496CD92DD92ED9250
:108FB000FC92179720E030E04AEF53E4C701B60176
:108FC0000F94061E18160CF096C080E090E0AAEFF1
:108FD000B3E4F80184839583A683B7838CC0609142
:108FE000CB0D70E084E50E940CF18C01823028F0FA
:108FF00086EA9CE00E94F84D7EC08BE40E94759B3F
:10900000882349F10E94F59A6B017C0120E030E051
:10901000A9010F94061E87FD19C020E030E040E250
:1090200051E4C701B6010F94A21418167CF00E94F7
:10903000497AF801FF27EE0FFF1FEE0FFF1FED55D6
:10904000F34FC082D182E282F38255C087E89CE070
:109050000E94F84D50C00E942A4E8DE79CE00E946D
:10906000F84D03EA1CE0C12CD12C760180E20E946D
:10907000E64DC701B6010E940D4F8DE30E94E64DFB
:10908000D8016D917D918D919D918D0142E00E945D
:10909000364FBFEFCB1ADB0AEB0AFB0AE2E0CE1633
:1090A000D104E104F10411F40C94163FDFCF81E008
:1090B000809348021092BC1360E083E50E94829B7B
:1090C000811119C00E94766D16C00E943FCF13C057
:1090D00010918B178091CB0D181729F060E083E574
:1090E0000E94829B01C081E0682F812F0E94C1A451
:1090F00002C00E943FCF2296FFAD2297F11102C01D
:109100000E94216D2CAD20931408CF5BDF4F0FB66A
:10911000F894DEBF0FBECDBFDF91CF911F910F91AD
:10912000FF90EF90DF90CF90BF90AF909F908F9087
:109130007F906F905F904F903F902F90089520E028
:1091400030E0A901C701B6010F94A214881F882737
:10915000881F181709F4F3C080E090E0A0E8BFEB87
:1091600088AF99AFAAAFBBAF28A539A54AA55BA523
:1091700068A979A98AA99BA90F94A51B2B013C0179
:109180002CA53DA54EA55FA56CA97DA98EA99FA97B
:109190000F94A51B6CA37DA38EA39FA3A301920193
:1091A000C301B2010F9408154B015C012CA13DA134
:1091B0004EA15FA1CA01B9010F9408159B01AC0132
:1091C000C501B4010F94A61B0F94541E4B015C0102
:1091D00020E030E040E05FE30F94081521966CAF8B
:1091E0007DAF8EAF9FAF2197A7019601C701B60152
:1091F0000F9408156B017C0121962CAD3DAD4EAD51
:109200005FAD2197CA01B9010F9408159B01AC010C
:10921000C701B6010F94A51B0F94541E6B017C016E
:109220008CA19DA1AEA1BFA1B0588CA39DA3AEA35C
:10923000BFA32DEB37E346E855EBC501B4010F940E
:10924000061E87FD0AC02DEB37E346E855E3C5014E
:10925000B4010F94A21418165CF4A501940160E007
:1092600070E080E89FE30F94A01C4B015C0103C0F9
:10927000812C912C5401A5019401C301B2010F94DA
:10928000081528AD39AD4AAD5BAD0F940815A7019F
:1092900096010F9408152B013C0128A939A94AA968
:1092A0005BA968A579A58AA59BA50F94A61B20E0BC
:1092B00030E040E05FE30F9408159B01AC01C3016F
:1092C000B2010F94A61B28A539A54AA55BA50F944A
:1092D000A51B69837A838B839C83A50194016CA170
:1092E0007DA18EA19FA10F94081528AD39AD4AAD7F
:1092F0005BAD0F940815A70196010F9408156B013B
:109300007C012CA93DA94EA95FA96CA57DA58EA5C0
:109310009FA50F94A61B20E030E040E05FE30F9490
:1093200008159B01AC01C701B6010F94A61B2CA523
:109330003DA54EA55FA50F94A51B0C94373880E082
:1093400090E0A0E8BFE30CCF412FBE016F5F7F4FDD
:109350008AEA9DE00E9465E60E9483D260937313BF
:10936000709374138093751390937613C4CE0E94F8
:10937000264E83ED96E00E94F84DBDCE0E94497ABC
:109380009091E40D9CAB80E00E94DE4C80916102E4
:1093900090916202A0916302B091640280931708D9
:1093A00090931808A0931908B0931A0880916C0242
:1093B00090916D02909316088093150884E690E0D2
:1093C00090936D0280936C0281E0809368090E9403
:1093D000F7E088E50E942C9B182F89E50E942C9BC2
:1093E000082F8AE50E942C9B1013ACC1181711F0AE
:1093F000012FA8C101E011E091E09CA780E1ECEC15
:10940000FDE0AAEABDE001900D928A95E1F782E5C0
:109410000E94759B882361F00E94F59A6B017C0184
:1094200020E030E0A9010F94A214882369F106C05E
:10943000C12CD12C80E8E82E80E4F82E111103C055
:10944000002309F4FCC0C092B20DD092B30DE0929B
:10945000B40DF092B50DA70196016091D40D7091F5
:10946000D50D8091D60D9091D70D0F94A21487FF42
:109470000BC019821A821B821C82BE016F5F7F4F54
:1094800082EB9DE00E9453DF112309F4D3C0002337
:1094900009F4CDC01092CC0D1092CD0D1092CE0DCE
:1094A0001092CF0D1092D00D1092D10D1092D20DBE
:1094B0001092D30D0E9498DFE4EAFCE1A491A8AFDA
:1094C000E8E9FCE1C590D590E590F490ECE9FCE189
:1094D00085909590A590B490A5019401C701B6011F
:1094E0000F94061E18162CF4A7019601C501B401AD
:1094F00004C0A5019401C701B6010F94A01C2B0163
:109500003C01EFE5FCE185919591A591B4918CA387
:109510009DA3AEA3BFA3EBE5FCE185919591A59139
:10952000B49188A799A7AAA7BBA79C01AD016CA17C
:109530007DA18EA19FA10F94061E181634F428A4B5
:1095400039A49AA598AB1BA505C02CA03DA0AEA13F
:10955000A8AB1FA1A3019201C301B2010F9408158A
:1095600020E030E040E85FE30F94A61B0F94541E08
:10957000910148A9512F0F94081568A379A38AA3D4
:109580009BA3E5EAFCE1149120E030E040EC5FE3CE
:10959000C501B4010F9408154B015C01612F110F37
:1095A000770B880B990B0F94A9149B01AC01C50193
:1095B000B4010F94081569837A838B839C8320E020
:1095C00030E040EC5FE3C701B6010F9408156B0172
:1095D0007C01B8AD6B2FBB0F770B880B990B0F94E9
:1095E000A9149B01AC01C701B6010F9408156C8F3B
:1095F0007D8F8E8F9F8FAE01405E5F4FBE016F5F8C
:109600007F4FCE014C960E9431DF0F944D0F109288
:10961000CC0D1092CD0D1092CE0D1092CF0D109258
:10962000D00D1092D10D1092D20D1092D30D80E07A
:109630000F94640C002319F081E00F94640CECA5E6
:10964000EE2309F45BC080917B138370833051F06B
:1096500060E084E297E00E947EFF0E942A4E85E14E
:1096600097E04AC00E9498DF8091D40D9091D50D6B
:10967000A091D60DB091D70D40E050E068E472E4BF
:109680004093AA0D5093AB0D6093AC0D7093AD0D4C
:1096900040E050E06CE872E44093AE0D5093AF0DA3
:1096A0006093B00D7093B10D8093B20D9093B30D94
:1096B000A093B40DB093B50D8AEA9DE00E9439F6EF
:1096C000882389F019821A821B821C82AE014F5FA7
:1096D0005F4F6EEA7DE08AEA9DE00E9431DF82E022
:1096E0000F94640C0BC060E084E097E00E947EFF62
:1096F0000E942A4E82EF96E00E94F84D0E9498DF69
:1097000080916709809368098CA90E94DE4C809142
:10971000170890911808A0911908B0911A08809321
:10972000610290936202A0936302B09364028091FD
:1097300015089091160890936D0280936C020E9418
:109740009ADFD9CC8CA75ACEB1100C94F13D0C9471
:10975000EA3D80E00E94E34F0C941D3E88E50E94A4
:109760002C9B81115F9889E50E942C9B81118A981E
:109770008AE50E942C9B882329F080910801817042
:109780008093060185E40E942C9B882309F4B3CCC6
:1097900012984798B0CC60E08EE398E00E947EFF7C
:1097A0005F988A98809108018170809306011298D1
:1097B0004798A1CC0E94BD9AAB01BC0140932017F1
:1097C0005093211760932217709323178BE594E130
:1097D0000E94319190CC61E0802F0E9425D16F2DA5
:1097E000802F0E94F6D06F2D70E0802F0E9461D1F3
:1097F000A7E0EA1203C0F0923B0D7DCCB9E0EB127A
:109800007ACCF0923A0D77CC0E94CD9A90E08536D2
:10981000910514F084E690E08093FA176CCC0F94D5
:109820006C010C945F41802F0E9420A10C947B411D
:109830000E94F59A0F94121DCB010E94AF9A0E94CC
:10984000F59A20E030E040EA50E40F94061E181626
:1098500014F40F946C016091440970914509072E2E
:10986000000C880B990B0F94A9142091400930919A
:10987000410940914209509143090F94061E181660
:109880001CF48EE599E002C08FE499E060E00E944C
:109890007EFF812F0E94C1A12ECC60E070E080E0AD
:1098A00090E4EFC860E070E080E090ECEAC882E508
:1098B0000E942C9B8111FDC81ECC88E40E942C9B29
:1098C000882321F00E94E19A8093120882E50E9489
:1098D0002C9B082F83E50E942C9B182F011102C09E
:1098E000882351F0109223090E94724D112321F018
:1098F0000E94E19A8093030284E40E942C9B8823B7
:1099000009F4F9CB0E94F59A60936E0270936F028E
:109910008093700290937102EECBB7FAB094B7F8CF
:10992000B094F70180829182A282B38296CA0E948B
:10993000264E84E59CE00E94F84D61E086E49CE0C0
:109940000E947EFF68E270E088EC90E00E941FFFBA
:10995000D2CB0C5F1F4FFFEFCF1ADF0A2CE10B3584
:10996000120709F04BCA4BE6E42E49E0F42E10E052
:10997000F10181919191A191B1911F01F701819321
:109980009193A193B1937F01812F0E945D801F5F0E
:10999000133071F70E949ADF60E086E39CE00E943A
:1099A0007EFF63E972E084E690E00E941FFF6AEBAD
:1099B00072E084E690E00E941FFF9DCB9091E40D41
:1099C0009817B1F00E94497A8091E40D882339F00C
:1099D0008CEC9DE00E94A77C1092E40D07C081E012
:1099E0008093E40D8CEC9DE00E94767C0C9498DFD3
:1099F0000895EF92FF921F93CF93DF9382E1E82EB9
:109A00008CE0F82E15E0C0E0D0E020E030E0A901C5
:109A1000F701EC0FFD1F60817181828193810F94AA
:109A2000A21481110CC02496C431D10571F71150D4
:109A300084E1E80EF11C1111E6CF80E001C081E065
:109A4000DF91CF911F91FF90EF900895CF92DF9219
:109A5000EF92FF926B017C0183E3C816D104E1040D
:109A6000F10470F082E3C81AD108E108F10862E35A
:109A700070E080E090E00E9449D20E9426F8ECCF8E
:109A8000C701B6010E9449D2FF90EF90DF90CF90BE
:109A90000C9426F8129A479A0895FF920F931F93F9
:109AA000CF93DF931F92CDB7DEB7F82E08ED1CE001
:109AB00041E050E0B801CE0101960F94DC1389819A
:109AC0008F1102C081E007C00F5F1F4F8CE0043F81
:109AD000180771F780E00F90DF91CF911F910F91E0
:109AE000FF90089580916E0290916F02A091700294
:109AF000B0917102EBECF8E080839183A283B38391
:109B000084839583A683B783089580912E0881115D
:109B100007C00E9496F0882319F081E080932E08F8
:109B200008959091241793FB882780F993FF06C02E
:109B300081E090915E14911101C080E0089560E091
:109B400070E080E00E943AFC60E070E081E00C94FC
:109B50003AFC8F929F92AF92BF92CF92DF92EF9298
:109B6000FF920F93CF93DF931F92CDB7DEB75C01C7
:109B70006B017A014901F501808191810F94D21A1C
:109B80008983002311F0F6018083BE016F5F7F4F50
:109B9000C4010E94ADE1F50180819181019691831C
:109BA0008083FFEFCF1ADF0A81E0E81AF10819F786
:109BB00080E00F90DF91CF910F91FF90EF90DF90B9
:109BC000CF90BF90AF909F908F9008959091C000DC
:109BD00095FFFCCF8093C6000895CF93C82FCC2368
:109BE00029F080E20E94E64DC150F9CFCF9108954F
:109BF000CF93DF93FC018491EF012196882321F01C
:109C00000E94E64DFE01F7CFDF91CF9108958111BB
:109C100003C08BE69EE202C08FE69EE20E94F84DF2
:109C20008AE00C94E64D0F931F93CF93DF938B0143
:109C30000E94F84DE8018991882319F00E94E64DB1
:109C4000FACFDF91CF911F910F91089583E19FE0AB
:109C50000C94F84D8DE09FE00C94F84D7F928F921C
:109C60009F92AF92BF92CF92DF92EF92FF920F93AB
:109C70001F93CF93DF931F92CDB7DEB77C015901BD
:109C80008B016B01C40ED51E0C151D0559F1F70192
:109C900080809180F80171908F017982C4010F94C6
:109CA000D21A781691F0672DC4010F94DA1AC40104
:109CB0000F94D21A9981891741F00E942A4E8EEB97
:109CC0009CE00E94F84D81E00EC0BE016F5F7F4FA7
:109CD000C5010E94ADE1F7018081918101969183D8
:109CE0008083D2CF80E00F90DF91CF911F910F91B1
:109CF000FF90EF90DF90CF90BF90AF909F908F90AC
:109D00007F9008958F929F92AF92BF92EF92FF92B1
:109D10000F931F93CF93DF93CDB7DEB7A0970FB606
:109D2000F894DEBF0FBECDBF6115710581059105A9
:109D300091F100E0842E912CA12CB12C102FEE2457
:109D4000E394F12CEC0EFD1EE00EF11C07FDFA94DD
:109D5000A50194010F94F81AF7016083B901CA01B3
:109D60000F5F611571058105910541F71F3F31F1C5
:109D7000E1E0F0E0EC0FFD1FE10FF11D17FDFA959A
:109D800080818A3010F097E301C090E3890F0E9430
:109D9000E64D1150EBCF80E3A0960FB6F894DEBFEE
:109DA0000FBECDBFDF91CF911F910F91FF90EF902C
:109DB000BF90AF909F908F900C94E64DA0960FB6F9
:109DC000F894DEBF0FBECDBFDF91CF911F910F91F1
:109DD000FF90EF90BF90AF909F908F900895CF929B
:109DE000DF92EF92FF926A017B010E94F84D4AE0F8
:109DF000C701B601FF90EF90DF90CF900C94824E98
:109E0000CF93DF93EB010E94F84DBE0180E090E01C
:109E10004AE0DF91CF910C94824ECF92DF92EF9285
:109E2000FF926B017C0197FF0BC08DE20E94E64D13
:109E3000F094E094D094C094C11CD11CE11CF11C9E
:109E40004AE0C701B601FF90EF90DF90CF900C94ED
:109E5000824ECF93DF93EB010E94F84DBE01DD0FE0
:109E6000880B990BDF91CF910C940D4F8F929F929D
:109E7000AF92BF92CF92DF92EF92FF92CF936B019E
:109E80007C01B42E20E030E0A9010F94A21487FFDA
:109E900007C08DE20E94E64DF7FAF094F7F8F094CF
:109EA000C0E060E070E080E09FE3CB1541F02DEC76
:109EB0003CEC4CEC5DE30F940815CF5FF6CF9B01B3
:109EC000AC01C701B6010F94A61B6B017C010F9476
:109ED000191D4B015C014AE00E94824ECC2389F19E
:109EE000C501B4010F94A7149B01AC01C701B601D1
:109EF0000F94A51B6B017C018EE20E94E64D20E0D1
:109F000030E040E251E4C701B6010F9408154B015F
:109F10005C010F94121D6B01770FEE08FF08C7015B
:109F2000B6010E940D4FC701B6010F94A9149B0101
:109F3000AC01C501B4010F94A51B6B017C01C1509C
:109F4000F1F6CF91FF90EF90DF90CF90BF90AF9060
:109F50009F908F900895CF92DF92EF92FF926A01C7
:109F60007B010E94F84D42E0C701B601FF90EF90DF
:109F7000DF90CF900C94364F8DE00E94E64D8AE042
:109F80000C94E64DCF93DF93EC018991882319F06F
:109F90000E94E64DFACFDF91CF910C94BC4F809197
:109FA000FE0A9091FF0A981759F0E92FF0E0E2506D
:109FB000F54F82819F5F9F779093FF0A90E008950D
:109FC0008FEF9FEF08952F923F924F925F926F9283
:109FD0007F928F929F92AF92BF92CF92DF92EF9239
:109FE000FF920F931F93CF93DF93CDB7DEB72897E0
:109FF0000FB6F894DEBF0FBECDBFE82E0E94B91B8E
:10A000000E9483D24B015C0180910202882359F1A6
:10A0100080911408882339F140912F08509130081D
:10A02000609131087091320895018401041B150B71
:10A03000260B370B37FD2AC0833079F03CF4813092
:10A0400094F00E942A4E83E29DE00BC0843059F4C4
:10A050000E942A4E84EF9CE004C00E942A4E8CE0AD
:10A060009DE00E94F84D2091020230E0A8EEB3E09E
:10A070000F944C1B860E971EA81EB91E80922F08A7
:10A0800090923008A0923108B09232088091030279
:10A09000882309F4BAC0809123098111B6C0809148
:10A0A0000D18813021F08091241782FF38C6F89472
:10A0B0002091CB0D8CB18295817030910301932F4B
:10A0C000917030FD92E0892B90E0A0E0B0E0022E8C
:10A0D00004C0B695A795979587950A94D2F714E092
:10A0E000219F9001112480FD0FC080916E029091FC
:10A0F0006F02A0917002B0917102F901E553F74F20
:10A1000080839183A283B383F901E553F74F608184
:10A11000718182819381789420E030E0A9010F94CD
:10A12000A21487FF72C011E0109323098091880B5D
:10A13000811169C08DE496E00E94C24F84E0809353
:10A14000071882E08093E40781E09AE590938115F7
:10A15000809380158EE490E0909383158093821510
:10A1600087E08093741582E88093771584E890E007
:10A17000A0E0B0E08093781590937915A0937A15BC
:10A18000B0937B150E9407E10091CB0D005D109309
:10A19000BD0C0E94F19B40E064E67DE087EB91E21C
:10A1A0000E94FD9B802F0E94E64D8AE00E94E64DB2
:10A1B0000E94E59B8091120860E0182719F08FE853
:10A1C00090E20DC082E59DE00E94CD9B802F0E9411
:10A1D000E64D8AE00E94E64D60E085E39DE00E9446
:10A1E000CD9B80E49DE00E94F84D802F0E94E64DBB
:10A1F0008AE00E94E64D112331F08BE39DE09093BD
:10A200007909809378090E94497A8091FB0A843009
:10A2100008F07FC20E9483D24B015C018091FB0A4F
:10A2200081111DC08091FE0A9091FF0A891B8F77D2
:10A23000B1F48091980890919908A0919A08B091F2
:10A240009B08A5019401281B390B4A0B5B0BDA0113
:10A25000C901885E9340A109B109B7FF65C560E6F1
:10A26000F62E8091FB0A843008F036C18091FE0AF8
:10A270009091FF0A891B8F7709F42EC10E94CF4F5E
:10A28000AC0197FDEECF2091800B3091810B8A308D
:10A2900019F08D3009F0E8C01092970821153105AA
:10A2A00019F40E9426F8DDCFF901E95CF74F10821E
:10A2B0001092810B1092800B07E318E0F801819156
:10A2C000803211F48F01FACF8E3409F07AC0011573
:10A2D000110509F476C06CE97EE0C8010F942014E2
:10A2E0006C01892B41F06EE470E0C80104960F9474
:10A2F000F91E009709F4C8014AE050E060E070E000
:10A3000001960F94981160933308709334088093EA
:10A310003508909336084090820B5090830B6090E4
:10A32000840B7090850B3FEF431A530A630A730A3C
:10A33000641575058605970531F0CD2821F460E098
:10A3400089E69EE0C7C06AE270E0C8010F94281F4A
:10A350009C01009709F1982F901BD12C992339F07B
:10A360009150F801E90FF11D8081D826F7CF4AE01E
:10A3700050E060E070E0C90101960F9498114D2CF7
:10A38000512C612C712C641575058605970541F0DB
:10A3900060E08AE49EE09EC060E080E29EE09AC0B9
:10A3A0008091330890913408A0913508B091360817
:10A3B0008093820B9093830BA093840BB093850BB7
:10A3C00012C08091241780FF0EC063E478E1C801B9
:10A3D0000F942014009709F47AC0FC018381805304
:10A3E0008A3008F474C08091480281111CC067E46F
:10A3F00070E0C8010F94F91E0097A9F04AE050E000
:10A4000060E070E001960F94981164307105810549
:10A41000910548F48FE79DE00E94F84D60E085E7E4
:10A420009DE00E947EFF8092980890929908A092E9
:10A430009A08B0929B08809137088B3309F411CFAA
:10A440008091FB0A843008F00CCF80917709F89E48
:10A45000C001112467E378E08658964F0F94041FDB
:10A4600081E00E94B6E4FDCE2F3531050CF0F9CE27
:10A470008C35C1F40E94CF4F97FDF3CE2091970801
:10A480002111EFCE2091800B3091810BA9014F5FFC
:10A490005F4F5093810B4093800BF901E95CF74FBC
:10A4A0008083DFCE8B3321F481E080939708D9CE6F
:10A4B000809197088111D5CEC90101969093810BA7
:10A4C0008093800BF901E95CF74F4083CACE60E0CE
:10A4D00086EF9DE00E94926D8091241782FF19C142
:10A4E0008091FB0A811102C010929D08DD24D39453
:10A4F00040912017509121176091221770912317D6
:10A5000080911C1790911D17A0911E17B0911F17D5
:10A51000481759076A077B0708F4D12C00E010E0C0
:10A52000CC24C39430E6B32E44E6A42E59E6952EEF
:10A530008091FB0A843008F0ECC0D110EAC0809111
:10A540009D088111E6C08091631490916414A091DC
:10A550006514B09166148093201790932117A093EF
:10A560002217B093231741E050E0BE016F5F7F4F89
:10A570008BE594E10E941695019719F4898190E08A
:10A5800002C08FEF9FEFF82E4090201750902117B8
:10A59000609022177090231740911C1750911D173F
:10A5A00060911E1770911F17DD24D3944416550631
:10A5B0006606770608F4D12C44165506660677061B
:10A5C000B0F4019609F461C02AE0F21609F46EC0F5
:10A5D0003DE0F31609F46AC043E2F41619F05AE3B9
:10A5E000F5127CC080919C08811178C054C00E94F3
:10A5F000497A8BE594E10E949D9480911B178823F2
:10A6000039F1815080931B17989EC001112441E0BD
:10A6100061E08357944F0E947F73E0911B1764E0C1
:10A62000E69FF0011124E757F44F40815181628188
:10A6300073814093201750932117609322177093D2
:10A6400023178BE594E10E9431910E94337016C06C
:10A650000E9422700E94F97B0F941C020E9479FDD7
:10A660006D3371058105910518F487EA9EE002C0FB
:10A670008CEA9EE00E94BB6DA092FA17809124178D
:10A6800082FD0DC08FEB9EE004C00E94264E80EB41
:10A690009EE00E94F84D73E2F71208C005C053E235
:10A6A000F5124FC300E010E0C0929D0810929C0884
:10A6B0000115110519F40E9426F80DC08091770943
:10A6C000B89E000D111D1124F801E658F64F1082B6
:10A6D00080E00E94B6E400E010E02ACF0F351105BB
:10A6E00008F026CF8BE3F81203C0C0929C0820CF5D
:10A6F00080919C0881111CCF80917709F801B89E48
:10A70000E00DF11D1124E658F64FF0820F5F1F4F48
:10A710000FCF0E9483D24B015C0140910E085091F3
:10A720000F086091100870911108411551056105DD
:10A73000710529F18091731390917413A091751391
:10A74000B0917613840F951FA61FB71F9501840142
:10A75000081B190B2A0B3B0B37FD11C00E94264E1C
:10A760006091BD0D7091BE0D83ED9EE00E94134E71
:10A770008AE00E94E64D80E090E00E9416E240915F
:10A780006702509168026091690270916A024115F6
:10A7900051056105710509F44EC09091D214809164
:10A7A000D314981759F00E9483D260937313709357
:10A7B000741380937513909376133DC08091880B2A
:10A7C000811137C0E11035C08091731390917413DB
:10A7D000A0917513B0917613840F951FA61FB71F14
:10A7E000A5019401281B390B4A0B5B0B57FD21C0B7
:10A7F0008091AE0881111FC081E08093AE085F9AFE
:10A8000080917B138E7F80937B138A9A80917B1338
:10A810008D7F80937B138091080180958170809358
:10A82000060180917B138B7F80937B130E944A4D9E
:10A8300002C01092AE088091AA089091AB08A09136
:10A84000AC08B091AD08B501A401481B590B6A0BC7
:10A850007B0B77FDAAC12091D2149091D3148091E3
:10A8600041021091420229130EC060913A0D869F59
:10A87000B0011124660F672F661F770B7195062FA5
:10A8800080913B0D17C02091D31454E6259F900171
:10A8900011242E5E374EF901EE59FF4F6081869FDD
:10A8A000B0011124660F672F661F770B7195062F75
:10A8B00031968081819FB0011124660F672F661F3A
:10A8C000770B7195162F002331F10E9483D2C0902F
:10A8D000A208D090A308E090A408F090A508DC019D
:10A8E000CB01C114D104E104F10469F48C599F4FE8
:10A8F000AF4FBF4F8093A2089093A308A093A408E2
:10A90000B093A50806C08C199D09AE09BF09B7FF11
:10A910000AC00FEF08C01092A2081092A30810926C
:10A92000A4081092A508602F70E089E00E9461D110
:10A93000112331F10E9483D2C090A608D090A708BD
:10A94000E090A808F090A908DC01CB01C114D10463
:10A95000E104F10469F48C599F4FAF4FBF4F8093CE
:10A96000A6089093A708A093A808B093A90806C0CA
:10A970008C199D09AE09BF09B7FF0AC01FEF08C0B7
:10A980001092A6081092A7081092A8081092A90881
:10A99000612F70E087E00E9461D18091E70C8823ED
:10A9A00009F4F6C0E0902D02F0902E0200912F02E3
:10A9B0001091300260912D0970912E096E5F7F4FCA
:10A9C000072E000C880B990B0F94A9149701A8016E
:10A9D0000F94A21487FDDCC03090D314212C1A826E
:10A9E0001B821C828091D214831509F467C0832DC9
:10A9F00090E064E6689FF001699FF00D1124EE5E1F
:10AA0000F74E458956896789708D452B462B472B14
:10AA100089F4418D528D638D748D452B462B472BC8
:10AA200049F4458D568D678D70A1452B462B472BDC
:10AA300009F43FC074E6789F9001799F300D11248E
:10AA4000C9018E5E974E6C01FC0161817281838128
:10AA500094810F94541E2B013C01F60161A172A157
:10AA600083A194A10F94A7146D837E838F8398870D
:10AA7000F60165A176A187A190A50F94A7149B016B
:10AA8000AC016D817E818F8198850F94A01CA301FC
:10AA900092010F9408153B016C01222D3A814B81E4
:10AAA0005C810F94061E181624F4262C7A82CB8221
:10AAB000DC8281E0830D8F70382E94CF209131029B
:10AAC000309132024091330250913402622D7A81EA
:10AAD0008B819C810F9408159701A8010F94A61BE8
:10AAE0003B016C012090290230902A0240902B02F9
:10AAF00050902C029B01AC01B701C8010F94061EB7
:10AB000018166CF09101A201B301C6010F94061E44
:10AB100018161CF47101820102C073018601409075
:10AB20009E0850909F086090A0087090A10897011F
:10AB3000A801C301B2010F94061E1816C4F420E048
:10AB400037ED43EA5CE3B701C8010F9408156B01C8
:10AB50007C0128E431EE4AE75FE3C301B2010F94C0
:10AB60000815A70196010F94A61B7B018C01C70154
:10AB7000D80180939E0890939F08A093A008B0935B
:10AB8000A108B701C8010F94121DCB010E94919931
:10AB9000F4E68F0E911CA11CB11C8092AA08909221
:10ABA000AB08A092AC08B092AD080E9426F8809144
:10ABB0000D18813009F06EC00E9483D26B017C01B8
:10ABC0008091B3089091B408A091B508B091B608EF
:10ABD00097018601081B190B2A0B3B0B37FD3AC066
:10ABE00080900E1890900F18A0901018B090111827
:10ABF0000E9479FD60930E1870930F1880931018BF
:10AC00009093111800915B0910915C0920915D09E6
:10AC100030915E09081919092A093B09DC01CB01A9
:10AC2000800F911FA21FB31F80935B0990935C0953
:10AC3000A0935D09B0935E09D701C601805F984D6E
:10AC4000AF4FBF4F8093B3089093B408A093B5085B
:10AC5000B093B6088091AF089091B008A091B10868
:10AC6000B091B208A7019601281B390B4A0B5B0B68
:10AC700057FD10C030E8C30E3EEED31EE11CF11CA0
:10AC8000C092AF08D092B008E092B108F092B2083A
:10AC90000F94F6010E9497FE80910D08882391F091
:10ACA0000E9483D20091090810910A0820910B0894
:10ACB00030910C08DC01CB01801B910BA20BB30B74
:10ACC000B7FF42C00E9483D26B017C01209108082B
:10ACD000222309F458C08091040890910508A0919E
:10ACE0000608B0910708B701A601481B590B6A0B6B
:10ACF0007B0B77FD48C030E0A8EEB3E00F944C1B0F
:10AD0000C60ED71EE81EF91EC0920408D092050890
:10AD1000E0920608F09207080E94FB6F34C0809111
:10AD2000880B8111C4C971CA81EA9EE00E94F84D66
:10AD30008092980890929908A0929A08B0929B08E5
:10AD40008ECA10929C08B7CC0E9483D26B017C0102
:10AD500020910D0830E0A8EEB3E00F944C1BC60E16
:10AD6000D71EE81EF91EC0920908D0920A08E09288
:10AD70000B08F0920C088091CB0D0E944AA18AE04A
:10AD80000E94E64D9FCF28960FB6F894DEBF0FBE07
:10AD9000CDBFDF91CF911F910F91FF90EF90DF908A
:10ADA000CF90BF90AF909F908F907F906F905F906B
:10ADB0004F903F902F9008951F920F920FB60F92D1
:10ADC00011240F900FBE0F901F9018951F920F9295
:10ADD0000FB60F9211240BB60F920F931F932F9360
:10ADE0003F934F935F936F937F938F939F93AF9313
:10ADF000BF93CF93DF93EF93FF930091FF0AD0911E
:10AE0000FE0A11E01D0F1F77C091C60090912D081A
:10AE1000492F092E000C550B660B770B413151055C
:10AE200008F064C0FA018827ED56FF4F8F4F0D944C
:10AE3000911BCD3449F0CE34B9F481E006C0CA3359
:10AE400038F0CD3409F043C082E080932D0875C0FE
:10AE5000C03308F072C0C03209F46FC0CD32B9F50A
:10AE60006CC0C13351F018F4C03289F566C0C433E8
:10AE700031F0C83361F58BE0E8CF83E0E6CF88E0BE
:10AE8000E4CFC03321F0C13311F586E0DECF84E09A
:10AE9000DCCFC833E1F485E0D8CFC233C1F487E01A
:10AEA000D4CFC133A1F489E0D0CFC03381F48AE09C
:10AEB000CCCFC73361F48CE0C8CFC63341F48DE00A
:10AEC000C4CFC032D1F1C33511F48EE0BECF80E1E2
:10AED000BCCF80ED8C0F8A3080F59FE090932D08D9
:10AEE00080932C082AC0CA3041F525C0CA3029F504
:10AEF0008091E2158823F9F0973089F03CF4953081
:10AF0000D1F4109220021092F91715C09A3059F01E
:10AF10009F3089F480912C080E94299C0CC081E00C
:10AF20008093C41708C00E944F7C0E94497A0E94F7
:10AF3000DDCE0E9498DF10922D08011731F0ED2F21
:10AF4000F0E0E250F54FC283D12FD093FE0AFF917B
:10AF5000EF91DF91CF91BF91AF919F918F917F91B1
:10AF60006F915F914F913F912F911F910F910F9092
:10AF70000BBE0F900FBE0F901F9018958EBD0DB495
:10AF800007FEFDCF08958FEF8EBD0DB407FEFDCFF8
:10AF90008EB50895909164009B7F90936400982FE4
:10AFA000906A96959CBD80FD03C091E0863009F4BF
:10AFB00090E09DBD08952F923F924F925F926F92C5
:10AFC0007F928F929F92AF92BF92CF92DF92EF9239
:10AFD000FF920F931F93CF93DF93CDB7DEB76297A6
:10AFE0000FB6F894DEBF0FBECDBF8FEF9FEF9093EB
:10AFF0008900809388002AE02A8B212C312C7894B8
:10B0000080911F0990912009A0912109B0912209F6
:10B01000892B8A2B8B2B09F0D7C18091A717882306
:10B02000E1F01092A7178091A5179091A617892B90
:10B0300009F4CAC11092D7081092A6171092A5174A
:10B040009091D2148091D314981709F4BDC18091C6
:10B05000D3148F5F8F708093D3148091A517909134
:10B06000A617892B09F4B0C140911B0950911C0906
:10B0700060911D0970911E0980911709909118091E
:10B08000A0911909B0911A0900910E0910E020E071
:10B0900030E0841B950BA60BB70B081719072A077E
:10B0A0003B0710F4D901C801E82F840F951FA61F94
:10B0B000B71F80931B0990931C09A0931D09B0939F
:10B0C0001E092091840030918500225E3F4F4091FF
:10B0D000E3085091E4086091E5087091E6088091DA
:10B0E000F3089091F408A091F508B091F608840F48
:10B0F000951FA61FB71F8093F3089093F408A093A1
:10B10000F508B093F608B7FD1CC0889A8091B7087F
:10B11000082E000C990BAA0BBB0B4091B417509151
:10B12000B5176091B6177091B717840F951FA61FBA
:10B13000B71F8093B4179093B517A093B617B09329
:10B14000B7174091E7085091E8086091E9087091BD
:10B15000EA088091F7089091F808A091F908B09159
:10B16000FA08840F951FA61FB71F8093F7089093C6
:10B17000F808A093F908B093FA08B7FD1CC08E9A9E
:10B180008091B808082E000C990BAA0BBB0B4091BC
:10B19000B8175091B9176091BA177091BB17840F07
:10B1A000951FA61FB71F8093B8179093B917A09348
:10B1B000BA17B093BB174091EB085091EC0860911F
:10B1C000ED087091EE088091FB089091FC08A09129
:10B1D000FD08B091FE08840F951FA61FB71F80932E
:10B1E000FB089093FC08A093FD08B093FE08B7FD00
:10B1F00021C080910B018095887080930901809116
:10B20000B908082E000C990BAA0BBB0B4091BC1778
:10B210005091BD176091BE177091BF17840F951F95
:10B22000A61FB71F8093BC179093BD17A093BE179E
:10B23000B093BF174091FF08509100096091010938
:10B24000709102098091EF089091F008A091F108A7
:10B25000B091F208840F951FA61FB71F8093FF08B7
:10B2600090930009A0930109B0930209B7FD3AC079
:10B270004091BA08042E000C550B660B770BC0905A
:10B28000C017D090C117E090C217F090C3174C0DB3
:10B290005D1D6E1D7F1D4093C0175093C1176093B5
:10B2A000C2177093C3174091DF085091E008609176
:10B2B000E1087091E208841B950BA60BB70B8093F5
:10B2C000FF0890930009A0930109B093020990919F
:10B2D000690980910C0993FF02C0815001C08F5F02
:10B2E00080930C09809184009091850082179307C8
:10B2F000C8F38091F3089091F408A091F508B091FB
:10B30000F608B7FD15C04091DF085091E008609144
:10B31000E1087091E208841B950BA60BB70B809394
:10B32000F3089093F408A093F508B093F608889872
:10B330008091F7089091F808A091F908B091FA0867
:10B34000B7FD15C04091DF085091E0086091E10819
:10B350007091E208841B950BA60BB70B8093F7083E
:10B360009093F808A093F908B093FA088E9880910A
:10B37000FB089091FC08A091FD08B091FE08B7FD74
:10B3800019C04091DF085091E0086091E108709188
:10B39000E208841B950BA60BB70B8093FB089093D8
:10B3A000FC08A093FD08B093FE0880910B01887003
:10B3B00080930901E15041F08091840090918500D3
:10B3C00082179307C8F381CE80910D0290910E02EF
:10B3D000A0910F02B0911002892B8A2B8B2B09F0C0
:10B3E000ADC080910D09882309F453C080901B09DA
:10B3F00090901C09A0901D09B0901E09C0900809EA
:10B40000D0900909E0900A09F0900B0940910C09CD
:10B41000C814D904EA04FB0480F48091DC089091FC
:10B42000DD082091DA083091DB082817390728F465
:10B43000415040930C09019714C08C149D04AE0434
:10B44000BF04E0F48091DC089091DD082091D808D9
:10B450003091D9088217930788F44F5F40930C0905
:10B4600001969093DD088093DC0840910902509189
:10B470000A0260910B0270910C020EC08FEF9FEFD9
:10B48000DC018093090290930A02A0930B02B0930F
:10B490000C024FEF5FEFBA01000000000000909136
:10B4A0000C098091DE0897FD06C0811102C0169A32
:10B4B00007C0439805C0811102C0169801C0439A85
:10B4C00000000000000080918400909185004E965D
:10B4D00020910C09222351F12091DE08211102C094
:10B4E000149A01C0419A2091840030918500281758
:10B4F0003907C8F320910C0927FF02C02F5F01C054
:10B50000215020930C092091DE08211102C01498CB
:10B5100001C0419820910C092223D1F2209184008E
:10B520003091850028173907C8F3D1CF40930D0219
:10B5300050930E0260930F027093100280911F09C6
:10B5400090912009A0912109B0912209892B8A2B81
:10B550008B2B11F00C945861A091A517B091A617F0
:10B56000109711F40C946F6380901B0990901C0944
:10B57000A0901D09B0901E0940911709509118091B
:10B580006091190970911A0984169506A606B706E6
:10B5900008F47BC080910302882309F45BC05596B0
:10B5A0004D915D916D917C915897452B462B472B82
:10B5B000C1F459964D915D916D917C915C97452BAD
:10B5C000462B472B71F45D964D915D916D917C9169
:10B5D0009097452B462B472B21F48091880B88238D
:10B5E000C9F191966D917D918D919C9194979996C9
:10B5F0000C919997E4E00E9F80011124F801E55326
:10B60000F74FC080D180E280F380AA5BBF4F2C91BE
:10B6100023FF07C090958095709561957F4F8F4F60
:10B620009F4F0F94A9142091C7083091C8084091EA
:10B63000C9085091CA080F9408159B01AC01C701B5
:10B64000B6010F94A51BF801E553F74F6083718392
:10B65000828393831092D7081092A6171092A51791
:10B660009091D2148091D314981711F40C946F63B5
:10B670008091D3148F5F8F708093D31440EDC42ECC
:10B6800047E0D42EE12CF12C1CC4409113095091B9
:10B6900014096091150970911609481559056A0534
:10B6A0007B0508F4ABC140910F09509110096091DE
:10B6B000110970911209D6960D911D912D913C9111
:10B6C000D997401751076207730708F078C14115F1
:10B6D00051056105710549F48090D3089090D40814
:10B6E000A090D508B090D60865C1E12CF980842ED1
:10B6F000952F862F0A811B81FD81EE813F81288550
:10B700009C80E091521EE89D912CFF273091531EA2
:10B71000389D900CF11D1090541E189CF00DE99F5F
:10B72000900CF11D399FF00DE89FF00D092D1F2F92
:10B73000099DE12D332722270F9FE00D311D2E1D7E
:10B74000199DE00D311D2E1D1F9F300D211D032F52
:10B75000122F099DF12C332722270F9FF00C311D4A
:10B760002E1D199DF00C311D2E1D1F9F300D211D0A
:10B77000032F122FEE278090D3089091D408809148
:10B78000D508009028080E2809F484C030912408B8
:10B79000309FE1198E089E098E0920912508209F6F
:10B7A000E01981089E098E09F0902608F09E801805
:10B7B00091098E09319FE01981089E098E09219F08
:10B7C000801891098E09F19E90198109099DF12C2B
:10B7D000332722270F9FF00C311D2E1D199DF00CD1
:10B7E000311D2E1D1F9F300D211D032F122F309153
:10B7F0002008309FE10D8E1C9E1D8E1D209121087A
:10B80000209FE00D811C9E1D8E1DF0902208F09E51
:10B81000800C911D8E1D319FE00D811C9E1D8E1D83
:10B82000219F800C911D8E1DF19E900D811D099D03
:10B83000F12C332722270F9FF00C311D2E1D199D4F
:10B84000F00C311D2E1D1F9F300D211D032F122FB7
:10B8500030911C08309FE1198E089E098E092091B5
:10B860001D08209FE01981089E098E09F0901E088E
:10B87000F09E801891098E09319FE01981089E0978
:10B880008E09219F801891098E09F19E90198109D6
:10B890000C94CC5C30912408309FE10D8E1C9E1DD1
:10B8A0008E1D20912508209FE00D811C9E1D8E1D60
:10B8B000F0902608F09E800C911D8E1D319FE00DAA
:10B8C000811C9E1D8E1D219F800C911D8E1DF19E41
:10B8D000900D811D099DF12C332722270F9FF00C1D
:10B8E000311D2E1D199DF00C311D2E1D1F9F300D79
:10B8F000211D032F122F30912008309FE1198E084F
:10B900009E098E0920912108209FE01981089E0937
:10B910008E09F0902208F09E801891098E09319FBF
:10B92000E01981089E098E09219F801891098E09CE
:10B93000F19E90198109099DF12C332722270F9F31
:10B94000F00C311D2E1D199DF00C311D2E1D1F9F59
:10B95000300D211D032F122F30911C08309FE10D57
:10B960008E1C9E1D8E1D20911D08209FE00D811CA8
:10B970009E1D8E1DF0901E08F09E800C911D8E1D48
:10B98000319FE00D811C9E1D8E1D219F800C911DFD
:10B990008E1DF19E900D811D11249C82F9820A83D7
:10B9A0001B83FD83EE833F832887912C992AA12C4A
:10B9B000B12CA82A8AE197E121E0298B14C0D29604
:10B9C0008D909D90AD90BC90D597F4CFB694A794F0
:10B9D00097948794D988DD0CD98A049627E1863319
:10B9E000920709F4E0C4FC01059115912591349169
:10B9F000081519052A053B0548F3D5C440900809E8
:10BA00005090090960900A0970900B094814590474
:10BA10006A047B0408F0C4C180910709811121C028
:10BA2000FD01EE5BFF4FE080F1800281138178968B
:10BA30002081318142815381D2966D917D918D918A
:10BA40009C91D5970F94B100DD24D394D09207092F
:10BA5000E091A517F091A61782A993A9A4A9B5A969
:10BA60008FC14091030950910409609105097091BB
:10BA70000609DA960D911D912D913C91DD974017A5
:10BA800051076207730708F074C14115510561053C
:10BA9000710549F48091D3089091D408A091D508FC
:10BAA000B091D6086DC1F0E0E985842F352F262F9F
:10BAB000AA857B856C855D85BE854F859889B0910B
:10BAC000521EB89F612D55274091531E489F600D0F
:10BAD000511D1090541E189E500DB39F600D511DA6
:10BAE000439F500DB29F500DA62F752FA69FB12DCD
:10BAF00044279927A59FB00D411D9F1F769FB00D2C
:10BB0000411D9F1F759F400D911DA42F792FA69F4A
:10BB1000E12D44279927A59FE00D411D9F1F769F8A
:10BB2000E00D411D9F1F759F400D911DA42F792F82
:10BB3000BB278091D3083091D4082091D50800907C
:10BB400028080F2A09F484C0409124084A9FB1199B
:10BB50008F0B3F0B2F0B909125089A9FB0198109ED
:10BB60003F0B2F0BE0912608EA9F801931092F0B1C
:10BB7000479FB01981093F0B2F0B979F80193109FF
:10BB80002F0BE79F30192109A69FE12D4427992704
:10BB9000A59FE00D411D9F1F769FE00D411D9F1F3A
:10BBA000759F400D911DA42F792F409120084A9F29
:10BBB000B10D8F1F3F1F2F1F909121089A9FB00D2D
:10BBC000811D3F1F2F1FE0912208EA9F800D311D2C
:10BBD0002F1F479FB00D811D3F1F2F1F979F800D67
:10BBE000311D2F1FE79F300D211DA69FE12D4427FA
:10BBF0009927A59FE00D411D9F1F769FE00D411DD8
:10BC00009F1F759F400D911DA42F792F40911C08F7
:10BC10004A9FB1198F0B3F0B2F0B90911D089A9FD4
:10BC2000B01981093F0B2F0BE0911E08EA9F801984
:10BC300031092F0B479FB01981093F0B2F0B979F9D
:10BC4000801931092F0BE79F301921090C94AA5E46
:10BC5000409124084A9FB10D8F1F3F1F2F1F9091C5
:10BC600025089A9FB00D811D3F1F2F1FE0912608C8
:10BC7000EA9F800D311D2F1F479FB00D811D3F1F73
:10BC80002F1F979F800D311D2F1FE79F300D211D06
:10BC9000A69FE12D44279927A59FE00D411D9F1FD9
:10BCA000769FE00D411D9F1F759F400D911DA42F94
:10BCB000792F409120084A9FB1198F0B3F0B2F0B12
:10BCC000909121089A9FB01981093F0B2F0BE091A9
:10BCD0002208EA9F801931092F0B479FB01981096B
:10BCE0003F0B2F0B979F801931092F0BE79F3019BE
:10BCF0002109A69FE12D44279927A59FE00D411D0D
:10BD00009F1F769FE00D411D9F1F759F400D911D48
:10BD1000A42F792F40911C084A9FB10D8F1F3F1F00
:10BD20002F1F90911D089A9FB00D811D3F1F2F1F3F
:10BD3000E0911E08EA9F800D311D2F1F479FB00D17
:10BD4000811D3F1F2F1F979F800D311D2F1FE79FC4
:10BD5000300D211D1124E987AA877B876C875D87B9
:10BD6000BE874F87988B90E0932BA0E0B0E0A22B8A
:10BD700007C0A65ABF4F8D919D910D90BC91A02DEB
:10BD80002AE137E141E0498BF901459155916591EF
:10BD90007491481759076A077B0708F48EC39CC340
:10BDA00080910C098823E1F0FD01E85BFF4F4081A1
:10BDB000518160E070E00091090210910A02209127
:10BDC0000B0230910C02401751076207730741F0D4
:10BDD00010920D0210920E0210920F021092100299
:10BDE000409105025091060260910702709108028D
:10BDF00077FF5FC0AE5ABF4FCD90DD90ED90FC90C5
:10BE00008AE197E121E0FC0145915591659174919A
:10BE10004C155D056E057F0550F4F694E794D794B4
:10BE2000C794220F0496F7E186339F0761F72093AA
:10BE30000E0920E2C216D104E104F10428F460E204
:10BE4000C62ED12CE12CF12C90E2C91AD108E108C0
:10BE5000F108C114A8E0DA06E104F10408F4F8C31B
:10BE6000B4E0DB9EC0011124865E9C4EFC0132963C
:10BE700025913491EC2D6627E39FA001E29F410DAF
:10BE8000561F0694461F561F112460E070E0FC0107
:10BE900025913491C901A0E0B0E0841B950BA60B5D
:10BEA000B70B8093050290930602A0930702B0930C
:10BEB0000802C0900502D0900602E0900702F090C0
:10BEC00008028091A5179091A617892B09F0E8C167
:10BED0000F9437019093A6178093A517892B09F427
:10BEE000DFC1E091A517F091A617808183FF3EC0C6
:10BEF000858D968DA78DB0A1418D528D638D748DEA
:10BF0000058916892789308D0093B4171093B517CA
:10BF10002093B6173093B7174093B8175093B917BB
:10BF20006093BA177093BB178093BC179093BD179B
:10BF3000A093BE17B093BF1781A192A1A3A1B4A1F2
:10BF40008093C0179093C117A093C217B093C317E3
:10BF50009091D2148091D314981709F4B9CF80919D
:10BF6000D3148F5F8F708093D314B2CFC588D688D7
:10BF7000E788F08C81E0C114D104E104F10409F4F4
:10BF800080E0018D128D238D348D01151105210561
:10BF9000310509F08260458D568D678D70A1411580
:10BFA00051056105710509F084608093D7081092EE
:10BFB00003091092040910920509109206091092C3
:10BFC0000F0910921009109211091092120985A1FF
:10BFD00096A1A7A1B0A58093170990931809A093E3
:10BFE0001909B0931A09882499245401881A990AC6
:10BFF000AA0ABB0A8092F3089092F408A092F5086E
:10C00000B092F6088092F7089092F808A092F9088A
:10C01000B092FA088092FB089092FC08A092FD086A
:10C02000B092FE088092FF0890920009A092010948
:10C03000B092020981A092A0A3A0B4A0880C991C80
:10C04000AA1CBB1CCC0CDD1CEE1CFF1CC092E30820
:10C05000D092E408E092E508F092E608000F111F84
:10C06000221F331F0093E7081093E8082093E90884
:10C070003093EA08440F551F661F771F4093EB0863
:10C080005093EC086093ED087093EE088092EF08EF
:10C090009092F008A092F108B092F208880F991FD0
:10C0A000AA1FBB1F8093DF089093E008A093E108CC
:10C0B000B093E20810921B0910921C0910921D09FE
:10C0C00010921E0982A593A5A4A5B5A58093130976
:10C0D00090931409A0931509B093160986A597A506
:10C0E000A0A9B1A98093080990930909A0930A090E
:10C0F000B0930B0981A58093DE0890910402891703
:10C1000021F01092DD081092DC08DF01A95BBF4F1F
:10C110002C9120930D09222339F115962D913C91F4
:10C1200011973093DB082093DA0812972D913C91F8
:10C1300011973093D9082093D80810920D021092CD
:10C140000E0210920F021092100212972D913C9144
:10C15000A90160E070E04093090250930A026093E5
:10C160000B0270930C020CC088248A94982C540102
:10C170008092090290920A02A0920B02B0920C02E5
:10C18000EA5BFF4F208130916909231302C08917B0
:10C1900031F020936909809304020F940301809188
:10C1A000680981110E944FE02FEF3FEFA901209312
:10C1B0000502309306024093070250930802E09173
:10C1C000A517F091A617DF01DE96ED90FD900D9179
:10C1D0001C9122A933A944A955A9EA5AFF4F6081AD
:10C1E0007181828193810F94B10010920709E091CF
:10C1F000A517F091A617EA5AFF4F80809180A28080
:10C20000B3808AE197E121E0FC0145915591659168
:10C210007491481559056A057B0558F4B694A7949E
:10C2200097948794220F049646E357E148175907DD
:10C2300059F720930E0950E285169104A104B10428
:10C2400028F4B0E28B2E912CA12CB12C30E2831A71
:10C250009108A108B108811448E09406A104B10432
:10C2600008F41AC254E0959EC0011124865E9C4ECB
:10C27000FC01329625913491782D6627739FA00199
:10C28000729F410D561F0694461F561F1124FC0134
:10C29000C590D490E12CF12CC41AD50AE108F1081C
:10C2A000C0921F09D0922009E0922109F092220940
:10C2B00000911F0910912009209121093091220934
:10C2C00040910D0250910E0260910F027091100288
:10C2D000F02E198BF22FE32F4017510762077307D7
:10C2E00020F4F42E598BF62FE72F8F2D9989AF2F3D
:10C2F000BE2F0097E1E0AE07B10520F08FEF9FEF72
:10C30000A0E0B0E0081B190B2A0B3B0B00931F09A0
:10C310001093200920932109309322094F3FFFEF0A
:10C320005F076F077F0761F0481B590B6A0B7B0B98
:10C3300040930D0250930E0260930F02709310020F
:10C34000F8942091840030918500205F3F4F4A8906
:10C3500041504A8B442341F0280E391E22163306E1
:10C3600010F40C94FF5701C01901309289002092FB
:10C370008800789462960FB6F894DEBF0FBECDBFEA
:10C38000DF91CF911F910F91FF90EF90DF90CF90B1
:10C39000BF90AF909F908F907F906F905F904F90E5
:10C3A0003F902F900895398930930E0980E28816C6
:10C3B0009104A104B10428F430E2832E912CA12C25
:10C3C000B12C30E2831A9108A108B108811488E0E9
:10C3D0009806A104B10420F1E4E09E9EC00111245E
:10C3E000865E9C4EFC01329625913491F82DEE2705
:10C3F000F39F7001F29FE10CFE1E0694EE1EFE1EDE
:10C400001124FC01C590D490860120E030E0480161
:10C4100059018E189F08A108B1087501640122C056
:10C42000950184013695279517950795F801EC7FBE
:10C43000CF01865E904FFC01C590D490FC013296EE
:10C4400025913491E82DE770E29FC001E39F900DA4
:10C45000112423E0969587952A95E1F7C81AD90A01
:10C46000E12CF12C4C0D5D1D6E1D7F1D40930F09BD
:10C4700050931009609311097093120990910D095E
:10C4800080910C09992309F474C0882309F419CD0B
:10C49000A85BBF4F8D919C91A0E0B0E04091090254
:10C4A00050910A0260910B0270910C02841795075B
:10C4B000A607B70709F060C004CDB695A795979574
:10C4C00087954989440F498B2C5F3F4FE6E3F7E19D
:10C4D000E217F30709F058CCD988D0920E098032C0
:10C4E0009105A105B10520F480E290E0A0E0B0E064
:10C4F0008097A109B109811558E09507A105B105FB
:10C5000008F443C074E0979F90011124265E3C4ECE
:10C51000F901329645915491EE27859FB001849F91
:10C52000610D7E1F06946E1F7E1F1124F901C590B8
:10C53000D490E12CF12CC61AD70AE108F1088091B9
:10C54000030990910409A0910509B09106098C0D89
:10C550009D1DAE1DBF1D8093030990930409A093F8
:10C560000509B093060980910D09811130C08091B1
:10C570000C09882309F4A5CC10920D0210920E022A
:10C5800010920F02109210029CCCAC01BD01769566
:10C59000679557954795FA01EC7F9F01265E304FCE
:10C5A000F901C590D490F901329645915491877064
:10C5B000849F9001859F300D1124F3E036952795D7
:10C5C000FA95E1F7C21AD30AE12CF12CB8CF898988
:10C5D000480E511C611C711C8091A5179091A617E3
:10C5E000481459046A047B04D8F420910C092223CE
:10C5F00009F467CCFC01E85BFF4F20813181A90180
:10C6000060E070E00091090210910A0220910B0293
:10C6100030910C02401751076207730709F451CC9F
:10C6200010920D0210920E0210920F021092100240
:10C63000FC01E85BFF4F80819181A0E0B0E0809336
:10C64000090290930A02A0930B02B0930C0239CC1A
:10C65000D701C601B695A79597958795FC01EC7F04
:10C66000CF01865E904FFC0125913491FC013296FA
:10C67000459154916C2D6770649FC001659F900D2A
:10C68000112453E0969587955A95E1F7281B390BAD
:10C69000C901A0E0B0E005CCD501C401B695A795CD
:10C6A00097958795FC01EC7FCF01865E904FFC014A
:10C6B000C590D490FC01329625913491482D477055
:10C6C000429FC001439F900D1124A3E0969587954A
:10C6D000AA95E1F7C81AD90AE12CF12CE1CD80ED39
:10C6E000C82E87E0D82EE12CF12CF2CB80910901E5
:10C6F00080FD06C08091241783FB882780F9089568
:10C7000080E0089590917B13977081E0973009F055
:10C7100080E008958091D2149091D314891B8F707A
:10C7200069F48091FB0A811109C081E020917809A8
:10C7300030917909232B19F480E0089581E0089560
:10C74000CF92DF92EF92FF926B017C0160917B139D
:10C7500070917C13072E000C880B990B0F94A91471
:10C760009B01AC01C701B6010F94A51B2091080DD8
:10C770003091090D40910A0D50910B0D0F94081541
:10C780000F94121DCB01FF90EF90DF90CF900C948F
:10C790007FE4E091CB0DE150E53028F4F0E0E45087
:10C7A000FD4F8081089580E008953F924F925F92FF
:10C7B0006F927F928F929F92AF92BF92CF92DF92B1
:10C7C000EF92FF920F931F93CF93DF9300D000D08F
:10C7D000CDB7DEB72B013C01342E24E0429FC001CF
:10C7E00011249E838D83FC01E453F24FC080D180DD
:10C7F000E280F38020E030E04AE754E4C701B6016C
:10C800000F94A51B4B015C0120E030E04AE754E4A3
:10C81000C701B6010F94A61B7B018C0180916B02AE
:10C820008823D1F181E0381639F13816A0F092E072
:10C83000391232C08090510290905202A09053025F
:10C84000B0905402E0905D02F0905E0200915F02B1
:10C850001091600221C08090490290904A02A090FD
:10C860004B02B0904C02E0905502F09056020091BD
:10C8700057021091580210C080904D0290904E02C5
:10C88000A0904F02B0905002E0905902F0905A02EE
:10C8900000915B0210915C029401A501B201C301F9
:10C8A0000F94A21487FD0BC09701A801B201C30128
:10C8B0000F94061E18162CF07201830102C0740139
:10C8C0008501ED81FE81E453F24FC701D8018083D9
:10C8D0009183A283B383ED81FE81E451FD4F20E07B
:10C8E00030E040E752E460817181828193810F944E
:10C8F000A01C69837A838B839C83CE0101960E945E
:10C9000055DE26960FB6F894DEBF0FBECDBFDF9181
:10C91000CF911F910F91FF90EF90DF90CF90BF903C
:10C92000AF909F908F907F906F905F904F903F90CF
:10C9300008952091BD1320FF14C020E83EE3629FBC
:10C94000A001639F500D729F500D1124CA0196954E
:10C95000879596958795009731F08A950000E9F7BD
:10C9600008950C94264D08959F92AF92BF92CF9256
:10C97000DF92EF92FF920F931F93CF93DF938091FB
:10C980000818833009F50E9482638823E9F06091DA
:10C99000440970914509072E000C880B990B0F94E0
:10C9A000A91420E030E040E85FE30F94A51B20913C
:10C9B00040093091410940914209509143090F9437
:10C9C000A21418160CF062C0D0E000E010E0FF24C2
:10C9D000F394EE24E39445E0D42EC0E0CC24C39439
:10C9E00055E0B52E65E0A62E72E8972EFC24DC16E5
:10C9F000D1F18D2F90E04897A4F5DF5FF801BC9E40
:10CA0000E00DF11D1124EE0FFF1FEE0FFF1FEE5E74
:10CA1000F34F20E030E04AE754E460817181828185
:10CA200093810F9408150F94121D709381156093D4
:10CA30008015A0927415909277158D2F90E08158F3
:10CA4000974F880F991F092E000CAA0BBB0B8093E0
:10CA5000781590937915A0937A15B0937B150E9461
:10CA600007E1CE0DC4CF0F5F1F4F0530110579F1DF
:10CA7000F11006C0EE24EA94DD24DA94C4E0B6CFC7
:10CA8000EE24E39435E0D32EC0E0B0CF81E09AE508
:10CA9000909381158093801580E490E090938315A6
:10CAA0008093821587E08093741582E880937715D0
:10CAB00084E890E0A0E0B0E0809378159093791539
:10CAC000A0937A15B0937B150E9407E17DCFDF918B
:10CAD000CF911F910F91FF90EF90DF90CF90BF907B
:10CAE000AF909F900895AF92BF92CF92DF92EF9256
:10CAF000FF920F931F93CF93DF93EC0188EEC82E24
:10CB000080E2D82EE12CF12C02E8A12C90E2B92E83
:10CB100015E000937715C0927815D0927915E092C0
:10CB20007A15F0927B15B0928115A0928015109322
:10CB300074150E9407E18FEFC81AD80AE80AF80AAC
:10CB400080E1C81681E2D806E104F10411F748EE4D
:10CB500050E260E070E0CE01DF91CF911F910F9124
:10CB6000FF90EF90DF90CF90BF90AF900C94C5E115
:10CB700084E08093071882E08093E40781E09AE5DF
:10CB800090938115809380158EE490E090938315A7
:10CB90008093821587E08093741582E880937715DF
:10CBA00084E890E0A0E0B0E0809378159093791548
:10CBB000A0937A15B0937B150E9407E184EA96E072
:10CBC0000C94C24FCF92DF92EF92FF926A017B01E9
:10CBD0000E94759B882331F0FF90EF90DF90CF90FB
:10CBE0000C94F59AC701B601FF90EF90DF90CF90BB
:10CBF00008952F923F924F925F926F927F928F9201
:10CC00009F92AF92BF92CF92DF92EF92FF920F93DB
:10CC10001F93CF93DF93CDB7DEB7CC54D1090FB6B6
:10CC2000F894DEBF0FBECDBF60E070E085E40E94E7
:10CC30000CF1182F81E0810F823018F087EA9AE119
:10CC400040C065E070E083E40E940CF189A760E0D9
:10CC500085E50E94829B2B968FAF2B9717FF05C00F
:10CC600040E050E06CE872E404C040E050E066E16F
:10CC700073E483E50E94E2650F94121D072E000CF9
:10CC8000880B990B0F94A9146D837E838F832D9647
:10CC90009FAF2D970E9483D22B013C011F3F09F0CB
:10CCA000EBC420E030E047E053E46D817E818F816A
:10CCB0002D969FAD2D970F94061E1816ECF48CE759
:10CCC0009AE1C45BDF4F0FB6F894DEBF0FBECDBF55
:10CCD000DF91CF911F910F91FF90EF90DF90CF9058
:10CCE000BF90AF909F908F907F906F905F904F908C
:10CCF0003F902F900C94F84D88E69AE10E94F84DF1
:10CD00000E9443AB8FE78093460924EB30E0A8EE06
:10CD1000B3E00F944C1B6BA77CA78DA79EA79B012C
:10CD2000AC01240D351D461D571D28AF39AF4AAF44
:10CD30005BAF81E080932002109243021F3FF9F421
:10CD40008BEA9AEAAAEABEE38CAF9DAFAEAFBFAF63
:10CD50002DEC3CEC4CE45EE324962CAF3DAF4EAFA3
:10CD60005FAF249740EB59E126965FAF4EAF269711
:10CD70008AE799E128969FAF8EAF28971EC020E0E2
:10CD800030E040E05EE32CAF3DAF4EAF5FAF8AE9ED
:10CD900099E9A9E1BFE324968CAF9DAFAEAFBFAFD9
:10CDA0002497AEE9B9E12696BFAFAEAF2697E7E686
:10CDB000F9E12896FFAFEEAF289749A25AA26BA2DD
:10CDC0007CA24FA658AA69AA7AAA2FE730E040E0D1
:10CDD00050E0288739874A875B87188A198A1A8A18
:10CDE0001B8A1C861D861E861F86C12CD12C7601AF
:10CDF0001E8A30E43F8B4CE1488F56E4598F1A8EDF
:10CE00001B8E1C8E1D8E1BAACCAADDAAEEAAFFAA21
:10CE1000FFE78F2E912CA12CB12C1DA21EA21FA2C8
:10CE200018A681E088A31D8A1C8A212C312C00E0E1
:10CE30002C961FAE2C97A7E11A02C00111248B5D1E
:10CE4000964FFC013A962A96FFAFEEAF2A979C01C7
:10CE50002C5F3F4F3F8F2E8F49A5042E000C550BA2
:10CE60005AA749A780912002882309F457C20E943B
:10CE700083D269837A838B839C838091E80C882397
:10CE800009F4BAC00E94BDF71F3F61F42090400929
:10CE90003090410900914209509143092C965FAFAF
:10CEA0002C970EC0AE8DBF8D2C9011963C90119793
:10CEB00012960C9112971396BC912C96BFAF2C979B
:10CEC0002A8D3B8D4C8D5D8DB101802F2C969FADB1
:10CED0002C970F94061E18163CF42A8E3B8E0C8F4E
:10CEE0002C96EFAD2C97ED8F2E893F89488D598D6B
:10CEF000B101802F2C969FAD2C970F94A21487FF21
:10CF000007C02E8A3F8A088F2C96FFAD2C97F98F89
:10CF100028A1222309F44DC09101402F2C965FAD2A
:10CF20002C976D817E818F812D969FAD2D970F94CB
:10CF3000A21487FF61C049815A816B817C814419A9
:10CF4000550966097709DB01CA0188589341A1098F
:10CF5000B109B7FD51C088859985AA85BB85881917
:10CF60009909AA09BB09B595A795979587951F3F7C
:10CF700019F48093460905C02A96EEADFFAD2A97B5
:10CF800080834DA35EA36FA378A7FD81FA8F2E81C6
:10CF90002B8F3F813C8F2D964FAD2D974D8F8981E3
:10CFA0009A81AB81BC8189A39AA3ABA3BCA318A22D
:10CFB00023C09101402F2C965FAD2C976D817E810F
:10CFC0008F812D969FAD2D970F94061E1816A4F4F1
:10CFD00089819A81AB81BC8129A13AA14BA15CA135
:10CFE000821B930BA40BB50BAC01BD0148585341F8
:10CFF0006109710977FFB1C120E030E040EF51E4F1
:10D000006D817E818F812D969FAD2D970F94A61BEC
:10D010009101402F2C965FAD2C970F94A21487FF9F
:10D0200003C082ED99E1BCC089819A81AB81BC814A
:10D030002FA538A949A95AA9821B930BA40BB50B9C
:10D04000B7FD93C01F3F19F48091CB0D01C0812F14
:10D050000E944AA18AE00E94E64D89819A81AB81B3
:10D06000BC818053984FAF4FBF4F8FA798ABA9ABF0
:10D07000BAAB9BA9911159C02CA93DA94EA95FA992
:10D08000B101802F2C969FAD2C970F94061E181679
:10D09000BCF520E030E040E050E4B101802F2C9658
:10D0A0009FAD2C970F94A61B6CAB7DAB8EAB9FAB4B
:10D0B0002BA53CA54DA55EA589819A81AB81BC813C
:10D0C000280F391F4A1F5B1F28AF39AF4AAF5BAF2C
:10D0D00020E030E040EC50E46D817E818F812D9620
:10D0E0009FAD2D970F94A51B9101402F2C965FADFE
:10D0F0002C970F94A214881F8827881F8BAB35C0EC
:10D1000089819A81AB81BC8128AD39AD4AAD5BADD7
:10D11000821B930BA40BB50BB7FD27C026964EAD13
:10D120005FAD269763EC79E11DC020E030E040EF71
:10D1300051E46D817E818F812D969FAD2D970F9447
:10D14000A51B9B01AC01B101802F2C969FAD2C97A4
:10D150000F94A21487FF09C028964EAD5FAD2897A3
:10D160006EE879E1812F0E94DAF789819A81AB819B
:10D17000BC81880F991FAA1FBB1F29A13AA14BA1EF
:10D180005CA1821B930BA40BB50B84199509A6090E
:10D19000B70981389F44A241B10528F089E499E19B
:10D1A0000E94F84DBBC049A55AA58C899D89481796
:10D1B00059070CF0B0C003970CF4ADC08CEE98E1A9
:10D1C0000E94F84D1F3F29F4ACEDB8E1BA83A98362
:10D1D00004C0EBEDF8E1FA83E9838AEC98E10E9460
:10D1E000F84D89819A810E94F84DB701A60188EE19
:10D1F00098E10E94AB4F8AE00E94E64D8AEC98E1EC
:10D200000E94F84D89819A810E94F84D4C855D8578
:10D210006E857F8584EE98E10E94AB4F8AE00E9484
:10D22000E64D8AEC98E10E94F84D89819A810E942E
:10D23000F84D488959896A897B8980EE98E10E9476
:10D24000AB4F8AE00E94E64D2B96FFAD2B97FF2354
:10D2500009F466C01F3F69F5C0924709D09248099A
:10D26000E0924909F0924A092CEA35EC47E25EE384
:10D270006C857D858E859F850F94081560934B097D
:10D2800070934C0980934D0990934E092CEA35EC2C
:10D2900047E25EE3688979898A899B890F94A01C9B
:10D2A00060934F09709350098093510990935209EC
:10D2B00037C047E11402900111242B5D364F3A83A9
:10D2C0002983D9011B96CD92DD92ED92FC921E9797
:10D2D0002CEA35EC47E25EE36C857D858E859F8583
:10D2E0000F940815E981FA816787708B818B928B87
:10D2F0002CEA35EC47E25EE3688979898A899B8963
:10D300000F94A01CA981BA8153966D937D938D9340
:10D310009C93569705C00E94B91BA4CD0E9443ABB5
:10D3200081E080934302C45BDF4F0FB6F894DEBF09
:10D330000FBECDBFDF91CF911F910F91FF90EF9066
:10D34000DF90CF90BF90AF909F908F907F906F9025
:10D350005F904F903F902F9008954C895D89452BA9
:10D3600009F451C14DA05EA06FA078A4480E591ECB
:10D370006A1E7B1E2DA13EA14FA158A5281B390B6B
:10D380004A0B5B0BC501B4010F94E81AA30192018B
:10D390000F941A1B88849984AA84BB84820E931EDE
:10D3A000A41EB51E54E185169104A104B1040CF12C
:10D3B0008CEE88169104A104B1043CF490E889161F
:10D3C0009104A104B10434F422C06BEE862E912C9A
:10D3D000A12CB12C88869986AA86BB862EEF30E0D8
:10D3E00040E050E0281939094A095B0949015A010E
:10D3F00012C084E190E0A0E0B0E088879987AA8716
:10D40000BB8754E1852E912CA12CB12C04C08886B9
:10D410009986AA86BB8680E69AE10E94F84D6885C7
:10D4200079858A859B850E940D4F8BE59AE10E9444
:10D43000F84DC501B4010E940D4F4E895F89688D7A
:10D44000798D84E59AE10E94AB4F4A8D5B8D6C8D9E
:10D450007D8D8DE49AE10E94AB4FAC89BD89139715
:10D460000CF4D1C0C501B4010F94A91420E030E040
:10D4700040E850E40F9408156B017C012E893F8928
:10D48000488D598D6A8D7B8D8C8D9D8D0F94A51B3C
:10D490002BED3FE049E450E40F94081520E030E024
:10D4A00040E05FE30F9408159B01AC01C701B60192
:10D4B0000F94A01C6B017C01C301B2010F94A9144D
:10D4C0002FE632E143E85AE30F9408152B013C01A3
:10D4D000B701A60187E49AE10E94AB4FB301A20114
:10D4E00081E49AE10E94AB4F1F3F09F044C02DEC4C
:10D4F0003CEC4CE45EE3C701B6010F9408156B01E8
:10D500007C019B01AC010F94A61BA30192010F9417
:10D51000A01C6C877D878E879F87A7019601C3011A
:10D52000B2010F94081520E030E040E450E40F947D
:10D53000A01C688B798B8A8B9B8B81E39AE10E947C
:10D54000F84DB701A6018BE29AE10E94AB4F4C85E2
:10D550005D856E857F8585E29AE10E94AB4F4889A3
:10D5600059896A897B898FE19AE10E94AB4F8AE0F1
:10D570000E94E64D4AC024962CAD3DAD4EAD5FAD48
:10D580002497C701B6010F9408156B017C019B011C
:10D59000AC01C301B2010F9408152CAD3DAD4EADE9
:10D5A0005FAD0F940815688B798B8A8B9B8BA701D5
:10D5B0009601C701B6010F94A61BA30192010F9417
:10D5C000A01C6C877D878E879F878FE09AE10E94E1
:10D5D000F84DB701A60189E09AE10E94AB4F4C8556
:10D5E0005D856E857F8583E09AE10E94AB4F488917
:10D5F00059896A897B898DEF99E10E94AB4F8AE056
:10D600000E94E64D11C01F3F79F488859985AA854F
:10D61000BB85880D991DAA1DBB1DB595A79597952E
:10D6200087958093460911C088859985AA85BB8511
:10D63000880D991DAA1DBB1DB595A7959795879532
:10D640002A96EEADFFAD2A9780832C893D892F5F06
:10D650003F4F3D8B2C8B3D813E8B4E814F8B5F81AD
:10D66000588F2D968FAD2D97898F49805A806B806A
:10D670007C8091E098A3C0CCE12E012E000CFF0825
:10D68000F70183E0EE0FFF1F8A95E1F7E85EFD4F9B
:10D69000668177816F507109072E000C880B990BFA
:10D6A0000F94A9149B01AC016D817E818F812D9611
:10D6B0009FAD2D970F94061E18160CF400CB88E62C
:10D6C0009AE10E94F84D0E9443AB87E18E9DF001E4
:10D6D0008F9DF00D1124EB5DF64F8FE7828722E3DB
:10D6E00030E015CB2F923F924F925F926F927F92D4
:10D6F0008F929F92AF92BF92CF92DF92EF92FF9262
:10D700000F931F93CF93DF93D62FC72FFC018080F9
:10D710009180A280B380C501B40120E831E541E0E9
:10D7200050E00F94F81AC9016DE671E00F94691B7F
:10D730006B017C01C501B40120E13EE040E050E016
:10D740000F94F81ACA01B90128E130E040E050E036
:10D750000F94F81A362E272E062F172F8CE3482EFB
:10D76000512C612C712CC501B401A30192010F94BD
:10D77000F81AB62EA72ECA01B901A30192010F947F
:10D78000F81ACB01C114D104D9F0AF92BF927F93A4
:10D790006F932F923F92FF92EF92DF92CF9286EBA0
:10D7A00098E19F938F93CF93DF930F943A148DB7A3
:10D7B0009EB70E960FB6F8949EBF0FBE8DBF5CC08D
:10D7C000E114F104C9F0AF92BF927F936F932F924F
:10D7D0003F92FF92EF9286EA98E19F938F93CF93C7
:10D7E000DF930F943A14EDB7FEB73C960FB6F8945A
:10D7F000FEBF0FBEEDBF40C0012BB9F0AF92BF928C
:10D800007F936F932F923F928AE998E19F938F9332
:10D81000CF93DF930F943A148DB79EB70A960FB645
:10D82000F8949EBF0FBE8DBF27C0892BA9F0AF9281
:10D83000BF927F936F9382E998E19F938F93CF93E9
:10D84000DF930F943A14EDB7FEB738960FB6F894FD
:10D85000FEBF0FBEEDBF10C0AF92BF928EE898E141
:10D860009F938F93CF93DF930F943A140F900F9061
:10D870000F900F900F900F908D2F9C2FDF91CF91D5
:10D880001F910F91FF90EF90DF90CF90BF90AF90DE
:10D890009F908F907F906F905F904F903F902F90D0
:10D8A00008958F929F92AF92BF92CF92DF92EF92A4
:10D8B000FF920F931F93CF93DF93CDB7DEB7E69719
:10D8C0000FB6F894DEBF0FBECDBF0091860B10914E
:10D8D000870BF80101900020E9F731976F01C01A1A
:10D8E000D10AF801CF01801B910B8C159D0534F4F2
:10D8F00080818F3209F410823196F4CF8BE1E4EB12
:10D90000F4E1DE015C9601900D928A95E1F7E12C3D
:10D91000F12CEC14FD040CF07AC0F801EE0DFF1DA3
:10D920008081811103C08FEFE81AF80A48018E0C3C
:10D930009F1CF4018081882309F469C0FFEFEF1A6E
:10D94000FF0AF801EE0DFF1D7F01E01AF10A819137
:10D950008111FACFCE014C960E9470938BE1FE01AB
:10D960007C96DE01119601900D928A95E1F7B40143
:10D97000CE0101960E941673CE0101960E94A694D4
:10D980008FE20E94E64D8091F40F811103C08EEB6F
:10D9900096E002C084EF9FE05C01F50181915F0198
:10D9A000882319F00E94E64DF8CF8091241784FF58
:10D9B0002EC019821C8221E0A401BE01645E7F4F4B
:10D9C000CE0101960E94A09881110FC08AE00E94AA
:10D9D000E64D0E942A4EB4018AE798E10E94134E58
:10D9E000CE0101960E94A69412C0CE014C960E94D0
:10D9F0009D948BE1FE013196DE015C9601900D92C3
:10DA00008A95E1F7CE0101960E94A69482CF8AE022
:10DA10000E94E64DCE014C960E94A694E6960FB663
:10DA2000F894DEBF0FBECDBFDF91CF911F910F9154
:10DA3000FF90EF90DF90CF90BF90AF909F908F902E
:10DA40000895CF93DF93E091FA0AF0E0E252FA4EA4
:10DA50008081882309F447C08EE698E10E94F84D42
:10DA6000C091FA0A80E6C89FE0011124C658D64F3B
:10DA700088818E3479F480E20E94E64D89910E947B
:10DA8000E64D899190ED980F9A30C8F38D32B9F335
:10DA90008B32A9F38BE698E10E94F84D8091D21465
:10DAA0009091D314891B8F706FE070E0681B71092F
:10DAB000072E000C880B990B0E940D4F88E698E109
:10DAC0000E94F84D8091FB0A64E070E0681B7109C8
:10DAD000072E000C880B990B0E940D4F8AE0DF91F6
:10DAE000CF910C94E64DDF91CF910895EEEFFAE0DF
:10DAF0008081818381E798E10E94F84D8091820BBB
:10DB00009091830BA091840BB091850BBC01CD014A
:10DB10006F5F7F4F8F4F9F4F0E940D4F0E94BC4FF2
:10DB20000C94216D0F931F93CF938C01C62F0E94ED
:10DB3000264EC8010E94F84D6091820B7091830BB4
:10DB40008091840B9091850B0E940D4F0E94BC4FD9
:10DB5000C11104C00E94CF4F0196E1F70E94766D7B
:10DB6000EC2FEE0FFF0BE058F44F11821082CF9193
:10DB70001F910F9108955F926F927F928F929F9263
:10DB8000AF92BF92CF92DF92EF92FF920F931F93CB
:10DB9000CF93DF93CDB7DEB76DB67EB67C0100E0E4
:10DBA00010E08DB69EB6F701E00FF11F5490C8014A
:10DBB00001965C01552029F09AE0591611F0850173
:10DBC000F2CF8DB79EB78A199B090FB6F8949EBF06
:10DBD0000FBE8DBF01966C01A801B7010F94DC1335
:10DBE000F601E00FF11F1082C6010E94CBE4552020
:10DBF00041F0EA0CFB1C0FB6F8949EBE0FBE8DBE22
:10DC0000D0CF0FB6F8947EBE0FBE6DBEDF91CF9120
:10DC10001F910F91FF90EF90DF90CF90BF90AF904A
:10DC20009F908F907F906F905F900895CF92DF923A
:10DC3000EF92FF920F931F93CF93DF936C017A01C2
:10DC40008B01C0E0D0E0CE15DF0581F0D8016D91E9
:10DC50008D01D601ED91FC910190F081E02DC6017E
:10DC60001995892B11F02196EECF7E01C701DF9126
:10DC7000CF911F910F91FF90EF90DF90CF9008957B
:10DC8000089580E090E00895FC01538D448D252F88
:10DC900030E0842F90E0821B930B541710F0CF9646
:10DCA000089501970895FC01918D828D981761F078
:10DCB000828DDF01A80FB11D5D968C91928D9F5FC3
:10DCC0009F73928F90E008958FEF9FEF0895FC016E
:10DCD000918D828D981731F0828DE80FF11D858D21
:10DCE00090E008958FEF9FEF0895FC01918D228DB4
:10DCF000892F90E0805C9F4F821B91098F73992739
:10DD000008958EEB93E10E94756E21E0892B09F452
:10DD100020E0822F0895FC01848DDF01A80FB11D42
:10DD2000A35ABF4F2C91848D90E001968F73992751
:10DD3000848FA689B7892C93A089B1898C9183702F
:10DD400080648C93938D848D981306C00288F38928
:10DD5000E02D80818F7D80830895EF92FF920F9355
:10DD60001F93CF93DF93EC0181E0888F9B8D8C8D87
:10DD7000981305C0E889F989808185FD26C0F62EB3
:10DD80000B8D10E00F5F1F4F0F731127E02E8C8D4E
:10DD9000E8120CC00FB607FCFACFE889F989808138
:10DDA00085FFF5CFCE010E948B6EF1CF8B8DFE01EA
:10DDB000E80FF11DE35AFF4FF0829FB7F8940B8FE5
:10DDC000EA89FB89808180620AC09FB7F894EE8956
:10DDD000FF896083E889F98980818370806480830A
:10DDE0009FBF81E090E0DF91CF911F910F91FF9055
:10DDF000EF900895CF93DF93EC01888D8823C9F0CD
:10DE0000EA89FB89808185FD05C0A889B9898C9143
:10DE100086FD0FC00FB607FCF5CF808185FFF2CFDE
:10DE2000A889B9898C9185FFEDCFCE010E948B6EB8
:10DE3000E7CFDF91CF91089580E090E0892B41F00A
:10DE400080E090E0892B21F00E940000811121C028
:10DE500080E090E0892B41F080E090E0892B21F078
:10DE60000E940000811118C080E090E0892B21F011
:10DE70000E94816E811113C080E090E0892BA1F097
:10DE800080E090E0892B81F00E94000081110AC09F
:10DE900008950E940000DCCF0E940000E5CF0E94A0
:10DEA0000000EACF0C94000008950F94B81ECF93A1
:10DEB000DF93EC01CB01E881F981608171810E94DF
:10DEC000379288819981DC01ED91FC912081AA81B2
:10DED000BB81222369F02C91293650F43196DC0164
:10DEE000ED93FC93EA81FB8180818F5F8083E9CF92
:10DEF0008C91893670F48FE28083E881F98180818A
:10DF00009181019691838083EA81FB8180818F5F7B
:10DF10008083DF91CF9108951F920F920FB60F92D9
:10DF200011240BB60F922F933F934F935F936F93F0
:10DF30007F938F939F93AF93BF93EF93FF938EEB5A
:10DF400093E10E948B6EFF91EF91BF91AF919F91F2
:10DF50008F917F916F915F914F913F912F910F9092
:10DF60000BBE0F900FBE0F901F9018951F920F922F
:10DF70000FB60F9211240BB60F922F938F939F938E
:10DF8000EF93FF93E091CE13F091CF138081E09156
:10DF9000D413F091D51382FD12C090818091D713D4
:10DFA0008F5F8F732091D813821751F0E091D713B0
:10DFB000F0E0E254FC4E958F8093D71301C080812E
:10DFC000FF91EF919F918F912F910F900BBE0F902A
:10DFD0000FBE0F901F9018958BE1E4EBF4E1A9E9D7
:10DFE000B4E101900D928A95E1F780912417806247
:10DFF0008093241708958091241782FF1FC08CE21C
:10E000009CE10E94F84D609120177091211780913A
:10E010002217909123174AE00E94824E8FE20E94BD
:10E02000E64D60911C1770911D1780911E179091FD
:10E030001F174AE00E94824E0C94BC4F8EE39CE175
:10E040000C94F84D1092880B809124178F7B8B7F56
:10E05000809324170E94914D882321F08BE594E151
:10E060000C949D9408958091241783FF03C08460CD
:10E07000809324170895CF92DF92EF92FF920F932F
:10E080001F93CF93DF93CDB7DEB7EDB6FEB6DC01BD
:10E090000D900020E9F79D01281B390B2C5F3F4FA5
:10E0A0004DB75EB7421B530B0FB6F8945EBF0FBE61
:10E0B0004DBF0DB71EB70F5F1F4F9F938F9388E221
:10E0C0009BE19F938F931F930F930F943A146801D2
:10E0D00054E0C50ED11C0F900F900F900F900F9031
:10E0E0000F90F6018081882349F0082E000C990BCF
:10E0F0000F94BD1EF60181936F01F3CFC8010E94FA
:10E10000CBE484E29BE10E94BB6D0FB6F894FEBEA7
:10E110000FBEEDBEDF91CF911F910F91FF90EF9059
:10E12000DF90CF9008958F929F92AF92BF92CF923F
:10E13000DF92EF92FF92CF9380912417877F809395
:10E1400024178091B714882321F084EB94E10E9476
:10E150009D94109298141092951485E380939414D2
:10E160000E9483D26B017C0120EDC20E27E0D21EFB
:10E17000E11CF11CA89561E0809194140E94F6D0F6
:10E1800061E0809194140E9425D1209A289A219AC6
:10E190002398229A81E00E94CA5785E080939614C2
:10E1A0000E94CA57CAE08FEF0E94BE57C150D9F7EC
:10E1B000A89520E030E0A90160E084E994E10E94A4
:10E1C0007D9380939714813061F00E9483D2DC01AB
:10E1D000CB018C199D09AE09BF09B7FDEACF81E0DB
:10E1E00062C0A8952AEA31E040E050E068E084E9A6
:10E1F00094E10E947D93853011F481E00AC0C4E06F
:10E200000E94C35780939714C150D1F78A3A61F4A2
:10E2100082E080939814A89580919814823081F0C0
:10E22000812C912C540111C00E9483D2DC01CB01BE
:10E230008C199D09AE09BF09B7FDD4CF82E033C068
:10E24000812C912CA12C80E4B82E20E030E0A90193
:10E2500067E384E994E10E947D93A501940169E25A
:10E2600084E994E10E947D9380939714882361F060
:10E270000E9483D2DC01CB018C199D09AE09BF0934
:10E28000B7FDE3CF8AE00FC080919814823021F56A
:10E2900020E030E0A9016AE384E994E10E947D93E3
:10E2A000882361F088E08093951484E994E10E94CA
:10E2B00075930E942A4E86E19BE122C00E94C357BB
:10E2C000807C803C19F483E0809398140E94C357AB
:10E2D0000E94C3570E94C35784E994E10E9475933A
:10E2E0001092961481E00E94AECC81110CC080E0A7
:10E2F0000E94AECC811107C00E94264E82E09BE1B5
:10E300000E94F84D1AC066E774E184EB94E10E9424
:10E31000C891811105C00E94264E81EF9AE1F0CF8D
:10E32000809124178860809324170E942A4E85EEDE
:10E330009AE10E94F84D0E94854DCF91FF90EF9099
:10E34000DF90CF90BF90AF909F908F900C94EC6F28
:10E35000FC0180818823E1F0853ED1F08E32C1F04E
:10E360008091F40F8E32A1F09385892F8A7081F409
:10E37000987121E0903109F020E08091241720FB72
:10E3800084F980932417903141F08085873411F00F
:10E3900080E0089581858E37D9F381E008950F9349
:10E3A0001F93CF93DF93CDB7DEB7EB970FB6F894FB
:10E3B000DEBF0FBECDBF89E994E10E9470938BE16F
:10E3C000E9E9F4E1DE01919601900D928A95E1F779
:10E3D00000E010E044EF5FE0BE016F5F7F4FCE01D1
:10E3E00081960E94329618163CF4CE0101960E9446
:10E3F000A871080F111DEECFCE0181960E94A69440
:10E40000C801EB960FB6F894DEBF0FBECDBFDF910B
:10E41000CF911F910F910895FC0120E03EE2DB01B6
:10E420004C91403241F0283011F430833196DB01B9
:10E430004C91408331962F5F6F5F7F4F2B3079F780
:10E44000108208956F927F928F929F92AF92BF92A7
:10E45000CF92DF92EF92FF920F931F93CF93DF93B0
:10E46000CDB7DEB7C356D1090FB6F894DEBF0FBEE5
:10E47000CDBF5C018B016DB67EB67E0187E5E80EEF
:10E48000F11C44EF5FE0BE016F5F7F4FC5010E944A
:10E49000329618160CF0AFC08C858871803109F067
:10E4A0006CC08DB69EB6BE016F5F7F4FC7010E94E4
:10E4B0000C720115110521F0F8018081811191C0C4
:10E4C00021E081E090E0F70101900020E9F7319729
:10E4D000EE19FF09E80FF91F32968DB79EB78E1B14
:10E4E0009F0B0FB6F8949EBF0FBE8DBFEDB7FEB762
:10E4F00031966F01211102C0B80102C062EC76E0D2
:10E50000C6010F94041FB701C6010F94EE1E62EC02
:10E5100076E0C6010F94EE1E19A21CA221E0A7010D
:10E52000B501CE0181960E94A09881110AC00E9477
:10E530002A4EB70181ED9AE10E94134E8AE00E94B3
:10E54000E64D8BE1FE01B196DE01DC9601900D9265
:10E550008A95E1F7B601CE01CC960E942272CE01D7
:10E56000CC960E94A694CE0181960E94A6940FB6E6
:10E57000F8949EBE0FBE8DBE84CFCE0101960E9440
:10E58000A871882309F47DCFBE016F5F7F4F86E3BA
:10E5900090E10E940C720115110529F486E3C82E42
:10E5A00080E1D82E09C06801F60181916F018823AE
:10E5B000A9F30E94E64DF8CFF60181916F018823FF
:10E5C00019F00E94E64DF8CF80E20E94E64D6D8D75
:10E5D0007E8D8F8D98A14AE00E94824E0E94BC4F92
:10E5E00050CFF80101900020E9F73197CF01801B4F
:10E5F000910B20E068CF0FB6F8947EBE0FBE6DBEC3
:10E60000CD59DF4F0FB6F894DEBF0FBECDBFDF91FF
:10E61000CF911F910F91FF90EF90DF90CF90BF901F
:10E62000AF909F908F907F906F900895EF92FF92A0
:10E630000F931F93CF93DF93CDB7DEB7A0970FB69D
:10E64000F894DEBF0FBECDBF7C018B0144EF5FE0CD
:10E65000BE016F5F7F4FC7010E9432961816A4F467
:10E66000CE0101960E94A871882381F3BE016F5FDD
:10E670007F4F86E390E10E940C7266E370E1C8016F
:10E680000F94DB1E892B11F7A0960FB6F894DEBF0E
:10E690000FBECDBFDF91CF911F910F91FF90EF90F3
:10E6A00008950F931F93CF93DF93CDB7DEB76B978A
:10E6B0000FB6F894DEBF0FBECDBF8C0189E994E19F
:10E6C0000E9470938BE1E9E9F4E1DE01119601907B
:10E6D0000D928A95E1F7B801CE0101960E9416735A
:10E6E000CE0101960E94A6946B960FB6F894DEBFF9
:10E6F0000FBECDBFDF91CF911F910F910895DF9293
:10E70000EF92FF920F931F93CF93DF93CDB7DEB7B6
:10E7100027970FB6F894DEBF0FBECDBF2091241708
:10E7200023FF37C1F42EE62E8C010E94914D8823E1
:10E7300009F480C0FF2009F48BC080911B17882347
:10E7400051F00E94264E87EE9BE10E94F84D80E03A
:10E7500090E00E9416E28EE89BE09E838D838FE21C
:10E7600080938D0B81E08F83CE0105969A838983F8
:10E7700002969C838B83F12C9BE1D92E80911A17F2
:10E78000F81658F4DF9CB0011124645F794ECE0175
:10E7900001960E94576FF394F1CF8F818B3558F417
:10E7A0006BE574E1CE0101960E94576F8D819E81C9
:10E7B00001979E838D83ED81FE811082E0911B176E
:10E7C00084E0E89FF0011124E757F44F809120176F
:10E7D00090912117A0912217B091231780839183E4
:10E7E000A283B3830E942A4EB8018EEC9BE10E9463
:10E7F000134E60911B1789E6689FB001112463577F
:10E80000744F83EC9BE10E94134E4091201750916E
:10E81000211760912217709123178DEB9BE10E94C5
:10E82000EF4E8AE00E94E64D80911B178F5F809328
:10E830001B1726C0FF2039F00E942A4E8DEA9BE16B
:10E840000E94F84D1DC010921B1782E0F82E02C0E6
:10E85000FF24F3940E942A4E88EA9BE10E94F84D1F
:10E8600081E0F81609F492C084E99BE10E94F84D1A
:10E87000B80180EA9BE10E94134E8AE00E94E64DB7
:10E880000E942270B801CE0101960E947DE38C01A6
:10E89000009709F47EC069817A81EE2009F44DC0A9
:10E8A00021E0AC018BE594E10E94A0988823E9F176
:10E8B00080916C1490916D14A0916E14B0916F14AE
:10E8C00080931C1790931D17A0931E17B0931F17CA
:10E8D00010922017109221171092221710922317CE
:10E8E000B80186E89BE10E94134E40911C1750919D
:10E8F0001D1760911E1770911F178EE79BE10E94F4
:10E90000EF4E8AE00E94E64D8FE69BE10E94F84DB3
:10E91000C8010E9451738091F40F811102C0C80197
:10E9200002C084EF9FE060E02EC0B8018BE59BE160
:10E930000E94134E88E59BE10FC026E5AC018BE5F4
:10E9400094E10E94A09881110AC0B80184E49BE17F
:10E950000E94134E81E49BE10E94F84D1AC0809101
:10E960002417816080932417C8010E94517310926C
:10E97000E215B8018FE29BE10E94134E8AE00E94EB
:10E98000E64D60E0C8010E94D9FF03C08AE99BE11F
:10E990006DCF27960FB6F894DEBF0FBECDBFDF91C7
:10E9A000CF911F910F91FF90EF90DF900895CF923C
:10E9B000DF92EF92FF92CF936B017C01C42F809185
:10E9C000E90F9091EA0FA091EB0FB091EC0F8C152D
:10E9D0009D05AE05BF05D1F00E942A94811102C0A9
:10E9E00080E018C029EE3DE0B701A6018091F20F4A
:10E9F0009091F30F0E94AC94882391F3C092E90F99
:10EA0000D092EA0FE092EB0FF092EC0F81E0C1118F
:10EA10008093F10FCF91FF90EF90DF90CF9008950A
:10EA20004F925F926F927F928F929F92AF92BF921E
:10EA3000CF92DF92EF92FF920F931F93CF93DF93CA
:10EA4000EC01423051056105710510F480E069C0A8
:10EA500089859A85AB85BC850196A11DB11D84175A
:10EA60009507A607B70790F38F89803149F4852E63
:10EA7000962EA72EBB248B899C89AD89BE890FC099
:10EA8000803221F78B889C88AD88BE88DB01CA0163
:10EA9000E7E0B695A79597958795EA95D1F7880E03
:10EAA000991EAA1EBB1E280139016A017B0141E0A3
:10EAB000C501B4010E94D774882341F29F89903127
:10EAC00061F4DD24EE24FF249601220F331FF901A7
:10EAD000E751F24F5182408211C0E894C7F8DD241B
:10EAE000EE24FF249601220F331F220F331FF9015A
:10EAF000E751F24F40825182628273829A8992304A
:10EB000080F04D815E816F817885840E951EA61EF2
:10EB1000B71E8092ED0F9092EE0FA092EF0FB09281
:10EB2000F00FDF91CF911F910F91FF90EF90DF9049
:10EB3000CF90BF90AF909F908F907F906F905F909D
:10EB40004F900895CF92DF92EF92FF920F931F9311
:10EB5000CF93DF93FC0181859285A385B4850196CF
:10EB6000A11DB11D84179507A607B70710F480E013
:10EB700061C08789803149F4BB27A72F962F852F45
:10EB8000C388D488E588F6880FC0803281F78389EE
:10EB90009489A589B6896A017B01C7E0F694E79458
:10EBA000D794C794CA95D1F78C0D9D1DAE1DBF1D7E
:10EBB000E9016A017B018F014091E90F5091EA0F51
:10EBC0006091EB0F7091EC0F84179507A607B707BC
:10EBD00039F040E0BC01CD010E94D774882339F29E
:10EBE000F8018789803179F4B701A6015527662796
:10EBF0007727440F551FFA01E751F24F8081918129
:10EC0000A0E0B0E012C0B701A6014F7755276627F4
:10EC10007727440F551F440F551FFA01E751F24F54
:10EC200080819181A281B381BF7088839983AA83F7
:10EC3000BB8381E0DF91CF911F910F91FF90EF9007
:10EC4000DF90CF9008954F925F926F927F92AF9234
:10EC5000BF92CF92DF92EF92FF920F931F93CF93C9
:10EC6000DF9300D01F92CDB7DEB78C0149835A8362
:10EC70006B837C835901C12CD12C7601412C82E01D
:10EC8000582E612C712C49815A816B817C819E01A7
:10EC90002F5F3F4FC8010E94A275882341F1D30125
:10ECA000C201F801058404C0880F991FAA1FBB1F69
:10ECB0000A94D2F7C80ED91EEA1EFB1E49815A815A
:10ECC0006B817C818789803139F481E0483F5F4FD7
:10ECD0006105710538F4D7CF81E0483F5F4F6F4F32
:10ECE0007F4088F2F501C082D182E282F3820F90E8
:10ECF0000F900F900F90DF91CF911F910F91FF9088
:10ED0000EF90DF90CF90BF90AF907F906F905F902B
:10ED10004F9008959F92AF92BF92CF92DF92EF9261
:10ED2000FF920F931F93CF93DF9300D01F921F92F8
:10ED3000CDB7DEB7E3E6FEE10027BB27462F572F0E
:10ED4000A82FAA2341F4A52F542FB85FAA2319F4A2
:10ED5000A52F5527B85FA03138F45295A295452FBD
:10ED60004F70507FA42BBC5FA03428F4550FAA1F0E
:10ED7000550FAA1FBE5FA03818F4550FAA1FB395F0
:10ED8000550FAA1FEA0FF01F449151E0AA27B8506F
:10ED900081F1C8F0B0FF02C0440F551FB1FF04C09D
:10EDA000440F551F440F551FB2FF06C052954295A0
:10EDB000142F1F70407F512BB3FF1BC0A52F542F62
:10EDC00044270C94F976B195B0FF02C0559547954C
:10EDD000B1FF04C05595479555954795B2FF05C0BD
:10EDE0005295407F4295452B5F70B3FF02C0452F7F
:10EDF0005527DD24CC24BB24B2E0649FD018C10881
:10EE0000B00AB00B749FC018B108B00B849FB01843
:10EE1000B109659FC018B108B00B759FB018B10952
:10EE2000859FB0196A9FB018B1097A9FB0194D9D9E
:10EE3000A12C99249927332722275D9DA00C911C92
:10EE4000901F301F201FAD9D900C911D301F201F63
:10EE50004C9DA00C911C901F301F201F5C9D900C9E
:10EE6000911D301F201FAC9D900D311D201F4B9D0B
:10EE7000900C911D301F201F5B9D900D311D201F98
:10EE8000AB9D300D211D4B9F900D311D201F5B9FB1
:10EE9000300D211DAB9F200DB1E0BB24CC24DD241F
:10EEA000699FD018C108B00AB00B799FC018B1088B
:10EEB000B00B899FB018B109639FC018B108B00B9F
:10EEC000739FB018B109839FB019629FB018B10940
:10EED000729FB019D61AC70AB80A20F0B1E09B0F8A
:10EEE000301F201F1124692F70E0732BCB01A0E08D
:10EEF000B0E0BC01CD01822B0F900F900F900F90CE
:10EF00000F90DF91CF911F910F91FF90EF90DF90C5
:10EF1000CF90BF90AF909F9008952F923F924F92C5
:10EF20005F926F927F928F929F92AF92BF92CF9299
:10EF3000DF92EF92FF920F931F93CF93DF93CDB7A2
:10EF4000DEB764970FB6F894DEBF0FBECDBF7A8BE5
:10EF5000698BDC018D909D90AD90BC9013971496B9
:10EF60002D913D914D915C9117972D833E834F8359
:10EF7000588720E030E040EA51E4C501B4010F9425
:10EF8000A51B21EC3FE04CE75CE30F9408150F94C0
:10EF9000121D643014F063E002C067FD60E0E62EED
:10EFA000660FFF08F701EE0FFF1FEE0FFF1FE9507E
:10EFB000FA4E40805180628073801701BFEF2B1A98
:10EFC0003B0A20E030E040EA51E46D817E818F8190
:10EFD00098850F94A51B21EC3FE04CE75CE30F9470
:10EFE00008150F94121D643014F063E002C067FD31
:10EFF00060E0062F660F110BF801EE0FFF1FEE0FFA
:10F00000FF1FE950FA4E20813181428153812983CB
:10F010003A834B835C83A8014F5F5F4F5C8B4B8BC4
:10F02000A5E0AE9DC001AF9D900D11249A87898700
:10F03000FC01E00FF11FEE0FFF1FEE0FFF1FEE5E52
:10F04000F34FC080D180E280F380F101EE0FFF1F0B
:10F05000EE0FFF1FE950FA4EA3019201608171810A
:10F06000828193810F94A51B6B877C878D879E87F8
:10F07000A3019201C501B4010F94A51B2B013C0112
:10F0800025E0229DF001239DF00D1124F88BEF87E0
:10F09000E00FF11FEE0FFF1FEE0FFF1FEE5EF34FAD
:10F0A000A701960160817181828193810F94A51BD4
:10F0B0002B853C854D855E850F94A01CA301920194
:10F0C0000F940815A70196010F94A61B6B017C01F4
:10F0D000E985FA854B895C89E40FF51FEE0FFF1F68
:10F0E000EE0FFF1FEE5EF34F80809180A280B38011
:10F0F000EF85F889E40FF51FEE0FFF1FEE0FFF1FDE
:10F10000EE5EF34FA501940160817181828193814C
:10F110000F94A51B2B853C854D855E850F94A01C07
:10F12000A30192010F940815A50194010F94A61B49
:10F13000A70196010F94A51B4B015C01EB89FC898B
:10F14000EE0FFF1FEE0FFF1FE950FA4E29813A81A3
:10F150004B815C8160817181828193810F94A51BB9
:10F160009B01AC01C501B4010F94A01C4B015C01D3
:10F1700029813A814B815C816D817E818F81988567
:10F180000F94A51B9B01AC01C501B4010F94081598
:10F19000A70196010F94A61BA989BA892D913D91CB
:10F1A0004D915C910F94081520910E0C30910F0C2D
:10F1B0004091100C5091110C0F94A61B64960FB641
:10F1C000F894DEBF0FBECDBFDF91CF911F910F919D
:10F1D000FF90EF90DF90CF90BF90AF909F908F9077
:10F1E0007F906F905F904F903F902F9008958F92F7
:10F1F0009F92AF92BF92CF92DF92EF92FF92CF9306
:10F20000DF93EC018090E50D9090E60DA090E70D66
:10F21000B090E80D20E030E0A901C501B4010F94E1
:10F22000A214882309F44AC0C880D980EA80FB80F0
:10F23000A7019601C501B4010F94A21418160CF091
:10F2400042C02091DC0D3091DD0D4091DE0D5091DA
:10F25000DF0DC701B6010F94A214882331F1C092CB
:10F26000DC0DD092DD0DE092DE0DF092DF0D2091ED
:10F27000E00D3091E10D4091E20D5091E30D688178
:10F2800079818A819B810F9408159B01AC0160E014
:10F2900070E080E89FE30F94A51B609321027093B8
:10F2A00022028093230290932402609121027091A4
:10F2B0002202809123029091240208C060E070E055
:10F2C00080E89FE303C060E070E0CB01DF91CF9165
:10F2D000FF90EF90DF90CF90BF90AF909F908F9076
:10F2E0000895CF93DF938091D2149091D314891B0A
:10F2F0008F708F3021F480E00E94E34FF4CF809133
:10F30000D2148F5F8F70A091D21494E69A9FD0018F
:10F310001124FD01EE5EF74EEF01292F19922A9577
:10F32000E9F728E02083A95DB74E20E1E8EFF4E19A
:10F3300001900D922A95E1F73091D2142091D314C7
:10F34000321302C09093CF148093D21480916F0037
:10F35000826080936F00DF91CF910895CF92DF920A
:10F36000EF92FF920F931F93CF93DF93CCEEDCE0ED
:10F370000BE81CE0C12CD12C7601C39469917991E2
:10F38000899199910F94A714288939894A895B89B1
:10F390000F9408150F94191DF801619371938193CF
:10F3A00091938F01C616D706E806F90610F46B0193
:10F3B0007C01FCE0CC3FDF0709F76FEF7FEFCB016B
:10F3C000A70196010F94F81A20939B0C30939C0C84
:10F3D00040939D0C50939E0C23EF34E045E35FE394
:10F3E0006091870C7091880C8091890C90918A0CA7
:10F3F0000F9408156B017C016091F80C7091F90C69
:10F400008091FA0C9091FB0C0F94A7149B01AC0116
:10F41000C701B6010F94081529E732E84AE550E420
:10F420000F9408150F94541E60939F0C7093A00CBA
:10F430008093A10C9093A20CDF91CF911F910F911B
:10F44000FF90EF90DF90CF9008950F931F93CF938D
:10F45000DF9300E01DE0CBEBD8E0F8012191319182
:10F46000419151918F0160E070E080E89FE30F943B
:10F47000A01C6993799389939993F8E0CB3CDF07BB
:10F4800061F70E9497CEDF91CF911F910F910C945D
:10F49000AE799091D2148091D314981306C08091C4
:10F4A000EA0C9091EB0C892B21F080E00E94E34F55
:10F4B000F0CF0895CF92DF92EF92FF92FC01C080CF
:10F4C000D180E280F38020910C0D30910D0D4091A0
:10F4D0000E0D50910F0DC701B6010F9408150F9432
:10F4E000131E609304157093051580930615909371
:10F4F0000715C092F414D092F514E092F614F0922D
:10F50000F7149091D2148091D314981731F0FF9092
:10F51000EF90DF90CF900C9471790E94497A80919E
:10F520006F00982F927081FF05C080916F008D7FD2
:10F5300080936F0040910415509105156091061558
:10F54000709107154093C0175093C1176093C2176D
:10F550007093C317992329F080916F008260809384
:10F560006F00FF90EF90DF90CF9008954F925F92E1
:10F570006F927F928F929F92AF92BF92CF92DF92C3
:10F58000EF92FF920F931F93CF93DF93EC018B01C8
:10F590007A016901F90180819181A281B381FA0127
:10F5A0004081518162817381F80180809180A280C5
:10F5B000B380488059806A807B804092E8145092E2
:10F5C000E9146092EA147092EB148092EC14909219
:10F5D000ED14A092EE14B092EF144093F0145093F7
:10F5E000F1146093F2147093F3148093F4149093D5
:10F5F000F514A093F614B093F71420910C0D3091EC
:10F600000D0D40910E0D50910F0DF601608171812D
:10F61000828193810F9408150F94131E4B015C0196
:10F620002091080D3091090D40910A0D50910B0D5C
:10F63000F70160817181828193810F9408150F9485
:10F64000131E6B017C012091040D3091050D40913A
:10F65000060D5091070DF8016081718182819381BF
:10F660000F9408150F94131E2B013C012091000DDF
:10F670003091010D4091020D5091030D6881798107
:10F680008A819B810F9408150F94131E6093F814C0
:10F690007093F9148093FA149093FB144092FC1425
:10F6A0005092FD146092FE147092FF14C0920015E7
:10F6B000D0920115E0920215F09203158092041584
:10F6C00090920515A0920615B09207159091D2144C
:10F6D0008091D314981791F0DF91CF911F910F91E2
:10F6E000FF90EF90DF90CF90BF90AF909F908F9062
:10F6F0007F906F905F904F900C9471790E94497A3F
:10F7000080916F00982F927081FF05C080916F00EB
:10F710008D7F80936F00409100155091011560918D
:10F720000215709103150091FC141091FD142091A5
:10F73000FE143091FF14C090F814D090F914E090AA
:10F74000FA14F090FB14C092B417D092B517E0925F
:10F75000B617F092B7170093B8171093B917209304
:10F76000BA173093BB174093BC175093BD176093E3
:10F77000BE177093BF174091041550910515609105
:10F780000615709107154093C0175093C1176093E9
:10F79000C2177093C317992329F080916F0082607C
:10F7A00080936F00DF91CF911F910F91FF90EF90A9
:10F7B000DF90CF90BF90AF909F908F907F906F9091
:10F7C0005F904F900895CF93DF93C82F0E9478FCED
:10F7D00024E0C29FE0011124C554D74F0F94A9140F
:10F7E000288139814A815B810F940815DF91CF917F
:10F7F00008959091D2148091D314981306C08091EB
:10F80000EA0C9091EB0C892B21F080E00E94E34FF1
:10F81000F0CF5F9A80917B138E7F80937B138A9ABF
:10F8200080917B138D7F80937B138091080180955D
:10F8300081708093060180917B138B7F80937B1373
:10F840000C944A4DCF93DF9390916F00292F227033
:10F8500091FF05C090916F009D7F90936F0094E0A1
:10F86000899FA0011124FA01E855F84E6081718149
:10F8700082819381222329F020916F0022602093BE
:10F880006F00EA01C554D74F0F94A914288139811C
:10F890004A815B810F940815DF91CF910895809183
:10F8A0006F00982F927081FF05C080916F008D7F4F
:10F8B00080936F008091D3148093D2148093D114DD
:10F8C0008093D01484E68093CF1428EE33E03093F5
:10F8D000EB0C2093EA0C992329F080916F00826051
:10F8E00080936F0081E08093A71708950F931F9373
:10F8F000CF93DF9300D01F92CDB7DEB72091E40DF8
:10F900002223E1F08C0108960E94F77869837A83BC
:10F910008B839C83BE016F5F7F4FC8010E948D77F0
:10F920009B01AC01F80160857185828593850F94F8
:10F93000A51BF80160877187828793870F900F90CE
:10F940000F900F90DF91CF911F910F9108950F931A
:10F950001F93CF93DF9300D01F92CDB7DEB72091D6
:10F96000E40D2223E1F08C0108960E94F778698368
:10F970007A838B839C83BE016F5F7F4FC8010E9497
:10F980008D779B01AC01F801608571858285938537
:10F990000F94A61BF80160877187828793870F9069
:10F9A0000F900F900F90DF91CF911F910F910895BD
:10F9B000AF92BF92CF92DF92EF920F931F93CF93AC
:10F9C000DF93CDB7DEB764970FB6F894DEBF0FBEF6
:10F9D000CDBFA98ABA8ACB8ADC8AFC018081918159
:10F9E000A281B38189839A83AB83BC83FB0180812D
:10F9F0009181A281B3818D839E83AF83B887FA0101
:10FA000080819181A281B38189879A87AB87BC87E6
:10FA1000F90180819181A281B3818D879E87AF8713
:10FA2000B88BCE0101960E94A77C8091EA0C909140
:10FA3000EB0C892B81F4CE0141966C019E01235F72
:10FA40003F4FAE01475F5F4FBE016B5F7F4F4097F7
:10FA50000E947D8001C080E064960FB6F894DEBFFE
:10FA60000FBECDBFDF91CF911F910F91EF90DF902F
:10FA7000CF90BF90AF9008957F928F929F92AF9258
:10FA8000BF92CF92DF92EF92FF920F931F93CF938B
:10FA9000DF937090760CC7E7DCE095E2C92E92E028
:10FAA000D92E25E3E22E22E0F22E0FE71CE077208C
:10FAB00059F1F80180809180A280B38020E030E08D
:10FAC000A901C501B4010F94A2148823E9F020E034
:10FAD00030E040E05FE3C501B4010F9408159B01DD
:10FAE000AC010F9408152BED3FE049E450E40F946E
:10FAF00008159B01AC0160E070E080E89FE30F9483
:10FB0000A01C4B015C0106C0812C912C80E8A82E22
:10FB10008FE3B82E89929992A992B992F6016191D8
:10FB200071916F01072E000C880B990B0F94A9148B
:10FB30002AE037ED43E25CE30F940815A501940138
:10FB40000F940815F70161937193819391937F014D
:10FB50000C5F1F4FFCE0CF37DF0709F0A8CFDF9124
:10FB6000CF911F910F91FF90EF90DF90CF90BF90BA
:10FB7000AF909F908F907F9008952F923F924F92D9
:10FB80005F926F927F928F929F92AF92BF92CF922D
:10FB9000DF92EF92FF920F931F93CF93DF93CDB736
:10FBA000DEB76C970FB6F894DEBF0FBECDBF8C01E9
:10FBB0005B015A834983FC01EE5AFF4F208131815A
:10FBC000428153812D873E874F87588BCA01B901E7
:10FBD0000F94A7146B017C01D5012D913D914D919E
:10FBE0005C910F9408150F94841C0F94191D698B58
:10FBF0007A8B8B8B9C8BE981FA81208131814281C8
:10FC00005381C701B6010F9408150F94841C0F94FB
:10FC1000191D6D8B7E8B8F8B988F29893A894B8923
:10FC20005C89283731054105510540F448E750E02B
:10FC300060E070E0498B5A8B6B8B7C8B6D897E8981
:10FC40008F89988D683771058105910540F488E7A3
:10FC500090E0A0E0B0E08D8B9E8BAF8BB88FF80169
:10FC6000E25AFF4F20813181428153812D833E83AF
:10FC70004F835887CA01B9010F94A9142B013C0185
:10FC800069897A898B899C890F94A71469877A87F7
:10FC90008B879C8720E030E0A901C301B2010F945B
:10FCA000A214882329F1A7019601C701B6010F9478
:10FCB00008154B015C0129853A854B855C85CA0195
:10FCC000B9010F9408159B01AC01C501B4010F9453
:10FCD000A51B4B015C01A3019201C301B2010F946A
:10FCE000A61B9B01AC01C501B4010F94A01C03C06D
:10FCF00060E070E0CB010F94841C0F94191D6983A0
:10FD00007A838B839C836D817E818F81988590958A
:10FD10008095709561957F4F8F4F9F4F0F94A914D9
:10FD20004B015C016D897E898F89988D0F94A71492
:10FD30006D837E838F83988720E030E0A901C50121
:10FD4000B4010F94A214882349F12D813E814F8183
:10FD50005885CA01B9010F940815698F7A8F8B8F66
:10FD60009C8FA7019601C701B6010F9408159B014E
:10FD7000AC01698D7A8D8B8D9C8D0F94A51B6B01C9
:10FD80007C01A5019401C501B4010F94A61B9B0140
:10FD9000AC01C701B6010F94A01C03C060E070E085
:10FDA000CB010F94481DD80195968D909D90AD90F4
:10FDB000BC9098977501640129813A814B815C81DF
:10FDC000C21AD30AE40AF50A0F94191DC61AD70AF3
:10FDD000E80AF90AF7FEA1C020E030E0A901C3015A
:10FDE000B2010F94A214882309F443C0C501B401E1
:10FDF0000F94A7146B017C01A3019201C301B2010E
:10FE00000F94A61B9B01AC01C701B6010F94081506
:10FE10006B017C0129853A854B855C85CA01B90156
:10FE20000F9408159B01AC01C701B6010F94A51BE7
:10FE30006B017C012D813E814F815885CA01B9013A
:10FE40000F9408159B01AC01C701B6010F94A61BC6
:10FE50006B017C0120E030E040E850E4C301B201D6
:10FE60000F9408159B01AC01C701B6010F94A01CAB
:10FE700003C060E070E0CB010F94841C7B018D8394
:10FE8000998320E030E0A9010F94061E181624F093
:10FE9000E12CF12C1D821982B7018D8199810F947B
:10FEA000191D69837A838B839C8386169706A8061F
:10FEB000B90620F489829A82AB82BC82A3019201A6
:10FEC000C301B2010F94A61B6B017C0169817A8189
:10FED0008B819C810F94A7149B01AC01C701B601D3
:10FEE0000F9408156B017C0129853A854B855C854B
:10FEF000CA01B9010F9408159B01AC01C701B601F5
:10FF00000F94A61B0F94541E0F94191D6D877E87A6
:10FF10008F87988BC12CD12C76016D857E858F853E
:10FF2000988929893A894B895C89621B730B840BF8
:10FF3000950B0F94A714A30192010F94A01C20E02D
:10FF400034E244EF59E40F9408150F94191D4B0146
:10FF50005C016D857E858F8598892D893E894F89C5
:10FF6000588D621B730B840B950B0F94A714A30180
:10FF700092010F94A01C20E034E244EF59E40F9466
:10FF800008150F94191D2B013C013FE683169104BF
:10FF9000A104B10480F4F401EE0FFF1FEE0FFF1F68
:10FFA000E955F34E85919591A591B4918D83292EB4
:10FFB0003A2EB98708C0C501B4010E948A766D83C4
:10FFC000272E382E99874FE6441651046104710498
:10FFD00070F4F201EE0FFF1FEE0FFF1FE955F34E15
:10FFE00045915591659174919A01CB0105C0C3016A
:10FFF000B2010E948A769B0149815A816B817C8182
:020000021000EC
:10000000D8019A964D935D936D937C939D974C0D7B
:100010005D1D6E1D7F1DF80146A757A760AB71AB34
:10002000EA5AFF4F49895A896B897C8940835183F9
:1000300062837383D6968D929D92AD92BC92D9972E
:10004000F80142AE53AE64AE75AEFE964D8140836C
:10005000218232825985538334962083318382836F
:1000600093836D857E858F859889D2966D937D93D8
:100070008D939C93D59778962D893E894F89588D7D
:1000800020833183428353836C960FB6F894DEBF8E
:100090000FBECDBFDF91CF911F910F91FF90EF90D9
:1000A000DF90CF90BF90AF909F908F907F906F9098
:1000B0005F904F903F902F900895CF93DF9324E06F
:1000C000829FC0011124EC01CA50D44FFC01E559B4
:1000D000F64FDC01AE5FB34F2D913D914D915C9198
:1000E00060817181828193810F94A61B68837983DB
:1000F0008A839B83DF91CF9108952F923F924F92F5
:100100005F926F927F928F929F92AF92BF92CF92A7
:10011000DF92EF92FF920F931F93CF93DF93CDB7B0
:10012000DEB7CD57D1090FB6F894DEBF0FBECDBFF5
:100130003B014A015901EBA66F96DFAECEAE6F9739
:10014000DC012D913D914D915C91A5962CAF3DAF79
:100150004EAF5FAFA5972091000D3091010D4091FA
:10016000020D5091030DA5966CAD7DAD8EAD9FAD8A
:10017000A5970F9408150F94131EE5966CAF7DAFED
:100180008EAF9FAFE597D3012D913D914D915C913D
:10019000A9962CAF3DAF4EAF5FAFA9972091040D4C
:1001A0003091050D4091060D5091070DA9966CAD4B
:1001B0007DAD8EAD9FADA9970F9408150F94131EBA
:1001C000E9966CAF7DAF8EAF9FAFE997D4012D91CB
:1001D0003D914D915C91AD962CAF3DAF4EAF5FAF71
:1001E000AD972091080D3091090D40910A0D509165
:1001F0000B0DAD966CAD7DAD8EAD9FADAD970F94F3
:1002000008150F94131EED966CAF7DAF8EAF9FAFA8
:10021000ED97D5012D913D914D915C9169962CAF53
:100220003DAF4EAF5FAF699720910C0D30910D0D32
:1002300040910E0D50910F0D69966CAD7DAD8EAD58
:100240009FAD69970F9408150F94131E6D966CAFB0
:100250007DAF8EAF9FAF6D9780913D0D83FF1CC02A
:100260006D962CAD3DAD4EAD5FAD6D9720930415F1
:1002700030930515409306155093071569968CAD7C
:100280009DADAEADBFAD69978093F4149093F51416
:10029000A093F614B093F7148091EA0C9091EB0CB4
:1002A000892B09F079C3D801BC91BBABF801F1816E
:1002B000FFAFD8011296BC912496BFAF2497F801E6
:1002C000F3812A96FFAF2A978091D2149091D3148C
:1002D000891B8F708F3021F480E00E94E34FF4CFB0
:1002E0002091D214EE962FAFEE978091D214282E43
:1002F000312C34E6839FC0011124AC014E5E574E71
:1003000029965FAF4EAF29978091F8149091F91418
:10031000A091FA14B091FB14E5968CAC9DACAEACF8
:10032000BFACE597881A990AAA0ABB0A8091FC1407
:100330009091FD14A091FE14B091FF14E9964CAC7D
:100340005DAC6EAC7FACE997481A590A6A0A7B0A21
:100350008091001590910115A0910215B09103159F
:10036000ED962CAD3DAD4EAD5FADED97281B390B35
:100370004A0B5B0B2FAB38AF49AF5AAF80910415D6
:1003800090910515A0910615B09107156D962CADAD
:100390003DAD4EAD5FAD6D97281B390B4A0B5B0B26
:1003A0002BA33CA34DA35EA3232B242B252B09F4C5
:1003B0009BC080913C0D81113CC020E030E0A90140
:1003C0006091290970912A0980912B0990912C093B
:1003D0000F94A61B0F94121D2091650230916602A6
:1003E0006217730734F56D968CAD9DADAEADBFADA4
:1003F0006D978093041590930515A0930615B093FF
:10040000071569962CAD3DAD4EAD5FAD6997209354
:10041000F4143093F5144093F6145093F7140E949B
:100420002A4E82E89FE10E94F84D1BA21CA21DA249
:100430001EA24BA534E0439F800111240B5C1D4F8D
:100440006BA17CA18DA19EA10F94A914D8012D911F
:100450003D914D915C910F9408156B017C0120E05A
:1004600030E0A9010F94061E87FF04C0F7FAF0944C
:10047000F7F8F09420E030E04AEF53E460910C0D7F
:1004800070910D0D80910E0D90910F0D0F94081528
:10049000A70196010F94A21487FF26C06D962CAD7C
:1004A0003DAD4EAD5FAD6D972093041530930515AE
:1004B000409306155093071569968CAD9DADAEAD72
:1004C000BFAD69978093F4149093F514A093F6143C
:1004D000B093F7140E942A4E83E69FE10E94F84DE4
:1004E0001BA21CA21DA21EA2D501C4018827B7FD14
:1004F00083959927AA27BB278FA377FE03C0E82FF0
:10050000E260EFA32FA938AD49AD5AAD57FF03C044
:100510003FA134603FA38BA19CA1ADA1BEA1B7FFB9
:1005200003C09FA198609FA3BBA5A4E0BA9F8001D0
:1005300011240B5C1D4F6BA17CA18DA19EA10F947A
:10054000A914F80120813181428153810F9408154B
:100550006B017C0120E030E0A9010F94061E87FFAB
:1005600004C0C701B601905802C0C701B60120E01F
:1005700030E040E05FE30F94A61B0F94191D6FA7B6
:1005800078AB89AB9AAB84E6829DF001839DF00D38
:100590001124EE5EF74E1082EA5BFF4F2FA12083FD
:1005A0008FA998ADA9ADBAAD61968CAF9DAFAEAF36
:1005B000BFAF6197B7FF0DC0B095A095909581959D
:1005C0009F4FAF4FBF4F61968CAF9DAFAEAFBFAFE8
:1005D00061974BAE5CAE6DAE7EAE77FE0BC0222750
:1005E0003327A90124193509460957092BAF3CAF18
:1005F0004DAF5EAF8FA298A6A9A6BAA6B7FE0BC054
:1006000088279927DC0188199909AA09BB098FA3B2
:1006100098A7A9A7BAA72FA138A549A55AA5299691
:10062000AEADBFAD299755962D933D934D935C93F9
:1006300058972BAD3CAD4DAD5EAD59962D933D9386
:100640004D935C935C9761962CAD3DAD4EAD5FAD27
:1006500061975D962D933D934D935C939097C50163
:10066000B4010F94A9142091BB083091BC084091AB
:10067000BD085091BE080F94081565966CAF7DAF0C
:100680008EAF9FAF6597698B7A8B8B8B9C8BC301E9
:10069000B2010F94A9142091BF083091C008409175
:1006A000C1085091C2080F9408152B013C016D8BB5
:1006B0007E8B8F8B988F6FA978AD89AD9AAD0F9493
:1006C000A9142091C3083091C4084091C5085091E5
:1006D000C6080F9408154B015C01698F7A8F8B8FC8
:1006E0009C8F2091C7083091C8084091C90850914B
:1006F000CA08C701B6010F9408156B017C016D8F04
:100700007E8F8F8F98A32FA138A549A55AA5263093
:10071000310541055105BCF58BAD9CADADADBEAD10
:100720000697A105B1057CF561962CAD3DAD4EADAA
:100730005FAD6197263031054105510524F520E074
:1007400030E0A901C701B6010F94061E87FF04C05F
:10075000F7FAF094F7F8F09484E6829D8001839D87
:10076000100D11240E5E174E20E030E0A901C701E4
:10077000B6010F94A61BD8011D966D937D938D93A2
:100780009C93509752C06F96EEADFFAD6F97C080AF
:10079000D180E280F38020E030E0A901C701B601FA
:1007A0000F94A214882369F084E6829DF001839D52
:1007B000F00D1124EE5EF74EC586D686E786F08AE8
:1007C00034C065962CAD3DAD4EAD5FAD6597CA01A9
:1007D000B9010F9408156B017C01A3019201C301BB
:1007E000B2010F9408159B01AC01C701B6010F942B
:1007F000A61B6B017C01A5019401C501B4010F94F6
:1008000008159B01AC01C701B6010F94A61B0F94FC
:10081000541E24E6229DF001239DF00D1124EE5E6E
:10082000F74E658776878787908B84E6829DF001F7
:10083000839DF00D1124EE5EF74E2FA538A949A92E
:100840005AA921A332A343A354A361968CAD9DADB5
:10085000AEADBFAD61972BAD3CAD4DAD5EAD82177A
:100860009307A407B50710F4DA01C9012FA138A531
:1008700049A55AA582179307A407B50710F4DA0112
:10088000C9012FA538A949A95AA982179307A40716
:10089000B50710F4DA01C90124E6229DF001239D79
:1008A000F00D1124EE5EF74E85A396A3A7A3B0A783
:1008B0000697A105B10510F40C949890DF01AE598C
:1008C000BF4F80913A0D8C93119680913B0D8C9384
:1008D0003BA531A78FA198A5A9A5BAA5892B8A2BDD
:1008E0008B2B09F05F9884E6829DF001839DF00DCB
:1008F0001124EE5EF74E818D928DA38DB48D892BE0
:100900008A2B8B2B09F08A9884E6829DF001839DC7
:10091000F00D1124EE5EF74E858D968DA78DB0A15A
:10092000892B8A2B8B2B29F0809108018170809371
:1009300006012FA538A949A95AA9232B242B252B19
:1009400071F18091BB0C882319F081508093BB0C0E
:100950008091BC0C882389F081508093BC0C3BA50E
:10096000332319F0313071F023C0811101C0479A4F
:10097000129880E28093BB0C1BC0FBA5FF23B9F348
:10098000F130B1F48091BB0C811101C0129A4798EB
:1009900080E28093BC0C0CC080E00C941791E09036
:1009A000300DF090310D0091320D1091330D08C0D3
:1009B000E0902C0DF0902D0D00912E0D10912F0D2B
:1009C0009701A8016BA97FAD24968FAD24972A9635
:1009D0009FAD2A970F94A21487FF08C0EBAAFFAE21
:1009E00024960FAF24972A961FAF2A9784E6829DFC
:1009F000F001839DF00D1124EE5EF74E4584568480
:100A000067847088A301920160E070E080E89FE352
:100A10000F94A01C6BA77CA78DA79EA72BA93FAD09
:100A200024964FAD24972A965FAD2A970F94081508
:100A30006B017C018091D2149091D014891B8F702E
:100A40008FAFA701960160E074E284E799E40F9408
:100A5000A01C0F94131E4B015C018FAD8250863099
:100A6000B0F58091FC0C9091FD0CA091FE0CB09122
:100A7000FF0C88169906AA06BB0648F5881999093D
:100A8000AA09BB09BC01CD01660F771F881F991FFA
:100A90004FAD042F10E020E030E0A90198010F9441
:100AA000F81ACA01B9010F94A7140F94131E680D08
:100AB000791D8A1D9B1D0F94A7149B01AC0160E05A
:100AC00074E284E799E40F94A01C6B017C01A701F8
:100AD0009601C301B2010F9408159B01AC010F945C
:100AE00008152D966CAF7DAF8EAF9FAF2D9784E626
:100AF000829D8001839D100D11240E5E174E2D9650
:100B00008CAD9DADAEADBFAD2D97F80181839283C5
:100B1000A383B48325A136A147A150A52FA338A74D
:100B200049A75AA7CA01B9010F94A7146FAB78AFB0
:100B300089AF9AAF9B01AC01C701B6010F940815AC
:100B40000F94841C0F94191D61966CAF7DAF8EAF0E
:100B50009FAF6197F801EE5AFF4F608371838283E4
:100B60009383FE0171962596FFAFEEAF259720E1A6
:100B70003DE063963FAF2EAF6397AE014F5D5F4F91
:100B80005AA349A31BAE1BAA00E81FE32596AEADEE
:100B9000BFAD25972D913D914D915D912596BFAFAC
:100BA000AEAF2597C701B6010F9408154B015C0144
:100BB00020E030E0A9010F94061E87FF04C0B7FAB9
:100BC000B094B7F8B0946396EEADFFAD63974190E3
:100BD0005190619071906396FFAFEEAF6397A5015E
:100BE0009401C301B2010F94A21487FF12C0A501A2
:100BF0009401C301B2010F94A01C5B014C012BAD09
:100C00003BA9A8010F94A21487FF03C0ABAEBBAAF7
:100C1000840125962EAD3FAD259749A15AA12417F1
:100C2000350709F0B3CF20E030E040E85FE36BAD7B
:100C30007BA9C8010F94A21487FF39C024E6229D26
:100C4000C001239D900D1124DC01AE5EB74E7D01E5
:100C50006D01B2E5CB0ED11C61966CAD7DAD8EAD54
:100C60009FAD61970F94A7142BAD3BA9A8010F94DA
:100C700008150F94191DF601608371838283938395
:100C80002BAD3BA9A8016BAD7BA9C8010F9408153A
:100C90002D962CAD3DAD4EAD5FAD2D970F94081543
:100CA000D70111966D937D938D939C9314972FA9E3
:100CB00038AD49AD5AAD6BA57CA58DA59EA50F9409
:100CC00008156BAB7CAB8DAB9EAB84E6829D80013F
:100CD000839D100D11240E5E174ED80155962D914F
:100CE0003D914D915C9158972BAF3CAF4DAF5EAFAE
:100CF000232B242B252B61F559968D919D910D90D9
:100D0000BC91A02D892B8A2B8B2B11F5F801858D99
:100D1000968DA78DB0A1892B8A2B8B2BC9F420919E
:100D2000240D3091250D4091260D5091270D6BA972
:100D30007CA98DA99EA90F9408150F94841C0F946B
:100D4000191D2B013C01F801E95BFF4F1082E7C23E
:100D50002FA538A949A95AA9232B242B252B49F0C3
:100D60002091200D3091210D4091220D5091230DA5
:100D700008C02091280D3091290D40912A0D5091E5
:100D80002B0D6BA97CA98DA99EA90F9408150F9412
:100D9000841C0F94191D2B013C018FA598A9A9A9AA
:100DA000BAA9892B8A2B8B2BE9F0E091CB0D94E02B
:100DB000E99FF0011124ED55F34F20E030E0A90147
:100DC00060817181828193810F94A214882351F0F4
:100DD00081E02BA13CA14DA15EA1121613061406C1
:100DE00015060CF080E094E6929D8001939D100D15
:100DF00011240E5E174EA801495B5F4F5CA34BA305
:100E0000DA018C93882309F4B8C02091E81430915A
:100E1000E9144091EA145091EB14A5966CAD7DADA8
:100E20008EAD9FADA5970F94A51B6FA778AB89AB2F
:100E30009AAB2091EC143091ED144091EE14509146
:100E4000EF14A9966CAD7DAD8EAD9FADA9970F94B3
:100E5000A51B4B015C012091F0143091F1144091DD
:100E6000F2145091F314AD966CAD7DAD8EAD9FAD87
:100E7000AD970F94A51B6B017C012FA538A949A93B
:100E80005AA9CA01B9010F9408156FA778AB89ABAD
:100E90009AABA5019401C501B4010F9408159B01FB
:100EA000AC016FA578A989A99AA90F94A61B4B013B
:100EB0005C01A7019601C701B6010F9408159B01BB
:100EC000AC01C501B4010F94A61B0F94541E6B0115
:100ED0007C012091F4143091F5144091F614509156
:100EE000F71469966CAD7DAD8EAD9FAD69970F948B
:100EF000A51BA70196010F94A01C6B017C01F801B2
:100F0000E25BFF4F608371838283938320E030E054
:100F100040E450E40F94061E181624F4EBA1FCA143
:100F200010822BC0E091CB0D24E0E29FF001112450
:100F3000ED55F34F2081318142815381C701B601C4
:100F40000F9408159B01AC0160919F0C7091A00C4F
:100F50008091A10C9091A20C0F94A01C2BA93CA9EC
:100F60004DA95EA90F9408150F94191D64157505F8
:100F70008605970510F42B013C0180919B0C909104
:100F80009C0CA0919D0CB0919E0C2996EEADFFADEE
:100F90002997818C928CA38CB48C258D368D478DAE
:100FA00050A12BA33CA34DA35EA321A132A143A139
:100FB00054A12FA738AB49AB5AAB2FA138A549A5EF
:100FC0005AA582179307A407B50708F4ADC08BADE7
:100FD0009CADADADBEAD892B8A2B8B2B61F16091A1
:100FE0008B0C70918C0C80918D0C90918E0C6415F3
:100FF000750586059705F8F42FA138A549A55AA5CA
:101000000F94E81A6B017C012BAD3CAD4DAD5EAD8C
:10101000C301B2010F94E81AC616D706E806F9060E
:1010200050F4C701B6012BAD3CAD4DAD5EAD0F9494
:10103000F81A29013A0181149104A104B10441F183
:1010400060918F0C7091900C8091910C9091920C0A
:101050006415750586059705D8F42FA138A549A50F
:101060005AA50F94E81A6B017C01A5019401C301F4
:10107000B2010F94E81AC616D706E806F90640F43E
:10108000C701B601A50194010F94F81A29013A018C
:101090002BA13CA14DA15EA1232B242B252B61F17B
:1010A0006091930C7091940C8091950C9091960C9A
:1010B0006415750586059705F8F42FA138A549A58F
:1010C0005AA50F94E81A6B017C012BA13CA14DA1FC
:1010D0005EA1C301B2010F94E81AC616D706E8064E
:1010E000F90650F4C701B6012BA13CA14DA15EA1A8
:1010F0000F94F81A29013A018FA598A9A9A9BAA9AC
:10110000892B8A2B8B2B09F40AC16091970C709163
:10111000980C8091990C90919A0C64157505860530
:10112000970508F4DDC0FBC02BAD3CAD4DAD5EAD09
:10113000232B242B252B09F43FC060918B0C70913D
:101140008C0C80918D0C90918E0C64157505860524
:10115000970590F50F94A7142FA938AD49AD5AAD56
:101160000F9408156B017C016BAD7CAD8DAD9EAD10
:101170000F94A7146FA378A789A79AA7C301B201F8
:101180000F94A7142FA138A549A55AA50F940815A7
:101190009B01AC01C701B6010F94A21487FF0CC0DC
:1011A0002FA138A549A55AA5C701B6010F94A01CC7
:1011B0000F94191D2B013C0181149104A104B10469
:1011C000B9F160918F0C7091900C8091910C90917D
:1011D000920C641575058605970550F50F94A714B4
:1011E0002FA938AD49AD5AAD0F9408156B017C019C
:1011F000C501B4010F94A7144B015C01C301B201F6
:101200000F94A714A50194010F9408159B01AC013C
:10121000C701B6010F94A21487FF0AC0A50194016B
:10122000C701B6010F94A01C0F94191D2B013C019E
:101230008BA19CA1ADA1BEA1892B8A2B8B2BC9F1BF
:101240006091930C7091940C8091950C9091960CF8
:10125000641575058605970560F50F94A7142FA9E9
:1012600038AD49AD5AAD0F9408156B017C016BA1E7
:101270007CA18DA19EA10F94A7144B015C01C30119
:10128000B2010F94A714A50194010F9408159B01B6
:10129000AC01C701B6010F94A21487FF0AC0A501D3
:1012A0009401C701B6010F94A01C0F94191D2B01C6
:1012B0003C012FA538A949A95AA9232B242B252B5A
:1012C00071F16091970C7091980C8091990C9091AC
:1012D0009A0C641575058605970508F479C61FC034
:1012E0002FA138A549A55AA50F94E81A6B017C01D6
:1012F0002FA538A949A95AA9C301B2010F94E81A28
:10130000C616D706E806F90650F4C701B6012FA5A0
:1013100038A949A95AA90F94F81A29013A0184E673
:10132000829D8001839D100D11240E5E174EF801E1
:10133000E25AFF4F4082518262827382C301B2013E
:101340000F94A7142BA93CA94DA95EA90F94A01C2A
:101350006FAB78AF89AF9AAFD80151966D937D93FB
:101360008D939C935497F801E95BFF4F808188230C
:10137000B1F17801B8E4EB0EF11CA091CB0DE4E0E3
:10138000AE9FD0011124AD55B34FF801E25BFF4F82
:1013900020813181428153816D917D918D919C910C
:1013A0000F9408152FA938AD49AD5AAD0F94081503
:1013B00020910C0D30910D0D40910E0D50910F0D9F
:1013C0000F9408159B01AC0160E074E284EF99E48E
:1013D0000F94A01C0F94191DD7016D937C9329893C
:1013E0003A894B895C896BA57CA58DA59EA50F9438
:1013F000081561966CAF7DAF8EAF9FAF61972D8959
:101400003E894F89588D6BA57CA58DA59EA50F940F
:10141000081565966CAF7DAF8EAF9FAF6597298D30
:101420003A8D4B8D5C8D6BA57CA58DA59EA50F94EB
:101430000815A1966CAF7DAF8EAF9FAFA1972D8D94
:101440003E8D4F8D58A16BA57CA58DA59EA50F94B3
:101450000815E1966CAF7DAF8EAF9FAFE197BFAD42
:10146000BB2309F490C2E091D414EBA3F091D514FE
:10147000FBA72091D6142FA33091D7143FA72DEBB3
:1014800037E346E855E3BF018FA19FA50F94A2144F
:1014900087FD79C28090AB0C9090AC0CA090AD0C05
:1014A000B090AE0CC090AF0CD090B00CE090B10CEE
:1014B000F090B20C8091B30C9091B40CA091B50C4B
:1014C000B091B60C8BAF9CAFADAFBEAF2091B70C57
:1014D0003091B80C4091B90C5091BA0C2BAB3CAB8D
:1014E0004DAB5EABC501B401905861962CAD3DADDE
:1014F0004EAD5FAD61970F9408152B013C01C701FC
:10150000B601905865962CAD3DAD4EAD5FAD65977B
:101510000F9408159B01AC01C301B2010F94A61BE7
:101520002B013C016BAD7CAD8DAD9EAD9058A1966D
:101530002CAD3DAD4EAD5FADA1970F9408159B014D
:10154000AC01C301B2010F94A61B2B013C016BA996
:101550007CA98DA99EA99058E1962CAD3DAD4EADCC
:101560005FADE1970F9408159B01AC01C301B20177
:101570000F94A61B2B013C012FEE3FEF4FE75FE3DB
:101580000F94061E18160CF4CFC12FEE3FEF4FE755
:101590005FEBC301B2010F94A21487FF08C05FEE96
:1015A000452E55245A945FE7652E5FEB752EA501F5
:1015B000940161966CAD7DAD8EAD9FAD61970F943A
:1015C000A51B23966CAF7DAF8EAF9FAF239769832A
:1015D0007A838B839C83A701960165966CAD7DAD64
:1015E0008EAD9FAD65970F94A51B27966CAF7DAF11
:1015F0008EAF9FAF27976D837E838F8398872BADA8
:101600003CAD4DAD5EADA1966CAD7DAD8EAD9FADEB
:10161000A1970F94A51B2D966CAF7DAF8EAF9FAF9A
:101620002D9769877A878B879C872BA93CA94DA921
:101630005EA9E1966CAD7DAD8EAD9FADE1970F9447
:10164000A51B6BAB7CAB8DAB9EAB6D877E878F870D
:10165000988BAE014F5F5F4F5CAF4BAFCE014196B1
:101660009AA389A38A01C12CD12C7601D8018D902F
:101670009D90AD90BD908D0120E030E0A901C501A5
:10168000B4010F94A214882371F0A5019401C5013F
:10169000B4010F9408159B01AC01C701B6010F946A
:1016A000A61B6B017C01E9A1FAA1E017F107F1F695
:1016B000C701B6010F94541E9B01AC0160E070E0BD
:1016C00080E89FE30F94A01C6B017C019B01AC019F
:1016D00023966CAD7DAD8EAD9FAD23970F9408150D
:1016E00069837A838B839C83A701960127966CADCF
:1016F0007DAD8EAD9FAD27970F9408156D837E83CA
:101700008F839887A70196012D966CAD7DAD8EAD28
:101710009FAD2D970F94081569877A878B879C87D3
:10172000A70196016BA97CA98DA99EA90F94081504
:101730006D877E878F87988B0CEE1CE0FFA9FBAB33
:1017400028AD2FAF39AD24963FAF24974AAD2A96E6
:101750004FAF2A97ABADBCADCD90DD90ED90FD9035
:10176000BCAFABAF20E030E0A901C701B6010F94D8
:10177000A214882371F1F8016081718182819381C3
:101780000F94A714A70196010F94A01C6B017C0174
:1017900020E030E0A9010F94061E87FF04C0F7FA8D
:1017A000F094F7F8F0942BA93FAD24964FAD249711
:1017B0002A965FAD2A97C701B6010F94A21487FF3E
:1017C00008C0CBAADFAE2496EFAE24972A96FFAED0
:1017D0002A970C5F1F4F29A13AA14BAD5CAD24178E
:1017E000350709F0B7CFA301920160E070E080E80F
:1017F0009FE30F94A51B20E030E040E05FE30F94EF
:1018000008150F94541E6B017C012091870C3091B8
:10181000880C4091890C50918A0C6BA97FAD24965D
:101820008FAD24972A969FAD2A970F940815A7018C
:1018300096010F9408154B015C01A701960160E029
:1018400070E080E89FE30F94A51B9B01AC01C501EC
:10185000B4010F94A01C7B018C0184E6829DF001F1
:10186000839DF00D1124EE5EF74E85849684A78447
:10187000B08820E030E040E85FE3C501B4010F9498
:10188000A21487FF57C0A3019201C301B2010F94B4
:10189000081523EC38EB42E35FEB0F94081523EFB8
:1018A00036E64FE55FE30F94A51BA30192010F9469
:1018B00008152BED3FE049EC5FE30F94A61B2CEEDF
:1018C00031E548E35EE30F94A51B2B013C0124EEB8
:1018D0003BEC46E150E40F94061E18165CF5A3019C
:1018E00092016BED7FE089E490E40F94A51B9B01CE
:1018F000AC01C501B4010F94A01C2BA93FAD2496E7
:101900004FAD24972A965FAD2A970F9408155B0177
:101910006C019B01AC01B701C8010F94061E18169B
:101920004CF47501860106C03BE0E32E47EDF42E32
:1019300003E21BE384E6829DF001839DF00D1124F8
:10194000EE5EF74EA180B280C380D4809501A601DF
:101950006BA17BA58FA19FA50F94061E181624F4DA
:10196000ABA2BBA6CFA2DFA62BA13BA54FA15FA533
:10197000B701C8010F94A21487FF09C0EBA2FBA610
:101980000FA31FA704C01BA21BA61FA21FA6619620
:101990008CAD9DADAEADBFAD61978093AB0C909318
:1019A000AC0CA093AD0CB093AE0C65962CAD3DADD8
:1019B0004EAD5FAD65972093AF0C3093B00C409364
:1019C000B10C5093B20CA1968CAD9DADAEADBFAD38
:1019D000A1978093B30C9093B40CA093B50CB093E3
:1019E000B60CE1962CAD3DAD4EAD5FADE1972093C9
:1019F000B70C3093B80C4093B90C5093BA0C84E6F2
:101A0000829D8001839D100D11240E5E174E8BA1C7
:101A10009BA5AFA1BFA5F80181879287A387B48753
:101A20006FA978AD89AD9AAD90589B01AC010F9428
:101A3000A61B2996AEADBFAD29971D962D913D9160
:101A40004D915C9150970F9408159B01AC016BE090
:101A500077ED83E29BE30F94A51B2BE0C22E27EDCD
:101A6000D22E23E2E22E2BE3F22EF801C582D6829B
:101A7000E782F086B080C180D280E380F480A70145
:101A800096010F94061E87FD02C083E001C081E02D
:101A9000B82A84E6829DF001839DF00D1124EE5E4C
:101AA000F74EB082C092D414D092D514E092D614DE
:101AB000F092D714E5962CAD3DAD4EAD5FADE597F8
:101AC0002093F8143093F9144093FA145093FB14B4
:101AD000E9962CAD3DAD4EAD5FADE9972093FC147A
:101AE0003093FD144093FE145093FF14ED962CADEB
:101AF0003DAD4EAD5FADED972093001530930115D0
:101B000040930215509303156D962CAD3DAD4EAD2F
:101B10005FAD6D972093041530930515409306151E
:101B200050930715A5962CAD3DAD4EAD5FADA59775
:101B30002093E8143093E9144093EA145093EB1483
:101B4000A9962CAD3DAD4EAD5FADA9972093EC1499
:101B50003093ED144093EE145093EF14AD962CADEA
:101B60003DAD4EAD5FADAD972093F0143093F114C1
:101B70004093F2145093F31469962CAD3DAD4EADE5
:101B80005FAD69972093F4143093F5144093F614E5
:101B90005093F7142091D2149091D314291302C0BA
:101BA0008093CF14EE968FADEE978F5F8F708093FA
:101BB000D2148091D2149091D11481508F708917D2
:101BC00009F492C0F090D2148FEF8F0D8F708BA319
:101BD000B090D1148091D214B81609F45CC0C12C15
:101BE000D12C3BA13B1509F456C0632E712C44E661
:101BF000469D8001479D100D11240E5E174ED801A1
:101C00008C9183FD2FC00FAB66961FAF66970115B1
